:10000000F01F001041C000003DC000003DC00000D6
:100010003DC000003DC000003DC0000000000000E9
:100020000000000000000000000000003DC00000D3
:100030003DC00000000000003DC000006DB60000A3
:1000400095B6000095B6000095B6000095B6000084
:1000500095B6000095B6000095B6000095B6000074
:1000600095B6000095B6000095B6000095B6000064
:1000700095B600003BC000003BC0000025B4000066
:1000800055B600003DB6000025B600000DB60000D4
:100090003BC000009DB500003BC000003BC000001D
:1000A0003BC000003BC000003BC000003BC0000064
:1000B0003BC000003BC000003BC000003BC0000054
:1000C0000223184A10B5116801240B431360202342
:1000D000154A164811680B431360154B1968014007
:1000E0001960196821431960124B13491A680240BC
:1000F0001A601A6822431A606C22104B1A60104B67
:1001000018680CF0B7F980220E4B120218600E4BE3
:1001100018600E4B20001A6080234022DB051A6015
:1001200010BDC0460480044080800440F8FCFFFFFE
:100130003040044034400440400D030018000040AB
:1001400018000010140000401000004000E100E022
:10015000802208201021094BD20510B511601860CB
:100160000023074814680C4201D0834204D105489B
:1001700098428041404210BD0133F3E7180000402F
:10018000FF0F0000FE0F0000802100222020134BF3
:10019000C90510B55A609A60DA600860104958685D
:1001A000012807D08A4203D1FFF7D2FF002010BDFB
:1001B0000132F4E78A42F7D000211A69013A5868FF
:1001C000FF2801D95868F2E71869904202D01A69ED
:1001D00059690A3158698142F1D1E5E718000010E8
:1001E000FF0F0000F8B5060003250C4B0C4C1F78E0
:1001F0000223A222A361013BE361E318DA77013312
:10020000DE77084BDF77FFF7BFFF0223FF3398420B
:1002100002D0013D002DEBD1F8BDC04678EC0000C6
:10022000180000101B000010064A537BD318D87327
:10023000537B0133DBB253735BB2002B01DA002333
:100240005373704728100010C143094A53699942FB
:1002500009D2591C08185169994200D27047516956
:100260008842FCD8F7E75169C91A8142FBD3F5E708
:10027000180000104023044A11680B431360012248
:10028000024B30331A707047808004401800001011
:10029000084B70B530331B7804000D00002B01D1E2
:1002A000FFF7E8FF182223689343236023681D4368
:1002B000256070BD180000100E4B70B530331B78F0
:1002C00006000D001400002B01D1FFF7D3FF701EB4
:1002D00002280AD8084B8000C25801231168AB409D
:1002E000012C04D10B43136070BD044AF5E7994318
:1002F0001160F9E71800001080EC0000FC3F00508E
:100300000F4B70B530331B7806000D001400002B26
:1003100001D1FFF7AFFF701E02280BD8094B8000F8
:100320001818C26801231168AB40012C04D10B439B
:10033000136070BD044AF5E799431160F9E7C046C0
:100340001800001080EC00000080005010B50C4C2C
:10035000606B002806D00220FFF744FF0238FF3808
:1003600043425841230038331A780A235106490F73
:100370004B430F210A4048349B186370E07110BD55
:1003800018000010F8B505000E000324A227094B41
:10039000B21C9A610022DA610133DF770133DD7725
:1003A000FFF7F2FE0223FF33984202D0013C002CFB
:1003B000EDD1F8BD1800001010B50120FFF712FFB5
:1003C0000223FF33984210D1094B01201A00383222
:1003D00014785863220706D0032203332240DA77C9
:1003E0000100FFF7CFFF200010BD01246442FAE7AF
:1003F0001800001070B50D4C636B002B13D0D5B2F4
:10040000E31CDD77130A251DDBB2EB77130CDBB29F
:10041000651D120E0634EB77E277FFF7B3FF023863
:10042000FF3843424341180070BDC0461800001019
:1004300010B5FFF7C1FF0220FFF7D4FE0223FF3300
:10044000984220D1104B1A00383212787F2A15D9E1
:100450005A6B002A12D01A000021082001242232EF
:100460009070D47051701170142226330638D970F0
:1004700018705C709A700731FFF784FF034A0421FB
:100480000920FFF7B7FF10BD1800001080808080A2
:10049000012210B510000B21FFF732FF00220B21C3
:1004A0000120FFF709FF012202210320FFF728FFA7
:1004B000002202210320FFF7FFFE10BD70B50600E9
:1004C0000024064D1835605D054B3100C01801341D
:1004D000FFF7DEFE0A2CF6D170BDC04680EC0000AE
:1004E00000400440F8B500240C4D22352B19665D00
:1004F0005F78012239003000FFF702FF023400224A
:1005000039003000FFF7D8FE142CEFD10020FFF7A0
:10051000D5FF0022024B5A65F8BDC04680EC0000B2
:1005200018000010F0B50125734B85B000900C0049
:100530009D6572B68022714B1202DA676C2200262A
:100540006F4B70481A60704B1968014019601A6847
:1005500004211A606D4B1A6802401A601A68002064
:100560001A602A00FFF7CCFE2A0004210020FFF7C2
:10057000A3FE2A0005210020FFF7C2FE2A00052164
:100580000020FFF799FE624B624D1E60FFF7AAFF45
:1005900031006148FFF77CFE31006048FFF778FECC
:1005A00031005F48FFF774FE31005E48FFF770FED0
:1005B00031005D48FFF76CFE5C4B1A685C4B1A60BB
:1005C000009B5A1E93413F225B429343594A9B181A
:1005D000594A13600423594A11680B431360584B5E
:1005E0002E601A685749584E0A401A602A680193CB
:1005F000A30700D47BE0EC235B0113432B60802333
:100600003360DB1833608023DB00336080235B01C1
:10061000336080231B013360009B002B52D00024E9
:100620004A4B4B4F1C604B4B21001C603800FFF7BE
:100630002FFE220009212000FFF762FE220009217F
:100640002000FFF739FE8021434A444813680B43DA
:10065000136007223B68763993433B603B68053A59
:1006600013433B60009B58430BF00CFD03223C4BB3
:100670003C4918603C4B01981C603C4B1A603C4B59
:100680001A680A4080211A601A680A431A60802397
:1006900080229B0052023360326002687E391A4326
:1006A00002602A6813432B600123324A1360324AE6
:1006B0001160324A254913601460136010681842B3
:1006C000FCD00B6001222E4B52421A600A4BDB6DAC
:1006D000039362B630BFC046074B039ADB6D9A4264
:1006E00000D130BF0023044A936505B0F0BD8023DC
:1006F0001B0113432B608CE71800001004E100E09D
:1007000018000040F8FCFFFF304004403440044033
:100710000480044004820440084004400040044037
:10072000AC400440144004401C4004403882044063
:1007300034820440FF1800003082044010ED00E0D5
:10074000008204407FE2FFFF00E100E004C00040BF
:10075000644004400400014080800440841E000086
:1007600018C000400FF0FFFF08C0004014C0004058
:100770003CC0004078800440708004407480044095
:1007800008820440F7B50F4D6C6D002C18D1102075
:10079000FFF794FE0C4B22330193019B0022E65C91
:1007A0001B195F7830003900FFF7AAFD02340122DF
:1007B00039003000FFF780FD142CEED101236B656A
:1007C000F7BDC0461800001080EC000070B572B68E
:1007D00080248020802180250F4BC0001A1D6400DA
:1007E0004901D567D467D067D167C02252009D50B8
:1007F0009C5098509950094A094913680B4013605E
:10080000AC22084B52011A60FFF7BCFF0022064BD6
:100810001A6662B670BDC04600E100E00482044082
:100820007FEAFFFF0882044018000010F8B50700B7
:10083000FFF7A8FF002F09D0012207210220FFF7B0
:100840005FFD002207210220FFF736FD124E330024
:1008500030331B78002B01D1FFF70CFD0F4D012425
:100860002B681B0509D530363378002B01D1FFF7F3
:1008700001FD01242B68DB0A9C43002F09D00022D4
:1008800007210220FFF73CFD012207210220FFF78C
:1008900013FD2000F8BDC04618000010FC3F0050BA
:1008A000F0B5012089B0FFF7C1FF012304930028B0
:1008B0004FD104001D0004902A4E630001330393BE
:1008C000330037002233E25C1B195B780192190078
:1008D0002A0001980293FFF713FD00220299019864
:1008E000FFF7EAFC204B343630333C37069607934B
:1008F0003B787E780593079B1B78002B01D1FFF78F
:10090000B9FC059B032B0DD818000BF09DFE0225AA
:100910002729164B2A00B2401B6813405A1E9341E8
:10092000002B02D16B461B7B0493039B023F0133D8
:100930000393069B9F42DBD1002202990198FFF7A7
:10094000DFFC02342A0002990198FFF7B5FC142C51
:10095000B2D1049809B0F0BD054BDBE7054BD9E7F0
:10096000054BD7E780EC000018000010FC3F00505A
:10097000FC3F0150FC3F0250FC3F0350F8B54A00D9
:10098000070004001E48520D1518132D18DC002D09
:1009900009DACB0FDB070022691C01D119490B438F
:1009A0001900100017E0184E2E4132000A4014437F
:1009B00012D0802212032A415318B3430022EFE7DA
:1009C000332D0BDD8023DB009D4205D13A000B0067
:1009D00038000CF0CFFB07003800F8BD01260B48AB
:1009E00076421218D6403E42F6D03322551B323A98
:1009F000AA40D219BA42A44164420B19B243CFE7CC
:100A000001FCFFFF0000F03FFFFF0F00EDFBFFFFC9
:100A100007B5002200280CD090231B0600920193FA
:100A200000980199802300225B050DF0C9FA03B0FC
:100A300000BD80235B05F1E707B5002200280CD03C
:100A4000F0231B060092019300980199E0230022F5
:100A5000DB050DF0B5FA03B000BDE023DB05F1E7DF
:100A6000F0B5D34A4B0089B007000E000C005B08BC
:100A700093423CD9CF4A934200D8F5E1CE4A934203
:100A80000DD90B031B0B034304D002000B000CF029
:100A900071FB0EE000290EDA0027C84E0BE0C84AB1
:100AA000C84B0BF005FE002800D1DDE10020FFF768
:100AB000C3FF07000E003800310009B0F0BDC24A84
:100AC000C24B380031000CF055FB002200230BF024
:100AD000DBFD0028E0D1BE4ABE4B380031000DF0EE
:100AE0006FFA002C00DAA8E00024BB4DA7E0BB4A57
:100AF000934200D8C5E0BA4A9342ECD8B94ABA4BFF
:100B0000002900DA8FE00DF0CDFC012304000D0078
:100B10000093B64AB64B02920393029A039B2000BD
:100B200029000DF0BFFC02000B0007000E002000A2
:100B300029000DF0B7FC029A039B0DF0B3FC029064
:100B400003910022A44B380031000DF039FA0490D3
:100B5000059102000B00380031000DF031FA04005D
:100B60000D00A44AA44B0DF02BFAA44AA44B0CF0A0
:100B700001FB22002B000DF023FAA24AA24B0DF03C
:100B800091FC22002B000DF01BFAA04AA04B0CF0A8
:100B9000F1FA22002B000DF013FA9E4A9E4B0DF045
:100BA00081FC22002B000DF00BFA00229B4B0CF075
:100BB000E1FA02000B0006900791049805990DF0E8
:100BC000FFF902000B00002095490DF06BFC0200BC
:100BD0000B0004900591069807990DF063FC049AA8
:100BE000059B06900791380031000DF0E9F90200ED
:100BF0000B0000208B490DF055FC02000B000698FD
:100C000007990CF0D3FD2B0022000DF0D9F9009BC1
:100C1000002B4CD102000B00380031000DF0D0F950
:100C200022002B003AE00CF0A5FA01235B4200936E
:100C300004000D006D4A7C4B6DE700247B4D0200E3
:100C40000B00200029000CF095FA0DF073FF0090C6
:100C50000DF0A6FF634A644B029003910DF0B0F9CA
:100C600002000B00380031000DF01CFC5F4A04004C
:100C70000D00029803995E4B0DF0A2F902900391CA
:100C80004BE700216A4A0091934200D959E7694A2B
:100C9000694B31000CF06EFA02000B000DF002FC03
:100CA00002000B00380031000DF0FCFB01E7029A56
:100CB000039B0DF0F7FB3A0033000DF081F9029A27
:100CC000039B0DF0EFFB2B0022000DF0EBFB009BD4
:100CD00004000D0001330CD102000B00380031007C
:100CE0000DF0E0FB00223C4B0DF06AF900223A4B7C
:100CF000DAE7009B012B26D10022504B380031004F
:100D00000BF0C2FC002811D00022334B3800310018
:100D10000CF030FA02000B00200029000DF0C2FB9D
:100D2000C02300221B060DF04BF9C2E622002B0067
:100D3000380031000DF0B6FB02000B000CF01AFA7F
:100D40000022364BA3E6009B1B050293009B013358
:100D5000392B0FD93A0033000DF0A4FB02000B0031
:100D600000202E490DF09EFB029C00226318190002
:100D70002A4B99E7009B132B62DC8023009A9B038C
:100D800013410020254AD11A009001913A00330006
:100D9000200029000DF086FB02000B00009801994D
:100DA0000DF080FB029C070063181E0083E6C0461E
:100DB00079684340412E8640FFFFEF7F0000F0BF7F
:100DC000EF39FAFE422E864059F3F8C21F6EA50194
:100DD000FE822B654715F73F0000E03F422ED63FCD
:100DE000B1A2F03F0000E0FE422EE63F763C7935AE
:100DF000EF39EA3D2DC3096EB7FD8ABE3952E6864A
:100E0000CACFD03EB7DBAA9E19CE143F8555FE1936
:100E1000A0015A3FF41011111111A13F0000F03F41
:100E20000000084000001840EF39EABD0000E0BFB4
:100E3000FFFF8F3C9C7500883CE4377E0000D0BFEC
:100E400000980E490022091A0B05200029000CF019
:100E500091F902000B00380031000DF023FB002255
:100E6000074B0CF087F99DE7002C00DA27E6054ACE
:100E7000054B380031000DF0A3F835E6FF03000004
:100E80000000F03FFE822B654715F73FF0B54A00A2
:100E90005708914A89B005000C00CE0F97422DD912
:100EA0008E4A974211D90B031B0B034306D0020055
:100EB0000B00280021000CF05DF910E0002E00D09E
:100EC00006E12800210009B0F0BD854A854B0BF0F2
:100ED000EFFB0190002805D00020FFF7ADFD0500D5
:100EE0000C00EEE7804A814B280021000BF0CCFB80
:100EF000002807D00198FFF78BFDF0E77C4B9F425D
:100F000000D89BE07B497C4BF2008F426FD89F1842
:100F10003A6C7B6C280021000DF0C4FA3B6D7C6DAF
:100F2000012502900391AD1B04930594AB1B019323
:100F3000049A059B029803990DF0B4FA05000C0081
:100F40002A002300280021000DF03AF806000F00C7
:100F50006A4A6B4B0DF034F86A4A6B4B0DF0A2FAFB
:100F600032003B000DF02CF8684A694B0CF002F996
:100F700032003B000DF024F8664A674B0DF092FA00
:100F800032003B000DF01CF8644A654B0CF0F2F89F
:100F900032003B000DF014F802000B002800210085
:100FA0000DF080FA0B00020006000F00280021005F
:100FB0000DF006F8019B06900791002B53D180237A
:100FC0000022DB05300039000DF06CFA02000B0046
:100FD000069807990CF0EAFB2A0023000DF062FA4C
:100FE00002000B0000204F490DF05CFA77E79E18D5
:100FF00028004D4A4D4B21000CF0E2FF326E736E1B
:101000000CF0B8F80DF096FD01900DF0C9FD484ABE
:10101000484B06000F000CF0D3FF02000B00280025
:1010200021000DF03FFA444A02900391434B3000F7
:1010300039000CF0C5FF0490059179E7404B9F42C1
:101040000CD8404A404B0CF095F80022354B0BF081
:101050002FFB002805D00022324B2AE70023019302
:101060006EE701906CE7802132003B000020C9054B
:101070000DF018FA02000B00069807990CF096FB89
:1010800002000B00049805990DF00CFA029A039BDC
:101090000DF008FA02000B00002022490DF002FAC0
:1010A0002A4B019A9A4205DB019C0500260573181C
:1010B0001C0006E7FA25AD00AC46019C0022644402
:1010C000260573181900B8235B040CF079FF06E7B6
:1010D00000252C00F5E6C046412E8640FFFFEF7F3D
:1010E000EF39FAFE422E864051302DD5104987C087
:1010F000422ED63FB1A2F03F80EC0000D0A4BE72D9
:101100006937663EF16BD2C541BDBB3E2CDE25AFD3
:101110006A56113F93BDBE166CC1663F3E5555558C
:101120005555C53F0000F03FFE822B654715F73F40
:101130000000E0FE422EE63F763C7935EF39EA3D8D
:10114000FFFFEF3D9C7500883CE4377E03FCFFFF0A
:10115000F0B5BA4B8DB00E00994223DC4B005B0812
:10116000034307D1002200230020B5490CF01EFBE9
:101170000DB0F0BD002906DA02000B000DF092F967
:1011800000220023F2E7AF4B00220CF019FF3623B8
:101190000E005B42AC4A964206DD02000B000BF0EB
:1011A000E9FFE5E70023F5E7A84C321512193603ED
:1011B000A74CD218330B02931C1980235B032340E6
:1011C000A44C029D5C401B159B18254300930022F4
:1011D000A04B29000DF066F9029B060002331B03A9
:1011E0000F001B0B0022022B64DC00230BF046FADD
:1011F000002819D0009B002B00D11CE118000DF035
:10120000CFFC954A954B04000D000CF0D9FE944A92
:1012100006000F00934B200029000CF0D1FE0200C5
:101220000B0030003900BAE78F4A904B300039008C
:101230000CF0C6FE02000B0000208D490DF032F9C3
:10124000320004000D003B00300039000CF0B8FE05
:101250000B000200290020000CF0B2FE009B02905F
:101260000391002B06D102000B00300039000DF075
:1012700019F97DE700980DF093FC774A774B04004D
:101280000D000CF09DFE764A00900191754B2000F8
:1012900029000CF095FE02000B00029803990DF056
:1012A00001F932003B000DF0FDF802000B00009840
:1012B0000199DCE78023DB050BF05CFF02000B00EB
:1012C000300039000CF072FA0490059100980DF08E
:1012D00067FC049A059B06900791100019000CF01A
:1012E0006FFE644A029B944663440B9302000B001A
:1012F000089009910CF064FE04000D005E4A5F4BFB
:101300000CF05EFE5E4A5F4B0BF034FF22002B00B8
:101310000CF056FE5C4A5D4B0BF02CFF22002B00BC
:101320000CF04EFE5A4A5B4B0BF024FF089A099BC7
:101330000CF046FE584A08900991584B20002900AD
:101340000CF03EFE564A574B0BF014FF22002B00C8
:101350000CF036FE544A554B0BF00CFF22002B00CC
:101360000CF02EFE02000B00089809990BF002FF0A
:10137000029A4F4B04009B1A0B9A0D001343002B4B
:1013800034DD00223A4B300039000CF019FE3200F7
:101390003B000CF015FE0290039102000B002000B0
:1013A00029000BF0E7FE049A059B0CF009FE009B58
:1013B00004000D00002B06D102000B0002980399D7
:1013C0000DF070F84FE7244A244B069807990CF06B
:1013D000F7FD234A0090019106980799214B0CF0E4
:1013E000EFFD22002B000BF0C5FE54E702000B00BE
:1013F000300039000DF056F8049A059B0CF0E0FD22
:10140000009B04000D00002B02D102000B002CE712
:10141000114A124B069807990CF0D2FD104A009021
:101420000191069807990F4B0CF0CAFD02000B00C2
:101430002000290033E70020002199E6FFFF0F007C
:10144000000050C300005043FFFFEF7F01FCFFFF8F
:10145000645F09000000F03F0000E0FE422EE63F1E
:10146000763C7935EF39EA3D555555555555D53FBB
:101470000000E03F86EBF9FF44523EDF12F1C23F2D
:10148000DE03CB966446C73F599322942449D23F4A
:10149000935555555555E53F9FC678D0099AC33F9A
:1014A000AF788E1DC571CC3F04FA97999999D93FB1
:1014B00051B80600434218434900C00F4908014390
:1014C0000348401A414201430120C90F401A7047A6
:1014D0000000F07F03004042184349004908C00F54
:1014E00008430249081AC00F7047C0460000F07F49
:1014F000564BF0B51A0085B005000C000A409A4220
:101500000FD102000B000CF05BFD02000B00280065
:1015100021000BF02FFE05000C002800210005B073
:10152000F0BD0200002910DC4B005B080343F4D03F
:101530000020814200D180E00B0028000CF0B2FFB7
:1015400002000B000CF032F9E5E7081575D0404BAE
:101550000903C0188023090B5B031943C30703D594
:10156000D30F4900C91852000024431049000393C7
:10157000D30FCB188021162520005200890346186E
:101580009E4202DC70189B1B6418D60F5B00013D65
:101590009B1952004908002DF1D1202680272900EF
:1015A00001963F067E19B446834202DC14D196426E
:1015B00012D865466646ED190290002E03DAEE4316
:1015C000F60F861902961B1A6245804140421B1A8B
:1015D0006046121A0298C919D60F5B00F318019ED3
:1015E0005200013E7F080196002EDBD1134303D049
:1015F0004B1C27D131000134164B6010C01849082C
:10160000E30702D580231B061943039B0D001C052D
:1016100023181C0081E7D10A153B52050029FAD096
:101620008024640321420AD020241600241AE640B4
:10163000451E82403143581B89E70023EEE74900ED
:101640000130EFE7012301319943D5E70000F07F36
:1016500001FCFFFF0000E03FF0B54F005E008DB0E1
:101660007F087608B74205DA3C0037002600040000
:1016700010002200330000920193F0223900040090
:101680003D00BB1B9204934206DD009A019B0BF0C8
:1016900071FD04000D0017E0804B9F4200DCA1E0CB
:1016A0007F4B9F4214DD3F033F0B074305D0009A59
:1016B000019B0BF05FFD04000D007A4B5E40009B28
:1016C0001E4301D1009C019D200029000DB0F0BDFA
:1016D000754BF618FF18009A019B33000092019396
:1016E00096233D009B000893704B9E421BDC704B81
:1016F0009E4200DD78E0009B3343E5D000980199DD
:1017000000226C4B0CF05CFC002200900191694BB4
:10171000200029000CF054FC674A040094460D0098
:10172000089B63440893009A019B200029000CF059
:10173000B9FE0200099102900B00049100980199F2
:101740000AF0A2FF002200285ED03B001000390002
:1017500016000CF035FC009B049005919C46009A05
:10176000019B8020614600068446029101996144F4
:101770000391029803990CF023FC32000090019130
:101780003B00200029000BF0F5FC32000290039191
:101790003B00200029000CF085FE02000B0002989F
:1017A00003990CF00DFC02000B00009801990CF05D
:1017B00079FE02000B00049805990CF073FEFFF708
:1017C00097FE089B04000D00002B00D17CE7002051
:1017D0003A4A1B0599180B000200290020000CF062
:1017E000EFFB56E700237EE79623354A9B05944698
:1017F000FF18F618089B3D0063440893009A019B6C
:101800003300009201938EE7330080210692079304
:10181000002249037B180698079916001F000CF058
:10182000CFFB0A900B918020000684460299049B0E
:1018300004910999029A61440591049805990CF064
:10184000BFFB2200029003912B00200029000BF027
:1018500091FC32003B000CF025FE009A019B0CF03D
:10186000AFFB069A079B04000D00009801990CF04D
:1018700019FE32003B000CF0A3FB02000B0020001D
:1018800029000BF077FC02000B00029803990CF082
:1018900009FE02000B000A980B998EE70000305FEA
:1018A000FFFFEF7F0000F07F000080DAFFFFAF2036
:1018B000FFFF0F000000D07F02FCFFFF0000F03FA1
:1018C000A8FDFFFFF0B589B002920393464A4B0092
:1018D00005000C005B08934203DC0DF02BF9002897
:1018E0004CD02A002300280021000CF069FB0600E0
:1018F0000F0002000B00280021000CF061FB3B4AA6
:10190000009001913A4B300039000CF059FB394AF4
:10191000394B0CF0C7FD32003B000CF051FB374A4D
:10192000374B0BF027FC32003B000CF049FB354AEB
:10193000354B0CF0B7FD32003B000CF041FB334B54
:10194000334A0BF017FC0E9B04900591002B19D124
:1019500002000B00300039000CF032FB2D4A2E4BF8
:101960000CF0A0FD009A019B0CF02AFB02000B007A
:10197000280021000BF0FEFB05000C0028002100D0
:1019800009B0F0BD002202980399244B0CF018FB1B
:10199000049A059B06900791009801990CF010FBA2
:1019A00002000B00069807990CF07CFD32003B000A
:1019B0000CF006FB029A039B0CF074FD154A06001E
:1019C0000F0000980199144B0CF0FAFA02000B007A
:1019D000300039000BF0CEFB02000B002800210084
:1019E0000CF060FDC8E7C046FFFF3F3E7CD5CF5AF4
:1019F0003AD9E53DEB9C2B8AE6E55A3E7DFEB15790
:101A0000E31DC73ED561C119A0012A3F1111813FD5
:101A1000A6F81011495555555555C53F0000E03FF2
:101A2000F8B50022324B0CF0CBFA0022002306005E
:101A30000F000AF023FE002854D100222D4B300065
:101A400039000AF01BFE00284FD132003B00300065
:101A500039000CF0B5FA04000D00274A274B0CF0B2
:101A6000AFFA274A274B0CF01DFD22002B000CF08B
:101A7000A7FA254A254B0BF07DFB22002B000CF02A
:101A80009FFA234A234B0CF00DFD22002B000CF093
:101A900097FA214A214B0BF06DFB22002B000CF032
:101AA0008FFA1F4A1F4B0CF0FDFC22002B000CF09C
:101AB00087FA1D4A1D4B0BF05DFB22002B000CF03A
:101AC0007FFA1B4A1B4B0CF0EDFC22002B000CF0A4
:101AD00077FA194A194B0BF04DFB32003B000CF022
:101AE0006FFAF8BD00200021FBE700201449F8E759
:101AF0000000E03F0000D03F98456D69B8D1B93F84
:101B0000722CC67097F7E63FA79ED5E9358F0E4039
:101B10000CD7D1DD74302E40CB905148830745401F
:101B2000437562CE2C2D53406EAA7567BC66544037
:101B300052BE25E6BCAB4440182D4454FB2119404D
:101B40000000F03FF8B505000C00FFF7B3FC0028DB
:101B500000D0E3E000220023280021000AF094FDD9
:101B600000280BD0280080252D066119FFF7EAFF19
:101B70004919002200230BF0FDFAF8BD00220023D2
:101B8000280021000AF07AFD061E02D00020010084
:101B9000EFE70022644B280021000AF06FFD0028C7
:101BA00000D0BEE00022614B280021000AF066FD53
:101BB0000028EBD15E4A60002300400890420BDD14
:101BC0002A00280021000BF0D5FA02000B000BF0D0
:101BD000EDFD05000C000FE08027E20F2900D20781
:101BE000FF05B84215DC07D1002D12D1D20FD3006A
:101BF000504AD218156F546F00224B4B2800210019
:101C00000AF04CFD002857D028002100FFF708FFFC
:101C1000AFE780241B031B0B64031C43464B0015DA
:101C2000C018464BE318002816D1002B00DA230019
:101C30001C0001200C43D9D0414CA3421ADD414C79
:101C4000A0421DDB3D4C0D001B191A433E4BC01832
:101C5000000502431400CFE7002B05DA6400CB0F28
:101C60001C1949000138DCE71C000C43BED05B00A6
:101C7000CC0FF5E7CD0F5B005B1949000138DCE7BD
:101C8000241A142C0ADC314DE14040191D00854016
:101C900023410D431A43110028009AE71F2C07DC4B
:101CA000E1402A4C001983400B431D001300F1E76B
:101CB0002749081A0341F8E700221C4B280021009D
:101CC0000AF0ECFC002806D02A0023000020174967
:101CD0000CF0E8FB9AE700221E4B280021000AF0D6
:101CE000DDFC002200280AD0280021000F4B0CF058
:101CF000D9FBFFF795FE80231B06C91839E780231F
:101D00002800DB0521000AF0C9FC002800D13DE7CE
:101D100080212A0023000020C905E8E700200E49A1
:101D200027E73000014924E70000E03F0000F03FD2
:101D3000FFFFEF7F80EC000000FCFFFF0000F0FFE2
:101D4000FFFF0F0002FCFFFFFF0300001E04000066
:101D5000E2FBFFFF0000F83F0000F87FF0B587B01E
:101D6000049205934B005B080093009A484B0500D2
:101D70000C009A4204DC0CF0DDFE002800D184E067
:101D80002A002300280021000CF01AF90022414B00
:101D900006000F000CF014F93F4A029003913F4BEC
:101DA000300039000CF00CF93D4A3E4B0BF0E2F9E3
:101DB00032003B000CF004F93B4A3C4B0CF072FB48
:101DC00032003B000CF0FCF8394A3A4B0BF0D2F9E8
:101DD00032003B000CF0F4F8374A384B0CF062FB51
:101DE00032003B000CF0ECF8354A364B0BF0C2F9F0
:101DF00032003B000CF0E4F832003B000CF0E0F85D
:101E0000049A059B06000F00280021000CF0D8F86A
:101E100002000B00300039000CF044FB2A4B009A02
:101E200004000D009A420DDC02000B000298039999
:101E30000CF038FB020000200B0024490CF032FBB0
:101E400007B0F0BD224B009A00269A421BDC13001B
:101E5000204A944663441F0032003B0000201B4987
:101E60000CF020FB320000900191029803993B0096
:101E70000CF018FB22002B000CF014FB02000B00EE
:101E800000980199DAE7144FE6E700200F49D7E7F9
:101E9000FFFF3F3E0000E03FD43888BEE9FAA8BD0E
:101EA000C4B1B4BD9EEE213EAD529C804F7E923EA9
:101EB0009015CB19A001FA3E7751C1166CC1563F5F
:101EC0004C5555555555A53F3233D33F0000F03F93
:101ED0000000E93F0000E0FF0000D23F70B51400B1
:101EE0004A000B00520D0DD14B005B0803430FD08D
:101EF000224B00220CF064F8214B9C4209DA214A63
:101F0000214B17E0214DAA4207D102000BF032F914
:101F100070BD0B004A00520D363A1D4DAC420CDD2F
:101F2000C90F1C48C907084303001B4A19001000C9
:101F3000184B194A0CF044F8EAE7A218174CA242D1
:101F4000EEDC002A05DD164C120523401343190070
:101F5000DEE71400353408DAC90F0B48C907084317
:101F60000300084A19001000C9E70D4C363223401F
:101F700012051A4311000B4B0022DBE7000050430F
:101F8000B03CFFFF59F3F8C21F6EA501FF07000028
:101F900050C300003CE4377E9C750088FE070000BB
:101FA000FFFF0F800000903CF0B54B00394A5B0DFD
:101FB00085B09E180D0004000390132E33DC002E14
:101FC00014DA354A354B0BF0D5F8002200230AF01D
:101FD0006FFB002807D0002D58DA6B005B081C430C
:101FE00001D000242E4D2000290026E02D4F37413E
:101FF0003B000B40034320D000900191264A274B21
:10200000009801990BF0B6F8002200230AF050FB6B
:102010000028E8D0002D03DA80235B033341ED185C
:10202000BD430024DFE7332E09DD8023DB009E4221
:1020300003D102000B000BF09DF805B0F0BD0127A5
:10204000194A7F429B18DF403842F6D00090019138
:10205000114A124B009801990BF08CF800220023D2
:102060000AF026FB0028BED0002D02DA142E02D181
:102070000135BC43B7E734239E1B333BB340E41820
:10208000039B9C429B415B42ED18F2E70024250034
:10209000A9E7C04601FCFFFF9C7500883CE4377E41
:1020A0000000F0BFFFFF0F00EDFBFFFFF0B5D14CCC
:1020B000A54408900991D01E1821140002930AF03B
:1020C000D9F91823421C5B4253431B190024009387
:1020D000029B05905D1EDF1C451BC74BAE00F6182A
:1020E000EC4200D5F1E0A300F0580CF059FDE300FC
:1020F00022AAD318013418605960A742F0DA0024EC
:10210000029BDB00D3180793079B00261D190023B1
:1021100000270693069B089ADB00E91A0839D318B2
:102120001A685B68086849680BF04AFF02000B00F8
:10213000300039000BF01EF8069B060001330693B1
:10214000069A029B0F009342E4D172AB1B1908342C
:102150001E605F60282CD7D10426059BA64A9B00F1
:102160009B180A93370072AAF300D3181C685D68A5
:102170000EA9B3005B1805930B9200229F4B200021
:1021800029000BF01DFF0CF0D5FC0CF009FDBB0085
:102190005B42079300229A4B029003910BF010FFD1
:1021A00002000B00200029000CF07CF90CF0C2FCAE
:1021B000059B079A013F98500B9AFB00D3181A68A9
:1021C0005B68029803990AF0D5FF04000D00002F08
:1021D000D3D1009AFFF782FEFF2300229B05040063
:1021E0000D000BF0EDFEFFF7DFFE0022854B0BF03C
:1021F000E7FE02000B00200029000CF053F90D004F
:1022000004000CF097FC07900CF0CAFC0B000200D5
:10221000290020000CF046F9009B04000D00002B63
:1022200056DD721E92000EAB9B5818211F000098BD
:10223000091A0F410798C0198F40DF1B0EAB9F5042
:102240001723009A07909B1A1F410597059B002BA7
:102250004FDD079B00270133079380235B043A007F
:102260009C4691000EABCB58002F00D0A5E0002B70
:1022700004D06746FB1A0EAFCB51012701329642BC
:10228000EFD1009B002B05DD012B00D19AE0022B42
:1022900000D1A1E0059B022B2BD122002B000020B6
:1022A00059490CF0FFF804000D00002F21D0009ACE
:1022B00000205549FFF712FE02000B002000290004
:1022C0000CF0F0F804000D0013E0002000210EE7F0
:1022D000009B002B06D1731E9B000EAAD758FB153E
:1022E0000593B3E70022494B0AF0ECF9002861D1CD
:1022F000059700220023200029000AF0BFF90028DA
:1023000000D1E0E00022731E0293013B022B00D0BB
:102310006AE0002A00D19BE0009B0EAA183B0093C4
:10232000029B9B009B58002B00D1C8E0009A002024
:102330003549FFF7D3FD06000F00029C002C00DB9F
:10234000FCE00025029B324FDC0072AB1C19029BA3
:102350005B1B00D40AE100263500029C002C00DB48
:1023600029E1059B2900002B02D080231B06E918D8
:102370000B003200099901240A604B604A984B997E
:102380002B000CF08FF8029BA34200DB20E1059BA1
:10239000002B02D080231B06C91802000B00072067
:1023A00009998A60CB60079B034018009B239B0020
:1023B0009D44F0BD022305934BE71648C31A0EA8AF
:1023C0000B505BE7721E92000EAB9B5802935B02B0
:1023D0005B0A0EA98B505DE7721E92000EAB9B58F4
:1023E00002939B029B0AF4E799000EA8091849681A
:1023F0000A438AE794FDFFFFA8F500000000703E45
:1024000000007041000020400000F03F0000E03F6D
:1024100000ED0000FFFFFF0001339A008A1A1269E5
:10242000002AF9D0721C0292069A00249219D20056
:102430000792079922AA8C4662440C92F318F20084
:102440000D920593029B059A934204DD160089E6DE
:1024500001230EA9E1E7079B0A9A1D1922AB5D191A
:10246000029B00269B00D0580CF09AFB00272860A6
:10247000696000250C9B1B190B93089AEB00D1187F
:102480000B9A08684968D31A1A685B680BF098FDC4
:102490000B000200390030000AF06CFE069B01358B
:1024A00006000F00AB42E8D10D9B72AA1B19D3188E
:1024B0009E60DF60029B083401330293C2E7029BF7
:1024C000013B029328E7009B20005A422900FFF7B6
:1024D00005FD0022434B04000D000AF0F3F800282C
:1024E00023D00022404B200029000BF069FD0CF0A6
:1024F00021FB07000CF054FB00223A4B0BF060FD6F
:1025000002000B00200029000BF0CCFF0CF012FBA6
:102510000EABB200D050731C0293009B0EAA18336E
:102520000093029B9B009F5000E7200029000CF0C5
:1025300001FBB7000EABF8500296F7E6E50072AB70
:102540000EAA5D19A30098580CF02AFB32003B003C
:102550000BF036FD002228606960234B3000390003
:102560000BF02EFD013C06000F00E7E600220023E1
:10257000002600920193B54213DBF300F918E3182B
:102580001A685B68086849680BF01AFD02000B00C6
:10259000009801990AF0EEFD013600900191052E98
:1025A000E9D1EB004AAAD31801350099019A083CF9
:1025B00019605A60CBE6E3004AAAD31830001A68C3
:1025C0005B6829000AF0D6FD013C06000D00C5E657
:1025D000E3004AAAD3181A685B680AF0CBFD0134FD
:1025E000D1E6C046000070410000703E49004B0833
:1025F00019007047F7B54B005B080193019A3F4BF8
:102600009A4204DD02000B000BF0DAFC2BE03C4B9D
:10261000019A9A422DDCFFF7E9FFFEF721FA00222A
:10262000384B06000F000AF0A5FD374B019A040055
:102630000D009A4219DD32003B00300039000BF0EA
:10264000BFFC220006000F002B00200029000AF02A
:1026500091FD02000B00300039000BF0A7F80022BA
:10266000284B0AF087FD04000D002000290003B06C
:10267000F0BD264B019A9A4216DCFFF7B7FFFEF732
:1026800005FC0022224B04000D000BF099FC2200F7
:1026900006000F002B0000201D490BF087F80200F8
:1026A0000B0030003900DCE71A4B019A9A4206DC35
:1026B000FFF79CFFFEF7EAFB0022154BA4E7164B41
:1026C000019A9A4205DD154B9A4213D1144A904261
:1026D00010D8FFF78BFF00220D4B0BF071FCFEF7BB
:1026E000D5FB04000D000022094B0BF069FC220011
:1026F0002B0089E70020FEF79FF9B4E7FFFFEF7F8B
:10270000422ED63F0000F03FFFFF7F3CFFFF3540E9
:102710000000E03F412E8640CD338640CE338640D8
:102720007DF8B98FF0B54C4A4E0085B005000C001D
:102730000B007608964208DD02000AF01BFD05003A
:102740000C002800210005B0F0BD0022002944DA69
:10275000424B00920193424B9E424FDC414B9E42C2
:102760000BDC414A414B280021000AF003FD002206
:102770003F4B09F09DFF0028E3D128002100FFF71F
:1027800035FFFEF76DF93B4B04000D009E4226DC41
:1027900002000B000AF0EEFC2200029003912B00D5
:1027A000200029000BF00CFC002206000F00304B2B
:1027B000200029000AF0DEFC02000B003000390086
:1027C0000AF0F4FF02000B00029803990BF06AFE76
:1027D000009A019B0BF0F4FBB1E7274BB9E700220D
:1027E000234B0AF0C7FC02000B00200029000AF06E
:1027F000DDFF22002B000AF0BDFCE9E71F4B9E42E3
:1028000006DC28002100FFF7F1FEFEF73FFBDFE7C3
:102810001B4B9E4205DD1B4B9E4217D11A4A954227
:1028200014D828002100FFF7E1FE0022124B0BF024
:10283000C7FBFEF72BFB04000D0002000B00009805
:1028400001990BF0BDFB22002B00C3E7064A074BA2
:1028500028002100BEE7C046FFFFEF7F0000E0BF79
:10286000FFFF3540FFFF2F3E3374AC3C1F7BAC7F36
:102870000000F03FFFFFEF3F0000E03F412E8640A9
:10288000CD338640CE3386407DF8B98FF7B517003B
:102890001E0004000D00FFF7A9FE00221B4B09F0EB
:1028A000FDFE00280CD020002900FFF7A3FE3860B1
:1028B000796020002900FFF735FF30607160F7BDB7
:1028C00020002900FEF7E2FA04000D0002000B00D0
:1028D00000200E490AF06AFF0022009001910B4B84
:1028E000200029000BF06CFB009A019B04000D00F6
:1028F0000BF0D8FD220030607160009801992B0028
:102900000AF038FC38607960D9E7C0460000E03F43
:1029100082B0F0B58BB00190109211930022129802
:102920001399002309F0AAFE0022002300283ED0BC
:102930001098119909F0A2FE00280CD01298139952
:10294000002200230BF03CFB002200230AF012FCC3
:10295000129C139D19E010981199FFF747FEFEF79E
:10296000C7FD0022002304000D001098119909F002
:102970008BFE00220023002812D0200029000BF03B
:102980001FFB002200230AF0F5FB019B1860596031
:102990009C60DD6001980BB0F0BC08BC02B0184729
:1029A000129813990BF00CFB22002B00CEE7109825
:1029B000119909F063FE002830D012981399FFF79F
:1029C00015FE0022764B0BF0FBFAFEF791FD00227C
:1029D000002305000C000BF0F3FA002206000F00A4
:1029E00012981399002309F063FE32003B0000287F
:1029F00004D0280021000AF0BDFB06E028002100D9
:102A00000BF050FD80231B06E418019B2A00186080
:102A10005960230001998A60CB60BBE71098119937
:102A2000FFF7E4FD00225F4B09F042FE00280AD1C7
:102A300012981399FFF7DAFD00225A4B09F038FE7D
:102A4000002800D175E0109811990022564B0BF028
:102A5000B7FA0022544B04000D00129813990BF0A2
:102A6000AFFA8023002202900391DB0504920593C4
:102A700002980399002200230BF0A2FA22002B00F7
:102A80000AF078FB029A039BFEF7E6FD0022444B16
:102A90000BF096FA002206900791414B2000290086
:102AA0000BF08EFA002206000F00029803993C4BAF
:102AB0000BF086FA002208900991002320002900DB
:102AC00009F0F6FD32003B00002846D00698079931
:102AD0000AF050FBFEF70CFD02000B0006000F0091
:102AE000089809990AF062FEFFF780FD049A059B99
:102AF0000BF066FA32003B0005000C0004980599C3
:102B00000BF05EFA06000F000022002328002100CF
:102B10000BF056FA002204900591029803990023C5
:102B200009F0B2FD049A059B002835D03000390029
:102B300066E70022109811991C4B0BF041FA002215
:102B40001A4B04000D00129813990BF039FAF9236F
:102B50000290039100229B0588E7069807990BF0E5
:102B6000A1FCFEF7C5FC02000B0004000D00089854
:102B700009990AF01BFEFFF739FD049A059B0BF03B
:102B80001FFA22002B0006000F00049805990BF095
:102B900017FA05000C00B7E7300039002BE7C046F4
:102BA0000000E03F000010400000D03F0000504314
:102BB000F0B593B002920393039B0E0002995D005F
:102BC00004930B006D0807002B4319D180210903E2
:102BD000714002000B0092185B419B498B4206D862
:102BE00001D000F0C7FC002A01D100F0C3FC029A1A
:102BF000039B380031000AF0BDFA009001917CE09F
:102C0000924B74000896009064089C469C4207DC36
:102C100001D1002804D1654502DC0CD100290AD07D
:102C20008B4BF3183B43E2D18021039809034840C2
:102C3000029A0300CFE700230693002E17DA854A95
:102C400095424BDC844A954211DD844B2A15D218FB
:102C5000142A23DD3420821A0298D04003009340C6
:102C60008B4204D1012210409218131A06930029B6
:102C70005ED1654521D1764BE3181F4301D100F0A9
:102C800079FC754B9C422BDD049B002B01DA00F094
:102C900075FC029B039C009301942EE0002947D110
:102CA00014239A1A2B00134119009140A94204D110
:102CB000012213409218D31A0693694B9D4220D1EA
:102CC00038003100049B00900191002B15DA3A0086
:102CD0003300002062490AF069FD8EE70223C5E750
:102CE000049B002B01DB00F049FC80221206944675
:102CF000029B0093039B634401930098019913B0D6
:102D0000F0BD8023049ADB059A4206D13A003300D5
:102D1000380031000BF054F96FE7524B049A9A4295
:102D200006D1002E04DB38003100FEF7E1FB64E73A
:102D300038003100FFF75AFC00900191002F2ED18E
:102D4000002C04D0464AB3009B08934227D1049B31
:102D5000002B07DA009A019B002041490AF026FD6A
:102D600000900191089B002BC7DA394BE418069BB1
:102D70001C4308D1009A019B100019000BF092FB34
:102D800002000B00A7E7069B012BB6D1009880211B
:102D9000020001980906431800920193ADE7F20F73
:102DA000069B013A134304D13A0033003800310046
:102DB000E4E7069B013B13430022002B14D0284B71
:102DC000069207938423DB059D4200DC0AE1264B33
:102DD0009D4212DD204B9C4208DC049B002B08DA4C
:102DE0000020FDF729FE08E7204BE9E7049B002BB4
:102DF000F6DC0020FDF70CFEFFE61D4B9C420FDCCD
:102E0000069807990023002209F03EFC431E9841D2
:102E100001244042049B04402000002BEADAE0E752
:102E20000F4B9C4226DD069807990023002209F0EB
:102E30002BFC431E984101244042049B0440200087
:102E4000002BCEDCD6E7C0460000F0FF0000F07F8C
:102E5000000010C0FFFF3F43FFFFEF3F01FCFFFFFB
:102E60000000F03F0000E03F0000F0430000F0BF32
:102E7000FEFFEF3F0098019900224F4B0BF012FB31
:102E8000C0224E4BD20506000F000BF099F84C4AB9
:102E9000049005914B4B300039000BF091F8002263
:102EA00000900191484B300039000BF089F8020086
:102EB0000B00464846490BF0F5FA32003B000BF098
:102EC0007FF802000B00002042490BF0EBFA3200C1
:102ED00004000D003B00300039000BF071F80200D7
:102EE0000B00200029000BF06BF83B4A334B0BF032
:102EF00067F802000B00009801990BF0D3FA02006A
:102F00000B0004000D00049805990AF033F9049AA7
:102F1000059B0020009001910BF0C4FA02000B0009
:102F2000200029000BF0BEFA029C039D002406003D
:102F30000F000298039922002B000BF0B3FA009ABD
:102F4000019B0BF03DF8029A039B04900591300021
:102F500039000BF035F802000B00049805990AF0CF
:102F600009F922002B0002900391009801990BF0BF
:102F700027F806000F000B00020002980399049640
:102F800005970AF0F7F8154B05000C0008919942D7
:102F900000DCCAE2124BCB18034300D1CCE1069807
:102FA00007990023002209F06FFB431E984101247A
:102FB00040420440200014E70000F03F4715F73F6F
:102FC00044DF5DF80BAE543E0000D03F55555555DB
:102FD0005555D53F0000E03FFE822B65FFFF8F4037
:102FE000000070BFBB4B00229C420ADC0098019994
:102FF0000022B94B0AF0E4FF352200900191019CB8
:103000005242B64923155B189B182403B44DB54AA8
:103010000E93230B1D430024934209DDB24A013471
:10302000934205DD0E9B1B1900240E93AF4BED1848
:10303000009801992900AE4AE300D3180F931A6C47
:103040005B6C0C900D910A920B930BF02BFA0C9A7F
:103050000D9B06000F000A980B990AF08BF80200EE
:103060000B0000209E490AF0A1FB10901191020074
:103070000B00300039000AF0A3FF08900991089A6C
:10308000099B802104920593002389056D100D434F
:1030900080210493049A059B009201930022090366
:1030A0006D18A4042B190098019914001D000AF052
:1030B00087FF02000B00300039000BF0F3F90A9A89
:1030C0000B9B06000F00200029000BF0EBF902001B
:1030D0000B000C980D990BF0E5F9009A019B0AF092
:1030E0006FFF02000B00300039000BF0DBF9109A83
:1030F000119B0AF065FF089A099B0A900B9110003A
:1031000019000AF05DFF06000F007A4A7A4B0AF0B8
:1031100057FF7A4A7A4B0AF02DF832003B000AF04A
:103120004FFF784A784B0AF025F832003B000AF04E
:1031300047FF764A764B0AF01DF832003B000AF052
:103140003FFF744A744B0AF015F832003B000AF056
:1031500037FF724A724B0AF00DF8320004000D007E
:103160003B00300039000AF02BFF02000B0020006A
:1031700029000AF025FF009A019B04000D00089821
:10318000099909F0F7FF0A9A0B9B0AF019FF220030
:103190002B0009F0EFFF009A019B0C900D9110009D
:1031A00019000AF00DFF00225E4B04000D0009F02B
:1031B000E1FF0C9A0D9B09F0DDFF049E0F00320029
:1031C0000B00009801990AF0FBFE0022009001918B
:1031D000544B300039000BF065F922002B000BF046
:1031E00061F902000B000C980D990BF05BF9089A3D
:1031F000099B0AF0E5FE320004000D000A980B99C5
:103200003B000AF0DDFE02000B002000290009F05F
:10321000B1FF04000D0002000B000098019909F0B5
:10322000A9FFE022049E12063F4B30000F000AF077
:10323000C7FE08900991009A019B300039000BF0FD
:1032400031F902000B00200029000BF02BF9374A5E
:10325000354B0AF0B5FE364A04000D00354B300000
:1032600039000AF0ADFE02000B002000290009F031
:1032700081FF0F9B1A6D5B6D09F07CFF0A900B912B
:103280000E980BF08DFC04000D00089809990F9B17
:103290001E6E5F6E0A9A0B9B09F06CFF32003B00BA
:1032A00009F068FF22002B0009F064FF0498220057
:1032B0002B00009001910BF0F5F832003B000BF071
:1032C000F1F8089A099B0BF0EDF802000B000A9840
:1032D0000B9927E6FFFF0F000000404301FCFFFFB2
:1032E0000000F03F8E98030079B60B000000F0FF5D
:1032F00000ED0000EF4E454A287ECA3F65DBC993CA
:103300004A86CD3F01411DA96074D13F4D268F51A2
:103310005555D53FFFAB6FDBB66DDB3F0333333322
:103320003333E33F0000084009C7EE3FFD033ADCBA
:10333000F5015B14E02F3EBE924A934B029803992D
:1033400009F018FF3200009001913B002800210095
:103350000BF0A8F802000B000098019909F0A8F9F9
:10336000002800D01BE60021884A63005B0800911A
:10337000934225DD864A1B159B18802252039446F2
:103380001A4114196000834B400D834DC01805414C
:103390002100A9430B0061462403240B214314247C
:1033A000201A0141009108990022002902DA0099AF
:1033B00049420091300039000BF074F804900591F7
:1033C000029A039B04980599002609F0D3FE002277
:1033D000724B30000F000AF0F3FD049A059B089031
:1033E0000991300039000BF05DF802000B000298E3
:1033F00003990BF057F86A4A6A4B0AF0E1FD6A4AF2
:1034000004000D00694B300039000AF0D9FD0200BC
:103410000B002000290009F0ADFE04000D000200A1
:103420000B000898099909F0A5FE089A099B060067
:103430000F000BF037F802000B00200029000BF002
:1034400031F83200029003913B00300039000AF05D
:10345000B7FD04000D00564A564B0AF0B1FD564A1E
:10346000564B0BF01FF822002B000AF0A9FD544A1E
:10347000544B09F07FFE22002B000AF0A1FD524AB6
:10348000524B0BF00FF822002B000AF099FD504A26
:10349000504B09F06FFE22002B000AF091FD020054
:1034A0000B00300039000AF0FDFF04000D0002009F
:1034B0000B00300039000AF083FD80230490059151
:1034C0000022DB05200029000AF0ECFF02000B00BF
:1034D000049805990AF06AF9029A039B04000D000A
:1034E000300039000AF06CFD029A039B09F042FE9D
:1034F00002000B00200029000AF0D4FF32003B003C
:103500000AF0D0FF02000B00002033490AF0CAFF86
:10351000009B1B055B181A15002A29DC009AFEF790
:10352000DDFC069A079BFFF7F5FB2C4A4B005B0876
:10353000934200DC17E72A4BCB1803430CD00698C4
:1035400007990023002209F09FF8431E98410124A7
:103550004042044020004DE432003B000AF0A2FF4C
:10356000029A039B09F0AEF8002800D1FBE6E6E7DB
:103570001900D6E70023184CFFF78DFB0023002429
:10358000FFF789FBFE822B654715973C0000E03F63
:1035900002FCFFFF01FCFFFFFFFF0F00432EE63F91
:1035A000EF39FAFE422EE63F396CA80C615C20BE72
:1035B000D0A4BE726937663EF16BD2C541BDBB3E39
:1035C0002CDE25AF6A56113F93BDBE166CC1663F17
:1035D0003E5555555555C53F0000F03FFFCB904037
:1035E00000346F3FF0B5984B85B04E0004000D00DD
:1035F000039176089E4218DD944B9E4202DC0AD16C
:10360000002808D022002B002000290009F0B2FD7C
:1036100004000D0005E0039B8D4C002B00DC10E145
:103620008C4D2000290005B0F0BD8B4B9E420FDC75
:103630008A4B9E4209DC8A4A8A4B09F09BFD002294
:10364000894B09F035F80028EBD101235B4225E0D6
:10365000FEF7CCFF854B04000D009E4200DDAAE082
:10366000834B9E4200DD90E002000B0009F082FDDA
:1036700000227D4B0AF016FF802306000F00002277
:10368000DB052000290009F075FD0B000200390060
:1036900030000AF08BF8002304000D000293220092
:1036A0002B00200029000AF08BFC02000B00009088
:1036B00001910AF085FC06000F006E4A6E4B0AF07D
:1036C0007FFC6E4A6E4B09F055FD32003B000AF05C
:1036D00077FC6C4A6C4B09F04DFD32003B000AF060
:1036E0006FFC6A4A6A4B09F045FD32003B000AF064
:1036F00067FC684A684B09F03DFD32003B000AF068
:103700005FFC664A664B09F035FD009A019B0AF0A2
:1037100057FC644A00900191634B300039000AF075
:103720004FFC624A624B0AF0BDFE32003B000AF0D9
:1037300047FC604A604B0AF0B5FE32003B000AF0DD
:103740003FFC5E4A5E4B0AF0ADFE32003B000AF0E1
:1037500037FC5C4A5C4B0AF0A5FE32003B000AF0E5
:103760002FFC02000B000098019909F003FD2B00CB
:1037700022000AF025FC029B013343D102000B001A
:10378000200029000AF08EFE42E70022364B0AF0A4
:1037900089FE002206000F00334B2000290009F0AB
:1037A000E9FC0B0002003900300009F0FFFF0123A3
:1037B00004000D0072E7454B9E4219DC0022444B89
:1037C0000AF070FE002206000F00414B2000290085
:1037D0000AF0F6FB0022244B09F0CCFC0B0002009F
:1037E0003900300009F0E2FF022304000D0055E724
:1037F0000B0002003749002009F0D8FF0323040022
:103800000D004BE7029B344FDE00344BBF199E196D
:10381000326973690AF046FE22002B000AF042FE6C
:103820000B000200386F796F0AF03CFE039B040026
:103830000D00002B00DBF4E6802109066B181D004B
:10384000EFE6274DEDE6C046FFFF0F440000F07F96
:10385000182D4454FB21F93FFFFFDB3FFFFF1F3EC4
:103860009C7500883CE4377E0000F03FFFFFF23F8C
:10387000FFFFE53F11DA22E33AAD903FEB0D7624EE
:103880004B7BA93F513DD0A0660DB13F6E204CC58A
:10389000CD45B73FFF8300922449C23F0D55555592
:1038A0005555D53F2F6C6A2C44B4A2BF9AFDDE5209
:1038B0002DDEAD3F6D9A74AFF2B0B33F711623FEAB
:1038C000C671BC3FC4EB98999999C93FFF7F0340EB
:1038D0000000F83F0000F0BF00ED000080ED0000A8
:1038E000FB21F9BFF7B554425E001443484F7608F8
:1038F000E40F00933443BC4209D844424D000443D2
:103900006D08E40F009101902C43BC4203D909F0EB
:1039100031FC03B0F0BD3F4C1C19144302D1FFF73A
:1039200061FEF6E79C17A446022467463C40009FD0
:10393000FF0F3C43019F2F4306D1022C62D0032C82
:10394000E7D135483549E4E73700174305D1009BF7
:103950003148002B59DA3249DBE72D4FBE421BD1EB
:10396000B5420ED1022C06D0032C07D02A48012CD8
:1039700046D12C49CDE72C482C49CAE72A482C4986
:10398000C7E7022C3ED0032CDBD000200021012C05
:10399000BFD180210906BCE71D4FBD42D7D0AD1B6A
:1039A0002D153C2D16DC002B01DA3C3515DB09F01A
:1039B000FDFEFEF71BFEFFF715FE012C10D0022CBA
:1039C00013D0002CA5D01B4A1B4B0AF06BFD124AEA
:1039D0001A4B12E010481A49EFE700200021ECE7EB
:1039E000802424060B19190093E7124A124B0AF09F
:1039F00059FD02000B00084810490AF053FD88E702
:103A0000104986E704480D4983E70D4981E7C04620
:103A10000000F07F000010C0182D4454FB2109C0A5
:103A2000FB21F9BFFB21E9BFD221337F7CD90240C2
:103A30007CD902C0075C143326A6A13CFB210940B7
:103A4000FB21F93FFB21E93F82B0F0B589B00E922E
:103A50000F93019000220E980F99002308F00EFE9C
:103A6000002808D0109811990022704B08F020FE11
:103A7000002800D0CCE00E9A0F9B100019000AF02D
:103A80009FFA0290039102000B00002067490AF0A0
:103A900009FD109A119B04000D00100019000AF096
:103AA0008FFA02000B00200029000AF0FBFC0E9A9E
:103AB0000F9B04000D001000190009F05BFB2200B1
:103AC0002B00FFF70FFF0022594B0AF079FA594AF1
:103AD000594B0490059109F069FE0022002304006F
:103AE0000D0008F0EFFD0022514B002800D18AE0C4
:103AF0002000290009F03EFB00224C4B04000D0081
:103B0000109811990AF0CEFC02000B000AF058FA46
:103B1000029A039B09F02EFB0022002306900791D6
:103B200008F0ACFD002800D072E0290020000BF066
:103B300001F80BF035F8002206000F0010981199DB
:103B40003A4B09F017FB02000B000AF039FA029A0F
:103B5000039B09F00FFB069A079B09F027FEFDF770
:103B6000F7FA0022354B0AF02BFA354A02900391FE
:103B7000344B300039000AF023FAA822069007914E
:103B8000D2052D4B300039000AF01AFA02000B0062
:103B9000049805990AF086FC802204000D00520565
:103BA000294B300039000AF00BFA02000B0020000C
:103BB00029000AF077FC002206000F000298039902
:103BC00000230AF0FDF9069A079B04000D0030005F
:103BD00039000AF067FC02000B002000290009F000
:103BE000C9FA019B002218605960029803990023CA
:103BF00009F0C0FA019B9860D960019809B0F0BC47
:103C000008BC02B01847200029000AF04BFC73E7FB
:103C10000E4B0198196B5A6BDC6B9B6B0160426019
:103C2000029303948360C460E7E7C0460000F03F5E
:103C30000000E03F182D4454FB2109400000D03F14
:103C40006EC0453163626A3C460B213E80ED000048
:103C500082B0D3B5069207930400089A099B069890
:103C60000799FDF7F9FCFDF773FA069A079B009098
:103C7000019108980999FFF735FE002200230600FC
:103C80000F000AF09DF9009A019B09F073FAA660F3
:103C9000E760206061602000D6BC08BC02B0184715
:103CA00082B0F0B593B004001A981B99189219933A
:103CB000002200230AF084F9189A199B09F05AFA95
:103CC00000260200002700200B00454902960397BA
:103CD000049005911A981B99009001910EA808F084
:103CE000FBFC0E9A0F9B08920993109A119B0A9263
:103CF0000B93189A199B1000190009F03BFA1A9AB5
:103D00001B9B0AF05DF90D00079032003B000798FD
:103D100029000AF055F91A9A1B9B06000F00189803
:103D200019990AF0BFFB1A9A1B9B0C900D911898D9
:103D3000199909F01FFA02000B000C980D990AF06E
:103D40003FF932003B0009F015FA02000B00002099
:103D500023490AF0A7FB32003B000AF0A3FB8023B3
:103D60001B06ED180B0007990200019500910EA8A3
:103D7000FEF7CEFD0E9A0F9B0898099909F0FAF903
:103D8000109A119B06000D000A980B9909F0F2F9A0
:103D900032002B00019100900EA8FFF759FF00227E
:103DA000104B0EA804920593802300221B0602925A
:103DB0000393109A119B009201930E9A0F9B08F0A7
:103DC0008BFC0E9A0F9B200022606360109A119B5F
:103DD000A260E36013B0F0BC08BC02B01847C04654
:103DE0000000F03F0000F0BF82B0F0B589B00F9343
:103DF000159B0E9207930600109A119B0E980F992F
:103E0000FDF72AFC00220023149F0290039108F082
:103E100035FC002810D0474B196C5A6CDC6C9B6C3D
:103E200031607260009301943000B360F46009B0B7
:103E3000F0BC08BC02B01847079B10981199069374
:103E40000E9A0F9BFFF74EFD129A139B049005915B
:103E500002980399FEF7ACFE374A0090019104984E
:103E60000599364B09F0A2FC02000B001298139939
:103E70000AF0A6F8002204000D000023380006997D
:103E800008F0FCFB00282AD1049A059B802000063C
:103E900084460799049761440591049805990AF0AE
:103EA0008FF8FCF7F3FF02000B00009801990AF06D
:103EB00087F80090019102980399FDF749F93A00BB
:103EC000069B0AF07DF81C4A1C4B09F06FFC0200AF
:103ED0000B002000290009F04DF904000D0020001E
:103EE0002900FDF72FFE009A019B0AF069F82200D5
:103EF0002B0002900391002011490AF0D3FAFDF73C
:103F000021FE02000B00009801990AF059F80022E6
:103F100004000D000298039900230AF051F80B00E9
:103F200002002900200009F025F9029B039C306063
:103F3000716079E780ED0000182D4454FB210940A1
:103F40000000E03FF0B58FB000934B005B08069394
:103F50000292D34B069A05000C000B919A425DDC4D
:103F60000AF0E8FD0490002800D07CE0149B069A3B
:103F700001332B4313430FD128002100FEF736FBFA
:103F800002000B000020C74909F010FC05000C00DE
:103F9000280021000FB0F0BD149B012BF8D0029A2D
:103FA000009B2800210009F0E5F8020004980B00AE
:103FB000069007910020BC4909F0F8FB2A00089000
:103FC000099106980799089E099F23000AF06AFA4A
:103FD000049E02000B00029800990AF063FA320076
:103FE0003B0009F0EDFF320004000D000698079930
:103FF0003B0009F0E5FF0022AA4B09F0BBF80200E4
:104000000B002000290009F0B5F8089A099B09F077
:10401000D7FF32003B0009F0ADF8B7E7A34B069A93
:104020009A4220DD002907DA802109068C466318B0
:104030001C00009B634400932A0023009C489D4978
:104040000AF030FA06000F00029A009B9A489B493A
:104050000AF028FA3B00320009F08CF80023050032
:104060000C00029300932A0023002800210009F08D
:10407000A7FF02000B000490059109F0A1FF049A2C
:10408000059B06000F002800210009F099FF8C4ACB
:10409000089009918B4B3000390009F091FF8A4A52
:1040A0008A4B09F067F832003B0009F089FF884A23
:1040B000884B09F05FF832003B0009F081FF864A27
:1040C000864B09F057F832003B0009F079FF844A2B
:1040D000844B09F04FF832003B0009F071FF824A2F
:1040E000824B09F047F8049A059B09F069FF804A62
:1040F0000C900D917F4B3000390009F061FF7E4A32
:104100007E4B09F037F832003B0009F059FF7C4A3A
:104110007C4B09F02FF832003B0009F051FF7A4A3E
:104120007A4B09F027F832003B0009F049FF784A42
:10413000784B09F01FF832003B0009F041FF764A46
:10414000764B09F017F802000B000C980D9909F056
:1041500011F8089A099B09F033FF029A009B09F0B5
:1041600009F8049A059B09F02BFF029A009B09F0BD
:1041700001F806000F0008980999694A694B09F08F
:104180001FFF32003B0008F0F5FF02900391020090
:104190000B002800210008F0EDFF444B069A0600B2
:1041A0000F009A423DDD14980AF0FAFC32000090AC
:1041B00001913B003000390009F002FF009A019B99
:1041C000049005913000390008F0D4FF02000B0084
:1041D0000498059909F0EAFA029A039B0AF062F939
:1041E00002000B00280021000AF05CF902000B001D
:1041F00008F0C0FF02000B00009801990AF052F984
:104200000B9B0400981702231840013B181A0D005D
:104210000AF0C6FC02000B002000290009F0D0FEC5
:10422000B4E6149B012B37D000230096019700932E
:10423000009A019B0492059302000B0000201A498A
:1042400009F0B4FA2A000690079104980599069E91
:10425000079F23000AF026F9009E02000B00029837
:1042600003990AF01FF932003B0009F0A9FE320061
:1042700004000D00049805993B0009F0A1FE0022FE
:10428000084B08F077FF02000B002000290008F01F
:1042900071FF069A079BBAE605000C0078E6C04657
:1042A000FFFF2F3E0000F03F0000F0BF2794E53FE6
:1042B000182D4454FB21E93F075C143326A6813CAA
:1042C000D47ABF74702AFB3EE9A7F0320FB8123FD0
:1042D00068108D1AF726303F1583E0FEC8DB573F84
:1042E00093846EE9E326823FFE41B31BBAA1AB3F44
:1042F000735360DBCB75F3BEA69237A0887E143F64
:104300000165F2F2D844433F280356C9226D6D3F40
:1043100037D60684F464963F7AFE10111111C13F1E
:10432000635555555555D53FF0B54B008FB05B08DB
:1043300000931700DA4B009A040007919A4209DCB7
:1043400002000B003A607B6000220023BA60FB6031
:10435000002624E0D34B009A9A4200DD6DE0D24A59
:10436000002935DDD14B0AF09DF8009B04001A00AE
:10437000CE4B0D009A4215D0CD4ACE4B0AF092F8A2
:1043800002000B0020003A607B6029000AF08AF8E6
:10439000C74AC84B0AF086F80126B860F9603000B9
:1043A0000FB0F0BDD322C34B52050AF07BF8C24ACE
:1043B000C24B04000D000AF075F802000B0020004B
:1043C0003A607B6029000AF06DF8BB4ABB4BE1E71D
:1043D000B64B08F0CFFE009B04001A00B34B0D0053
:1043E0009A4214D0B24AB34B08F0C4FE02000B004C
:1043F00020003A607B6029000AF054F8AC4AAD4BCB
:1044000008F0B8FE0126B860F9607642C7E7D3220B
:10441000A84B520508F0AEFEA74AA84B04000D00B9
:1044200008F0A8FE02000B0020003A607B60290023
:104430000AF038F8A04AA14BE2E7A14B009A9A4251
:1044400000DDD0E0FEF7D2F89E4A9F4B04000D003D
:1044500009F0B6FD00229D4B08F08CFE0AF06AFBC5
:1044600006000AF09DFB904A904B0490059109F0DC
:10447000A7FD02000B00200029000AF013F88C4A67
:1044800002900391049805998A4B09F099FD040064
:104490000D0002000B00029803990AF003F81F2E8A
:1044A00028DC8B4A731E9B009B58009A934221D0B4
:1044B00002000B003A607B60029803997B683A68BF
:1044C0000093009B09F0EEFF22002B0009F0EAFFA9
:1044D0000B000200BA60FB60079B002B00DB5EE76D
:1044E000802212069446009B891863447B60B86062
:1044F000F9608AE7009B1B150693069A4B005B0D3B
:10450000D31A102BD4DD04980599D322694B520598
:1045100009F056FD04000D0002000B0002980399FB
:1045200009F0C0FF02000B0000900191029803996E
:1045300009F0B8FF22002B0009F0B4FF04000D00C1
:10454000049805995C4A5D4B09F03AFD22002B0066
:1045500009F0A8FF02000B0004000D00009801996B
:1045600009F0A0FF069A4B005B0DD31A312B08DC33
:1045700002000B003A607B60009A019B0292039359
:104580009AE7B8220498059992054C4B09F018FD5A
:1045900004000D0002000B000098019909F082FF51
:1045A00002000B00029003910098019909F07AFF34
:1045B00022002B0009F076FF04000D0004980599F5
:1045C000444A454B09F0FCFC22002B0009F06AFF2D
:1045D00002000B0004000D000298039909F062FF2D
:1045E0003860796068E73D4B009A9A4208DD020026
:1045F0000B0009F057FFB860F96038607960A7E6F2
:10460000009B374A1B159B18009A02931B05D51A6D
:1046100029000AF08FFA0AF0C3FA02000B0020000A
:1046200029000892099309F03DFF00222D4B09F063
:10463000C7FC04000D000AF07DFA0AF0B1FA02008E
:104640000B0008AEB260F3602000290009F02AFFD9
:104650000022244B09F0B4FC032430617161651E13
:10466000EB00F318186859680022002308F006F8D8
:10467000002813D123003000029A3900FDF716FDFF
:10468000079B0600002B00DB89E680227B68120670
:104690009B187B60FB689B18FB60B6E62C00DEE78E
:1046A000FB21E93F7BD9024000004054FB21F93F48
:1046B0003163621A61B4D03D7370032E8A19A33B33
:1046C000FB21394183C8C96D305FE43F0000E03F02
:1046D00028F50000C14920259A837B39FFFFEF7F31
:1046E000EAFBFFFF0000704130B5204A4B0087B065
:1046F0005B08934206DC0023002200930023FDF7B1
:10470000E1F806E01A4A934205DD02000B0009F0C9
:10471000C9FE07B030BD02AAFFF706FE049C059D46
:1047200003230340012B0AD002980399022B0DD0DA
:10473000002B15D10133009322002B00DFE722006C
:10474000029803992B00FDF709FBE2E70123220001
:1047500000932B00FDF7B6F880231B06C918D8E795
:1047600022002B00FDF7FAFAF6E7C046FB21E93FED
:10477000FFFFEF7F30B51E4A4B0087B05B089342C6
:1047800004DC00220023FDF7E9FA06E0194A93420F
:1047900005DD02000B0009F085FE07B030BD02AA5E
:1047A000FFF7C2FD049C059D03230340012B08D0A5
:1047B00002980399022B0FD0002B12D122002B005C
:1047C000E1E700932200029803992B00FDF77AF8A5
:1047D00080231B06C918E0E722002B00FDF7BEFA74
:1047E000F6E70123220000932B00FDF76BF8D4E7D6
:1047F000FB21E93FFFFFEF7F82B0D0B586B0040018
:104800000C980D990A920B9304AA02ABFEF73EF89E
:104810000A980B99FFF7AEFF029A039B09F0D0FBB1
:1048200006000F000A980B99FFF75EFF049A059B9C
:1048300009F0C6FB002200900191002330003900EE
:1048400009F0BEFB02000B000098019908F092FCF1
:10485000206061602000A660E76006B0D0BC08BCA4
:1048600002B0184782B0D3B50692079304000698A9
:104870000799FCF70BFB06000F0008980999FFF752
:1048800033FF32003B0009F09BFB00900191089838
:104890000999FFF76FFF32003B0009F091FB0022FE
:1048A00006000F0000980199002309F089FB02001F
:1048B0000B003000390008F05DFC009A019B20607D
:1048C0006160A260E3602000D6BC08BC02B018475B
:1048D00082B0F0B50026002797B01D931E9B1F9D48
:1048E0000E9304001C923B0032000E98290006959E
:1048F00007F0C4FE002821D01C981D9932003B000F
:1049000007F0CCFE002819D01C981D99FDF74CFB30
:104910001C9A1D9B07F0B2FE00280FD032003B000E
:1049200000208B4908F042FFA660E76020606160CC
:10493000200017B0F0BC08BC02B0184780231C98B8
:104940001D991B06EB180F930022824B07F09CFE6B
:10495000002854D01C981D997F4A804B09F030FBE9
:104960007D4A06000D007D4B0E98069909F028FB44
:1049700032002B000191009012A8FFF73DFF149A1E
:10498000159B129E139F069207931C9A1D9B002055
:104990006F4909F087FD0B000F99020001910E99F4
:1049A00012A80091FFF794FF149A159B12A8049285
:1049B0000593129A139B02920393069A079B009207
:1049C000019332003B0007F087FE149A159B049276
:1049D0000593129A139B029203930022002312A8BC
:1049E000009201935C4A5D4B08F0EAF8129A139B1F
:1049F00022606360149A159BA260E36098E700222E
:104A00001C981D99524B09F04DFD002200230C9279
:104A10000D93012201254E4B089009910A920B93A8
:104A20004F4B50331093109AEB00D3181E685F68F9
:104A30000E9A069B2800049205930AF0B1F8089A92
:104A4000099B08F097FB002200230290039100923B
:104A5000019312A832003B0008F0B2F8129A139B9F
:104A60000A980B9908F086FB149A159B0A900B91F3
:104A70000C980D9908F07EFB01350C900D910B2DD3
:104A8000D1D1089809990022364B08F073FB002217
:104A9000304B08F06FFB0500109111912E48324900
:104AA000FCF726FD002206000F0008980999294B03
:104AB00008F060FB0E9A069B029003910492059306
:104AC000069B2A0001930E9B12A80093119BFFF7EF
:104AD0008BF91298139932003B0009F071FA3200F9
:104AE00006900791149815993B0009F069FA802205
:104AF000120694460F0006000F9A109B01920E9A20
:104B00006344009212A82A00FFF7ACFE149A159B8A
:104B100012A804920593129A139B00960197029291
:104B20000393069A079B07F0D7FD0C9A0D9B12A8DA
:104B3000049205930A9A0B9B02920393149A159B75
:104B400000920193129A139B07F0C6FD4EE7C046F0
:104B50000000F03F0000E03F182D4454FB210940C5
:104B600080ED000000002240FB211940F7B506004F
:104B70000F0014001D00FCF7ADFC002805D120003B
:104B80002900FCF7A7FC00280BD0200029003200E8
:104B90003B0008F0EFFA04000D002000290003B0EC
:104BA000F0BD22002B003000390007F067FD00281F
:104BB000F3D1002200233000390007F05FFD002808
:104BC0000CD0200029000022002307F05DFD012405
:104BD00000250028E1D080252D06DEE701236A4666
:104BE0003000137039000022002307F061FD002817
:104BF00001D16B4618706A460123127830005A4082
:104C000001926A463900137022002B0007F03CFD28
:104C1000002801D16B4618706B466A461B781279E2
:104C2000934204D001240025A4197D41B5E7012455
:104C30006442E517F8E7F7B5071E21DA124C134D69
:104C400047420022124B01260092019312E03742A4
:104C500007D00098019922002B0009F0B1F90090CB
:104C6000019122002B002000290009F0A9F904007D
:104C70000D007F10002FEAD10098019903B0F0BD1C
:104C80000024044DDDE7C0469A9999999999B93F56
:104C90000000F03F00002440F8B50D0017001E0092
:104CA000040009F047FF386009F07AFF02000B00AA
:104CB0002000290009F0F6FB0022104B09F080F9D2
:104CC00004000D00FBF75AFE09F034FF306009F0D4
:104CD00067FF02000B002000290009F0E3FB00221F
:104CE000074B09F06DF9FBF749FE09F023FF002897
:104CF00000D10130069B1860F8BDC04600408F40CF
:104D00000000594030B50A4B652804DD0322873383
:104D10001A70002030BD000118180930FF300268F9
:104D200043688468C5680A604B608C60CD60F0E7BA
:104D3000A808001070B505000C0000220023280010
:104D4000210007F0A1FC002807D0280080252D06AF
:104D50006119FDF729F9491970BD28002100FDF7F7
:104D600023F9F9E7F7B514001D0000900191002226
:104D7000184B2000290007F087FC002801D00024F0
:104D8000144D0026134F009A019B2000290007F0C4
:104D900085FC002803D13000390003B0F0BD30009D
:104DA000390022002B0009F00BF906000F00FCF778
:104DB00081FB0028EFD130003900FCF78BFB002885
:104DC000E9D1200029000022024B08F0D3F90400A9
:104DD0000D00D8E70000F03FF7B506000D003000E9
:104DE0002900FCF777FB071E51D130002900FCF7A2
:104DF00061FB041E4DD1002200233000290007F082
:104E00003DFC002837D1002200233000290007F0A4
:104E10003BFC002803D080231B06ED18DFE70022AF
:104E20001D4B3000290007F04DFC002815D0002252
:104E30001A4B009201930098019932002B0007F061
:104E400037FC002817D1009801990022134B09F074
:104E5000B7F8013400900191EDE7114C114B00932C
:104E6000019401240098019932002B0007F016FCF0
:104E7000002802D064422000FEBD00980199002263
:104E8000064B08F093FC013400900191EAE70024FE
:104E9000F1E73C00EFE7C0460000F03F000024408F
:104EA0009999B93F9A9999990A4B10B51A007E328F
:104EB0001278002A0BD17F331B780022002B07D0F9
:104EC000054B09F07DF8054A054B08F06FFC10BD55
:104ED000044BF6E7A808001000007940182D445450
:104EE000FB2119400080764010B50122802806D8A9
:104EF000044980004358002B01D09847002210003D
:104F000010BDC04624F30000020008210300012068
:104F1000473A8A43D2B210B5824220D91A000424FB
:104F20006F3AA243D2B2002A19D01A00763A0A2A5E
:104F300015D9402218009043020001202B2A0ED0E0
:104F40009A1F82420BD9073AA243D2B20400002A28
:104F500005D000208B43433BDBB29C42404110BD57
:104F6000F8B501240C4D0D4E2F5D002F06D12B19E5
:104F7000013B1878FFF7C8FF00280AD03800FFF778
:104F8000C3FF431E98410019441CB442ECDDFA24CF
:104F9000E4002000F8BDC046D4000010CF07000098
:104FA00070B504000D00FFF7DBFF154B1A1AAA427B
:104FB00004DA0322134B87331A7070BD9C42FCDC69
:104FC0002919FAD4002DF8D00ADD00210E4BED1876
:104FD000A042F2DBC21816782E5411700138F7E7A0
:104FE000FA2200230848D200121B091824189A42FA
:104FF000E3DDE05CC8540020E0540133F7E7C0462D
:10500000CF070000A8080010D400001070B57C265F
:105010000C4D0D4BAC5B185DFFF776FF002807D0F9
:105020000A4B9C420AD9872303220120EA5470BD0F
:10503000074B9C42F7D80134AC53F8E70234AC5329
:105040000020F4E7A8080010D4000010CD070000ED
:10505000CE070000F7B5114C019123007C331B886B
:105060000F4D0700EA5C002A01D1002B01D1FFF7A8
:10507000CDFF7C3420880121FFF792FF268838007D
:10508000AF55FFF741FF002807D0701C0121FFF743
:1050900087FF2388ED18019B6B70F7BDA8080010EF
:1050A000D4000010F8B506000400064F351B002C94
:1050B00005DD013C385DFFF727FF0028F6D1012010
:1050C0002840F8BDD400001070B50A4E04B223B2D7
:1050D000002B01DC084809E0A5192B782B2B06D101
:1050E0002000FFF7DFFF002801D1687870BD013C88
:1050F000EDE7C046D4000010FFFFFF7FF8B57C2528
:10510000084E745B671E3800FFF7CCFF002805D1FE
:10511000002C01D07753F8BD0120FCE7023C74530A
:105120000020F8E7A808001030B5FA240023084949
:10513000E400CD5C5A1C2B2D04D18D5C854201D13D
:10514000981C30BD1300A242F3D10020F9E7C046FD
:10515000D400001010B5682802D8FFF7E5FF10BD95
:105160000A4BFE280CD1E922D2009B181868596816
:1051700009F0E0FC03004042002BF0DBD8B2ECE782
:10518000032287331A700020E9E7C046A808001000
:1051900083280DD80F290BD88423CA085343181825
:1051A0000723194079330B41024A115C0B43135416
:1051B0007047C046B8100010F0B587B003923C4A63
:1051C0000493D3780C00834204D21378019301989E
:1051D00007B0F0BD002153689278801A1A7888428F
:1051E0001ADC991C5B78009101938B1805930C9B3A
:1051F000002B02D0019BE41A0134049BE5B2002786
:10520000002B1BD10025E4B20295019B029A934228
:10521000DDDD082600273DE002329B180131DDE785
:10522000039B2800F118C9B2FFF7B2FF0136204BEB
:105230005B789E42F4DB01350137EDB2019BBB4246
:10524000E0DD0026F3E7082E08D1059B009A934283
:10525000BDD01300002601331578009301231D42B1
:1052600015D0039BF918049BC9B2002B1CD0832CCA
:105270000DD80F290BD88422CB0853437D3A0A401E
:10528000802111410B481B19C25C8A43C2546D1026
:1052900001370136064B5B789F42D4DB029B013419
:1052A00001330293E4B2B0E72000FFF771FFEEE7AD
:1052B00000000010B810001070B50D0004000122AD
:1052C000FBF71EF8290001222000FAF7F5FF70BD58
:1052D0000122F8B5082107001000FAF7EDFF0724B6
:1052E0000826002231000120FAF7E6FF3A000125E6
:1052F000224102212A400020FAF7DEFF2A00310075
:105300002800FAF7D9FF013CEBD2F8BD002210B516
:10531000040011000220FAF7CFFF2000FFF7D8FFAA
:1053200010BDF7B5012300245026134D00930194BE
:1053300076426A46A300D05800273043C0B2FFF738
:10534000E5FF0020FFF7E2FF1020FFF7DFFFE0207E
:10535000FFF7DCFF012200210220FAF7ADFFE85D34
:105360000137FFF7B5FF842FF4D18435012C00D12C
:10537000F7BD0124DDE7C046B81000107047704744
:105380000122024B80331A707047C046A8080010F3
:10539000054B002219007C310A80190086310A7001
:1053A000A43301321A707047A808001010B5074CDA
:1053B000230085331B78002B03D00C217620FFF7C8
:1053C00049FE0123A434237010BDC046A808001074
:1053D000044B84331A787F2A02D8FF221A70704750
:1053E0000022FBE7A808001010B5064C7C34238887
:1053F000002B02D0FFF782FE10BDFFF7B1FD208029
:10540000FAE7C046A808001010B5074C2300853302
:105410001B78002B03D00B217620FFF71BFE012306
:10542000A434237010BDC046A80800108022024B8F
:1054300052007E331A807047A80800100122024BE8
:105440007E331A807047C046A80800100022024B25
:105450007E331A807047C046A808001070470022AB
:10546000014B80331A707047A80800100122024BCC
:10547000A4331A707047C046A80800100122024BDE
:10548000A4331A707047C046A80800100022054BCC
:1054900084339A56002A02DC01221A7070470022D7
:1054A000FBE7C046A8080010054B00211A00813216
:1054B000117082331A7851424A411A707047C046BF
:1054C000A8080010054B00211A00823211708133A8
:1054D0001A7851424A411A707047C046A808001015
:1054E00070B5114C114923007C331A88885C002860
:1054F00003D1002A01D0188070BD230085331B78AA
:10550000002B02D0FFF782FDF6E725000123863548
:105510002B70FFF7E9FC2B78002B01D0FFF776FD0D
:10552000002386342370E7E7A8080010D400001099
:10553000F0B585B00500019114008A4206DD002215
:10554000002302604360002005B0F0BD1000FFF7AB
:1055500072FB06000F002868696807F0F5FD0290ED
:1055600003913000390007F0D1FD07F0EDFD0B008D
:1055700002000298039908F019F9FBF7FFF907F008
:10558000C5FD019B03C59C4203D10843411E8841D0
:10559000DAE707F0D9FDFFF71FFC019BC1171C1BC1
:1055A000E30FA04259410800CEE773B51D00114B2F
:1055B00014001E001A00B836C8320090019110681D
:1055C0005168306071609068D168B060F1601E0011
:1055D000A833D836306871689C60DD601060516017
:1055E000B068F1689060D1600099019A19605A60C2
:1055F00073BDC046A808001073B514000C4A009093
:10560000019116001D000B4B983618685968103B25
:10561000186259629869D9699862D962B342F4D123
:1056200000980199A8329460D5601060516073BDF4
:10563000A808001070090010F8B51F00074B0400FF
:10564000A4331B780D001600002B05D02000290084
:1056500032003B00FFF7D0FFF8BDC046A80800109D
:10566000D0B5154C154A23000833DB6F13400CD11D
:10567000134AA534516E002902DD21705366D0BD56
:105680002378536604232370F9E7230086331B78BD
:10569000002BF4D00A4B58690A4BE358A434C01AC3
:1056A00009F0B8FA0022084B08F080F80023002225
:1056B000FFF7C2FF0123E6E7A808001000FFFF0084
:1056C000180000107C07000000408F4010B50C4C03
:1056D00000232100A83100228868C96806F0CEFFA7
:1056E00003000120002B09D0B8340023A068E16832
:1056F000002206F0C3FF43425841400010BDC0469F
:10570000A808001070B5FFF7E1FF03000020012B8F
:1057100016D00C4B0022A8331C685D680A4B200091
:10572000290006F0BBFF00280AD0084B0022200009
:10573000290006F0C7FF431E98414342012018404C
:1057400070BDC046A80800100000F03F0000F0BF88
:10575000F8B55F4D2B0087331B78082B07D1FBF77B
:105760009FF80028FBD12B00072287331A70FBF724
:1057700097F8584F0400031EBE6E3FD1032E2DD163
:105780002B0085331B78002B05D12B007A331B7837
:10579000002B00D134002B0081331A78002A03D06B
:1057A000052E01D000221A702B0082331A78002AAD
:1057B00003D0092E01D000221A702B00002284335E
:1057C0009A56002A05D02F2E0FD0572E0DD000222A
:1057D0001A703A2E09D1FFF743FF06E0532E02D18B
:1057E0002B008533D3E7002ED5D12A0000237A324F
:1057F00079351370BB662B70FB663DE02A00813261
:105800001278002A21D02834FB22053B134204D110
:105810002000282106F014FF0C00B44242D1032CD2
:105820002CD12B0085331B78002B15D00025FB6E67
:10583000022B32DD642D1FDC0120FAF705FDFBF79A
:105840002FF8002810D00135F1E72A0082321278B3
:10585000002AD9D05034D7E71F4C0120FAF7F4FCC6
:10586000FBF71EF8002801D1002405E0013C002CC4
:10587000F3D101237A352B702000F8BD532CD5D0FD
:10588000164D0120FAF7E0FCFBF70AF80028EBD0F0
:10589000013D002DF5D1A034EEE7114A9542CBD160
:1058A0000133A9E72B000833DA6F0E4BBC661A42AE
:1058B000E2D1032C01D0532CDED1C820FAF7C4FC6E
:1058C000FAF7EEFF0028CFD0012379352B70CBE714
:1058D000A808001018000010D1070000E90300001C
:1058E0005902000000FFFF00F8B51D4B1A6E002A98
:1058F00035D101321A66FFF72BFF0028FBD172B6B3
:105900008026802180208027164D174A2B6876003C
:1059100013402B60154BC9004001DF67DE67D96774
:10592000D867FAF7DFFD124A0F49136880200B4051
:105930001360AC230F4A5B0113608021C0220E4C20
:105940005200C9004001A750A650A150A0502A689B
:1059500013432B60276026602160206062B6F8BD8B
:1059600018000010048204407FEAFFFF04E100E019
:10597000008204400882044000E100E0F0B585B0F8
:1059800002900C0003921F0006F038FB451E002D0C
:1059900001DB002C01DC05B0F0BD029B2100585D4D
:1059A0000123039A00933B00FFF706FC241A002F03
:1059B00002D1013C013DEAE70026B542F9D0064B91
:1059C0005B789E42F5DA039BE0B29919C9B2FFF702
:1059D000DFFB0136F3E7C04600000010F0B5264DAE
:1059E00085B02C007034200006F008FB0023C2B202
:1059F000A275E37523766376A376E3769A4201D0A7
:105A00000133237670352B782D2B01D12C3BAB76CF
:105A10000022C3B2039316001500140011000123E5
:105A2000029201920398884212DC002D02D0124BA0
:105A30007033DC75002E03D00F4B0199703359760B
:105A4000002A03D00C4B029A7033DA7605B0F0BD11
:105A5000094870300F5C01312E2F07D0452FE1D15E
:105A6000085CCCB201942D2803D01E001D001C0040
:105A7000D8E71A000293F8E7180000107FB51C4C15
:105A80000600230070331B7E002B1DD1194D2B0007
:105A90009C331B78002B17D1174BA835196C5A6C07
:105AA000009101929A6CDB6C009801990292039329
:105AB000029A039BFFF7C0FD009A019B2A606B606E
:105AC000029A039BAA60EB600A4970347831A07D8A
:105AD000E27D0978821A8A4204DB637E002B01D1C1
:105AE000452E02D1024B70331E54FFF777FF7FBD66
:105AF00018000010A808001080ED000010B50B4C35
:105B0000230070331B7E002B06D13120FFF7B6FF38
:105B10000122074BA4331A707034637E002B04D12A
:105B20004520FFF7ABFFA37D637610BD1800001082
:105B3000A808001010B5074B7033DA7D002A08D191
:105B40001B78002B02D13020FFF798FF2E20FFF7A3
:105B500095FF10BD1800001010B53920FFF78EFF1B
:105B600010BD10B53820FFF789FF10BD10B53720E4
:105B7000FFF784FF10BD10B53620FFF77FFF10BD83
:105B800010B53520FFF77AFF10BD10B53420FFF7B0
:105B900075FF10BD10B53320FFF770FF10BD10B5B5
:105BA0003220FFF76BFF10BD10B53120FFF766FF05
:105BB00010BD10B53020FFF761FF10BDF0B5012317
:105BC000050085B02800029306F018FA2B780390A0
:105BD0002D2B09D000240194039B9C4208DB0298E2
:105BE000019B584305B0F0BD029B01355B42E9E7DC
:105BF000039B581E001BFFF71EF806000F00285DD0
:105C00000134303808F0CCFF32003B0008F0D8F9FE
:105C1000060001980F0008F0C3FF02000B003000DF
:105C2000390007F0A7FA08F085FF0190D4E7F0B536
:105C300087B0019006F0E2F9019B03901B782D2BB1
:105C400026D101980130FFF7F2FF80231B06C91807
:105C500007B0F0BD019AD25C2E2A17D0452A00D198
:105C600002930133039A9342F4DB8C4206D1029BE8
:105C7000A34212D1019806F0C1F9040000250026C4
:105C80000027039B9D420ADB002011E01C00E8E78F
:105C9000214C002302942100E4E7029CEEE7029BE2
:105CA000AB420CD11800019B01301818FFF786FF9A
:105CB000FEF7C1FF32003B0008F082F9C8E7AC42B2
:105CC00014DD0022154B3000390008F079F9060088
:105CD0000F00019B585D303808F062FF32003B0036
:105CE00007F048FA06000F000135CAE7AC42FBDABC
:105CF000601BFEF7A0FF019B04900591585D3038B2
:105D000008F04EFF049A059B08F05AF902000B00B8
:105D100030003900E4E7C046E703000000002440FB
:105D2000F0B5060085B00F0006F068F935000024D4
:105D30000390039AAB1B9A4201DD832C01DD05B071
:105D4000F0BD00232878210000933A00FFF734FAD1
:105D5000241801340135ECE7802273B500210725B2
:105D60002B4B2C4C920301912000DA67902206F015
:105D70000DF9019B284EA360284B1A68AA431A60AC
:105D80000122196811431960254B1968A94319604C
:105D9000196811431960802322495B010868034395
:105DA0000B60214B1A6082323260204A12681968F7
:105DB0001F4B1868504306F065F9E121090306F00E
:105DC00061F910221B4B1C491A60030A0B60032364
:105DD0001A4AC0B210603360194B1D60194B593517
:105DE00018680190080011001A682A40602AFBD147
:105DF0005F3A1D68154207D122708022124B920330
:105E00001A600523036073BD0D680195F1E7C04674
:105E100004E100E0281000100C800040A440044081
:105E2000A84004408080044098800440788004406A
:105E300018000010288000400480004000800040CE
:105E4000088000401480004000E100E0FA2110B515
:105E50000C4C8900206806F00DFB0B4B984209D8CA
:105E600000230A4A013863611060094A136007225F
:105E7000084B1A60FFF770FFFAF722F9FAF7D8FA21
:105E800010BDC04618000010FFFFFF0014E000E046
:105E900018E000E010E000E010B5002839D08021C3
:105EA0001D4A13688B43136001231C490A681A4278
:105EB000FCD003221A4B1A6001230021194A1360F7
:105EC0001160136011681942FCD0174A174913601A
:105ED00080230C685B0223430B601100002804D16F
:105EE00080230D4A146823431360114B9A68824241
:105EF0000ED09860431E98410E4B404218400E4B06
:105F00000968C01806F0BEF80C4B1860FFF79EFF3A
:105F100010BD034B1860CFE7388204400C8004406A
:105F20007080044074800440788004408080044085
:105F30000000001000512502001BB70018000010DF
:105F400010B5044816220021703006F01FF8FFF744
:105F500045FD10BD1800001070B5FFF7F1FF084BAC
:105F600008491A000C6C4D6C886CC96CA83214601E
:105F700055609060D1600022A4331A7070BDC04695
:105F8000A808001080ED000070B50E4C23009C3373
:105F90001B78002B14D10C4D7035280006F02EF81C
:105FA00000280DD02800FFF742FE2300A833186018
:105FB000596000220023B03422606360FFF7C0FF05
:105FC00070BDC046A808001018000010F0B589B0D8
:105FD000FFF7DAFF464B5C681B680093019400985A
:105FE0000199434BDC689B6802930394029A039BDC
:105FF000FFF722FB3F4B1C6C5D6C9E6CDF6C20003E
:10600000290032003B00FFF7F7FA3B4B2933FF33FF
:106010001C685D68384B20003933FF331A685B68B1
:1060200000920193344B29004933FF331A685B68AF
:1060300004920593304B00225933FF331E685F688A
:106040002E4B08F02FFA22002B0007F0B9FF2A4B45
:10605000029003916933FF331A685B6820002900BE
:1060600007F0AEFF3200069007913B003000390088
:1060700007F0A6FF02000B000698079908F012FA35
:10608000029A039B07F092FBFBF732FA00260027E7
:10609000194BB83318605960174B2000C0331E608D
:1060A0005F60049A059B290007F08AFF009A019B14
:1060B00004000D001000190007F082FF02000B0021
:1060C0002000290008F0EEF9029A039B07F06EFB0E
:1060D000FBF70EFA0122064B18605960064BB033ED
:1060E0001E605F60044BA4331A7009B0F0BDC04657
:1060F0005009001080ED0000A80800100000F03FDB
:10610000F7B5FFF741FF204C2500A83528686968DE
:10611000AA68EB68FFF790FA1C4B1E6C5F6C9A6CD8
:10612000DB6C00920193009A019B30003900FFF76D
:1061300063FA2300210029335931FF33FF311A68F4
:106140005B682600086849680092019307F02EFBFF
:10615000B8363060716021002300002600273931F5
:10616000C033FF311E605F6008684968009A019B78
:1061700007F01CFB2300B0331E605F600123A434D2
:10618000286069602370F7BDA808001080ED00004A
:1061900070B5FFF7F9FE0B4C2500A835AA68EB682F
:1061A00028686968FFF748FA2300E83319685A68D5
:1061B00029606A609A68DB68AA60EB600123A434F6
:1061C000237070BDA8080010F8B5FFF7DDFE084B7E
:1061D000D8331E685F689C68DD6830002B0039008A
:1061E0002200FFF729FA0123014CA4342370F8BDE3
:1061F000A808001070B5FFF7C7FE0B4C2500A835A6
:10620000AA68EB6828686968FFF716FA074BA43498
:10621000996ADA6A29606A601A6B5B6BAA60EB6044
:106220000123237070BDC046A808001000EE0000D6
:10623000F0B587B0FFF7A8FE484B1C685D68484B77
:1062400020001E685F68474B29007933FF331A68C6
:106250005B6807F0B5FE444B009001911A685B68DB
:106260003000390007F0ACFE02000B0000980199E5
:1062700008F018F93B4B029003914933FF331A6839
:106280005B682000290007F09BFE320004000D002F
:106290003B003000390007F093FE02000B002000A5
:1062A000290008F0FFF82F4E00900191A8363068C1
:1062B0007168B268F368FFF7BFF92C4B1C6C5D6C1A
:1062C0009A6CDB6C04920593049A059B20002900CC
:1062D000FFF792F9009A019B0298039907F066FA7A
:1062E000204C0022B8342060616000211D4BC03377
:1062F00019605A60009801991B4B1A685B6807F097
:106300005FFE174B04001A685B680D000298039942
:1063100007F056FE02000B002000290008F0C2F82A
:106320000E4B04001A685B680D000098019907F095
:1063300047FE02000B002000290007F037FA002278
:10634000306071600021074BB03319605A60012240
:10635000044BA4331A7007B0F0BDC046D00900103A
:10636000E0090010A8080010000A001080ED0000ED
:10637000F8B5FFF709FE0D4C00222500A8352E6860
:106380006F6800233000390007F01AFE02000B008E
:10639000A868E96806F0EEFE2300B0331E605F6077
:1063A0000123A434286069602370F8BDA808001098
:1063B00073B5FFF7E9FD124B1E00A836B168F2680D
:1063C0000091019234687568009801991A00F832BA
:1063D000146055609060D1601A00B832106851683E
:1063E00014605560306071609068D168B060F16091
:1063F000009801999060D1600122A4331A7073BD96
:10640000A8080010F7B5FFF7BFFD144C25002300C6
:10641000F835A83319685A6829606A609A68DB6899
:10642000AA60EB602300B8331E685F689A68DB6877
:1064300000920193009A019B39003000FFF7B5F8F4
:1064400029686A682300D83319605A60A968EA6825
:106450009960DA600123A4342370F7BDA808001006
:10646000D0B52A4C8CB0220083321378002B07D091
:10647000012B03D10B3313700CB0D0BD013BFAE7F5
:10648000FFF782FD2300A83319685A680691079226
:106490009E68DF68069807990022002306F0EEF850
:1064A00000280BD0002200233000390006F0E6F867
:1064B000002803D0873401232370DDE723000699E9
:1064C000079AE83319605A602300F0331E605F605A
:1064D00013000A00029203930022002304960597FA
:1064E0000092019308A80022094B06F069FB089965
:1064F000099A2300A83319605A600A990B9A23005D
:10650000B03319605A60A434D5E7C046A80800101B
:106510000000F03F10B5FFF737FD064B1A00A83317
:10652000E83218685968106051609868D9689060BE
:10653000D16010BDA8080010F7B5FFF7C7F8284EC6
:10654000002803D0022387363370F7BDFFF7E2FF40
:106550003300A836B833776836681C685D68320047
:106560003B002000290007F09DFF009001910200F0
:106570000B003000390006F091F80022194B00287A
:106580002AD00098019906F0F5FD02000B002000CA
:106590002900FEF7E7FB009A019B04000D00300084
:1065A000390006F07BF8002801D1009E019F0022EF
:1065B0000C4B30003900FEF7D5FB02000B00200029
:1065C000290007F0F3F800220023FEF7EEFF012276
:1065D000034BA4331A70B8E730003900D3E7C04644
:1065E000A80800100000F03FF0B589B0FFF76EF882
:1065F000394C0590002804D002238734237009B059
:10660000F0BD26002936FF36FFF784FF3068716839
:106610000022324B07F046FF069007910B00210045
:106620002500270002003931F835A837FF312A63E9
:106630006B63086849683A687B680092019307F0C9
:1066400031FF009A019B286469641000190007F06B
:10665000B7FC0B00224902000868496807F022FFD6
:1066600028656965210023005931B833FF311A6864
:106670005B68086849680292039307F013FF029A67
:10668000039B286669661000190007F099FC0B004F
:10669000144902000868496807F004FF029A039B46
:1066A0002867696700980199250007F089FC79350A
:1066B000FF3502000B002868696807F0F3FE069AB0
:1066C000079B286069603A607B60B268F368A43415
:1066D000BA60FB60059B91E7A80800100000F03F3E
:1066E000F0090010100A0010F7B5FFF713FF134C64
:1066F0002500A835A868E968FEF71CFB2E686F68BE
:106700000090019130003900FEF714FB06000F00E5
:10671000009801990022002307F052FC32003B0050
:1067200006F028FD2300B033286069600099019AC3
:1067300019605A600123A4342370F7BDA808001023
:1067400070B5FEF7C3FF104C012803D10223873434
:10675000237070BD2500A835FFF7DCFE2868696846
:1067600000220A4B07F02CFC094B0A4A07F01EF8DE
:1067700023002860696000200021B0331860596050
:10678000A4340123E4E7C046A80800100080764046
:10679000FB211940182D4454F0B587B0FEF796FF41
:1067A000334C012804D102238734237007B0F0BD95
:1067B0002500A835FFF7AEFE2E686F68300039005F
:1067C000FEF7B8FA0090019102000B00300039008A
:1067D00007F068FE0022274B07F0F2FB0022264B51
:1067E00007F0EEFBFAF7CAF80022234B06F0DEFFB3
:1067F00023000290039100200021B03318605960FB
:106800000298039908F096F908F0CAF91B4A1C4B44
:1068100006000F0007F0D4FBFAF7B0F8320004903E
:106820000591029803993B0007F03CFE0022114BB2
:1068300007F0C6FB134A144B07F0C2FBFAF79EF8A9
:1068400002000B000498059906F094FC00220F4BFF
:1068500006F0ACFF00220E4B06F0A8FF009A019B49
:1068600006F088FCA4342860696001239DE7C046D7
:10687000A80800100000594084D797415555555538
:1068800043DEA341E4388EE35831454180842E41F4
:106890000088C34010B5084C230086331B78002BBA
:1068A00004D185342278002A01D0237010BDFFF76F
:1068B00031FE0123F9E7C046A8080010F0B587B003
:1068C000FFF728FE144D02A82C00A834E3680193BA
:1068D000A368009322686368FDF7B6F8029E039FE1
:1068E00026606760049A059BA260E360FEF7EEFEF7
:1068F00001280BD030003900FEF7D6FA2B002060BB
:10690000616000200021B033186059600123A43574
:106910002B7007B0F0BDC046A8080010F0B58BB0D2
:10692000FFF7F8FDFEF7EEFE204E07003500A83514
:10693000A968E8682A686B680190009106A8FDF7CD
:10694000AFF9089B099C1A4802930394069A079B87
:10695000184907F0A7FD00220490059102980399B9
:10696000002307F02DFB02000B000498059907F0A7
:1069700099FD340028606960B034002F0CD1029A70
:10698000039B0020002107F08DFD20606160012342
:10699000A43633700BB0F0BD002200232260636088
:1069A000FEF782FA28606960F1E7C046A808001087
:1069B000182D4454FB21F93F70B586B0FFF7AAFDAE
:1069C000FEF7A0FE124E05003400A834E36802A8CA
:1069D0000193A368009322686368FDF761F9029848
:1069E000039920606160049A059BA260E360002D1A
:1069F00009D0350000220023B0352A606B60FEF715
:106A000053FA206061600123A436337006B070BD74
:106A1000A808001070B5FFF77DFD0A4C2500A835C9
:106A2000AA68EB6828686968FAF716FE23002860F0
:106A3000696000200021B033186059600123A4343C
:106A4000237070BDA8080010F8B5FEF73FFE144C87
:106A5000002803D0022387342370F8BDFFF75AFDC6
:106A600025002300A835B8331E685F682868696868
:106A700032003B0007F016FD00220A4B07F0A0FA97
:106A80003B00320006F092FE23002860696000207F
:106A90000021B03318605960A4340123DCE7C046FC
:106AA000A80800100000594070B5FEF70FFE114C09
:106AB000002803D002238734237070BDFFF72AFD1E
:106AC00025002100A835B8312A686B680868496834
:106AD00007F076FA084B002206F068FE23002860D3
:106AE000696000200021B03318605960A43401238C
:106AF000E2E7C046A808001000005940F0B58DB08C
:106B0000FFF708FD1D4C2500A835A968E8682A682C
:106B10006B680190009108A8FDF79AF80A9A0B9B00
:106B2000089E099F164906920793086C8A6BCB6BE7
:106B3000496C0090019108A8FDF78AF80A9A0B9B0E
:106B400008A804920593089A099B02920393069A57
:106B5000079B0092019332003B0006F031F8089A3F
:106B6000099B2A606B600A990B9A2300B033196065
:106B70005A600123A43423700DB0F0BDA8080010A2
:106B800000EE000030B587B0FFF7C4FC0C4D02A842
:106B90002C00A834E368A4350193A368009322680D
:106BA0006368FDF755F8029A039B22606360049ABC
:106BB000059BA260E36001232B7007B030BDC04687
:106BC000A808001030B58BB0FFF7A4FC104C2500CE
:106BD000A835AA68EB680492059328686968009252
:106BE00001930290039106A82A686B6805F074FD72
:106BF000069A079B2A606B600899099A2300B033B4
:106C000019605A600123A43423700BB030BDC04614
:106C1000A8080010D0B5FEF759FD134C002803D08A
:106C2000022387342370D0BDFFF774FC2300B833F0
:106C30001E685F682300A8331A685B68300039005B
:106C400007F030FC0022094B06F094FA02000B001A
:106C500030003900FEF786F800230022FEF7A5FC7D
:106C6000A4340123DEE7C046A80800100000F03F6E
:106C7000F0B591B0FFF74EFC644E33002933FF337B
:106C80005C681B68009301940098019933003933C4
:106C9000FF335C681B680293039433005933FF335E
:106CA0005C681B680493059433007933FF331A68DA
:106CB0005B6807F085F9049A059B04000D000298B3
:106CC000039907F07DF902000B002000290007F06E
:106CD000E9FB33004933FF330A900B911A685B6874
:106CE0000098019907F06CF9029A039B04000D00CB
:106CF0001000190007F064F902000B0020002900C1
:106D000007F0D0FB33006933FF33069007911A6810
:106D10005B680098019907F053F9049A059B0400F9
:106D20000D001000190007F04BF9370002000B00AE
:106D30002000290007F0B6FBA8373B687C68089361
:106D40000994BA68FB680C900D9108980999FEF7B0
:106D500073FC2F4B1C6C5D6C9A6CDB6C0E920F936A
:106D60000E9A0F9B20002900FEF746FC0C9A0D9B03
:106D70000698079907F024F9FAF7BAFB34000200E5
:106D80000B000A980B9906F011FDB834330020600F
:106D9000616000220021C03319605A60089A099B83
:106DA0000098019907F00CF9029A039B07F07AFB0F
:106DB0000A9A0B9B07F004F9069A079B04000D0042
:106DC0000498059907F0FCF802000B002000290048
:106DD00006F0D0F9069A079B04000D00009801996F
:106DE00007F0EEF802000B002000290006F0DEFCA0
:106DF00033003860796000220021B03319605A6096
:106E000033000122A4331A7011B0F0BDA80800109D
:106E100080ED0000F0B587B0FFF77CFBFEF756FC75
:106E2000244C012819D02500A8352E686F6800224F
:106E3000214B3000390005F027FC00280DD1390026
:106E4000300007F077FE07F0ABFE02000B003000C9
:106E5000390005F013FC00281DD12500A83528684D
:106E600069680022144B06F085F902000B00E868FF
:106E7000A9680190009102A8FDF72AFD029A039BE0
:106E80002A606B60049A059BAA60EB600123A4341E
:106E9000237007B0F0BD084B002230003900FDF729
:106EA00061FF23002860696000200021B033186072
:106EB0005960EBE7A80800100000F03FF0B587B07C
:106EC000FFF728FB1A4C2500A835AE68EF683000A4
:106ED0002A686B68390002920393FDF72BFF00903C
:106EE000019102980399FDF725FF00220490059176
:106EF00000980199002307F063F8049A059B06F0B7
:106F000039F902000B000298039907F0CBFA009AB6
:106F1000019B2860696025003000390007F0C2FA43
:106F20000123B035A43428606960237007B0F0BD38
:106F3000A8080010F8B5FEF7C9FB194C012803D1C9
:106F4000022387342370F8BD2500A835FFF7E2FA45
:106F5000A868E9680022134B06F028FC02000B0029
:106F600006F008F9104A114B07F02AF80022060033
:106F70000F00286869680B4B06F018FC02000B0034
:106F800006F0F8F8094B084A07F01AF82300B03366
:106F90001E605F6028606960A4340123D2E7C046A8
:106FA000A808001000807640182D4454FB210940A9
:106FB000F0B585B0FEF78AFB3D4C012804D10223D1
:106FC0008734237005B0F0BDA834FFF7A3FA6568D5
:106FD000246820002900FDF7ADFE00900191020019
:106FE0000B002000290007F05DFA0022314B06F06B
:106FF000E7FF0F00060007F09DFD040007F0D0FD3D
:1070000002000B003000390007F04CFA0022294B37
:1070100006F0D6FF0022284B06F0D2FFF9F7AEFCAF
:107020000022254B06F0C2FB0022224B06000F0077
:1070300005F048FB002808D03000390000221D4B25
:1070400007F030FA06000F0001343B2C08DD0098F1
:1070500001990022194B06F08DF8009001913C3CFB
:107060006420604307F09CFD002202900391009889
:107070000199134B06F0A4FF02000B00029803993C
:1070800006F078F832003B0006F074F80C4B002252
:1070900006F08CFB064D0B4B186059602B0000204E
:1070A0000021B033186059600123A4352B7089E7A3
:1070B000A808001000004E4080842E410000F03FE0
:1070C0000088C34050090010F7B5154C23009C33CD
:1070D0001B78DB0603D52B22124BE254F7BD2500AB
:1070E0002600B835A836FFF715FA326873682868A5
:1070F000696806F03FF8B268F36800900191A868EB
:10710000E96806F037F806000F00009801993B0087
:107110003200FEF74AFA0123A4342370DEE7C046AA
:10712000A808001076070000F0B589B0FEF7CEFA87
:10713000394C0590002804D002238734237009B00D
:10714000F0BD26002936FF36FFF7E4F93068716894
:107150000022324B06F00EF8069007910B0021003A
:107160002500270002003931F835A837FF312A639E
:107170006B63086849683A687B680092019305F080
:10718000F9FF009A019B286469641000190006F059
:1071900017FF0B00224902000868496805F0EAFF62
:1071A00028656965210023005931B833FF311A6819
:1071B0005B68086849680292039305F0DBFF029A56
:1071C000039B286669661000190006F0F9FE0B00A3
:1071D000144902000868496805F0CCFF029A039B35
:1071E0002867696700980199250006F0E9FE79355E
:1071F000FF3502000B002868696805F0BBFF069A9E
:10720000079B286069603A607B60B268F368A434C9
:10721000BA60FB60059B91E7A80800100000F03FF2
:10722000F0090010100A0010F7B5154C23009C332C
:107230001B78DB0603D52D22124BE254F7BD250047
:107240002600B835A836FFF765F9326873682868F4
:10725000696807F027F9B268F36800900191A8689F
:10726000E96807F01FF906000F00009801993B003C
:107270003200FEF79AF90123A4342370DEE7C046FA
:10728000A808001076070000D0B5184C8AB023007B
:107290009C331B78DB0604D52A22154BE2540AB036
:1072A000D0BDFFF737F923002100B83318001E685E
:1072B0005F68A8318A68CB68049205930A684B68B6
:1072C000029203938268C36806A800920193320079
:1072D0003B0005F001FA089A099B06980799FEF70A
:1072E00064F90123A4342370D9E7C046A80800102C
:1072F00076070000F0B5A1B0FFF70CF97B4D2B002D
:107300002C0084331B78A8345BB20693012B4CD13C
:1073100022686368A668E7681000190005F02AFF74
:1073200008900991FBF766F932003B000C900D9133
:107330003000390005F01EFF0A900B91FDF71AFA94
:1073400002000B000C980D9905F014FF06000F00C9
:107350000A980B99FDF7C8F932003B0006F026FAAF
:107360000A900B9108980999FBF7DCF932003B0071
:1073700006F01CFA002206000F000A980B99002361
:1073800006F01EFE02000B003000390005F0F2FE90
:107390002B00B033206061600A990B9A19605A6023
:1073A000069BA4352B7021B0F0BD069B276866684C
:1073B000013338D100224E4B18A8049205930022C5
:1073C000002302920393A268E368009201933A00BB
:1073D000330005F081F91A99189A00911B99199BAD
:1073E000019118A8FCF730FB0022424B18A8049228
:1073F0000593802300221B06029203931A9A1B9B7B
:1074000000920193189A199B05F066F9189A199B36
:10741000226063601A991B9A2B00B03319605A607E
:10742000A4350123BEE7FEF751F901286ED02B00E9
:107430007E331B78002B34D02F4A73005B089342B5
:1074400008DC012300220093380000233100FCF700
:1074500079FD08E0294A934213DD3A0033003800F1
:10746000310007F01FF82B00A83318605960B035C1
:10747000002300242B606C6001221C4BA4331A7083
:1074800091E71CAA31003800FCF74EFF1E9A1F9BA3
:107490000221400008400139081A00901C981D99EB
:1074A000D5E72B007F331B78B0350022002B1BD093
:1074B000134B3800310006F079F906000F00FAF797
:1074C00041FB3200069007913B0000200D4906F079
:1074D000E9FFFAF737FB02000B000698079906F060
:1074E00065F920606160C3E7074BE2E7A808001078
:1074F0000000F03F0000F0BFFB21E93FFFFFEF7FFE
:10750000000069400000E03F008066403A00E56806
:10751000A46833003800310005F02CFE0690079176
:10752000FDF728F9220006000F002B00200029009B
:1075300005F020FE08900991FBF75CF802000B00B3
:107540003000390005F016FE06000F00FBF74EF87C
:1075500000229C4B05F098F8002800D1F7E006982F
:107560000799FBF743F80A900B9108980999FBF7E4
:107570003DF8954A0C900D910A980B99934B06F0A3
:1075800015F90022002304000D0005F09BF80022ED
:107590008F4B002800D10BE12000290005F0EAFD07
:1075A00007F0C8FA07F0FCFAA822884BD2050600BB
:1075B0000F0006F005FD02000B000A980B9906F07B
:1075C00071FF802204000D005205824B300039000B
:1075D00006F0F6FC02000B002000290006F062FF16
:1075E0007D4A04000D007D4B3000390006F0E8FCB8
:1075F00002000B002000290006F054FF02000B00DF
:1076000006F0DEFC0C9A0D9B0026002710901191CD
:107610001000190006F0D4FC002234003D00704B2D
:10762000129013910E920F930C920D930A920B935A
:1076300000226B4B2000290005F09CFD0A9A0B9B51
:1076400004000D0006F0BCFC00220A900B91644B74
:107650002000290005F08EFD04000D0002000B0043
:107660000A980B9906F0ACFC0C9A0D9B0A900B91B2
:107670001098119906F0A4FC0E9A0F9B0C900D9196
:107680001298139906F09CFC02000B000E900F91CB
:107690000C980D9905F06EFD0A9A0B9B06F086F882
:1076A00032003B0005F066FD0022169017914C4B0E
:1076B0002000290005F05EFD04000D0002000B0013
:1076C0000A980B9906F07CFC002206000F00444B40
:1076D0002000290005F04EFD02000B0004000D0003
:1076E0003000390006F06CFC0C9A0D9B0A900B914F
:1076F0001098119906F064FC0E9A0F9B0C900D9156
:107700001298139906F05CFC0C9A0D9B0E900F9149
:1077100006F0C8FE0A9A0B9B06F048F802000B0020
:10772000149015911698179905F024FD02000B008E
:1077300006000F001498159906F038F8FAF756FF6E
:10774000284A294B04F0B4FF002800D070E700223B
:1077500000233000390004F091FF00282DD1089853
:107760000999FAF7DFFF32003B0006F01FF804002A
:107770000D0006980799FCF7B7FF32003B0006F0B2
:1077800015F8002206000F0000232000290006F053
:1077900017FC02000B003000390005F0EBFC134B26
:1077A0001A00B033A832106051601C605D6063E65F
:1077B0002000290006F076FEF2E600240C4D0020A1
:1077C0000C49ECE70000D03F182D4454FB21094040
:1077D0000000E03F460B213E6EC0453163626A3CCB
:1077E0000000F03F4F64A14091B49F3CA8080010F6
:1077F0000000F07F0000F87FF0B5842597B0FEF719
:1078000089FE824B814C5D57A834012D42D12668F8
:107810006768A268E3683000390006920793FAF7B8
:1078200081FF0890099106980799FCF75DFF020017
:107830000B000898099906F0C3FB089009913000E5
:107840003900FAF7D7FE06000F0006980799FCF7F3
:1078500091FF02000B003000390006F0B1FB00225E
:1078600006000F0008980999002306F0A9FB020002
:107870000B003000390005F07DFC644B2060616036
:107880000899099AB03319605A60604BA4331D708F
:1078900017B0F0BD22686368069207936B1C5AD13B
:1078A00006980799E36800220893594B05F062FC9B
:1078B000A768089D02000B0001950EA80097FBF732
:1078C00027F80E9A0F9B069807990A920B93109A25
:1078D000119B0C920D9300224D4B06F0E3FD019598
:1078E0000B00020000970EA8FBF712F8109A119BEC
:1078F0000EA8049205930E9A0F9B029203930C9A82
:107900000D9B009201930A9A0B9B04F0E5FE069AE8
:10791000079B0E980F9905F02DFC089B06000D00A3
:10792000109811993A0005F025FC32002B000191C6
:1079300000900EA8FCF78CF90E9A0F9B22606360F2
:107940001099119A314BB03319605A6001222F4BB4
:10795000A4331A709CE7FDF7B9FE2C4DB035012811
:1079600025D02A4B00267E331B780027002B08D019
:1079700006980799FCF7FEFE206061602E606F603C
:10798000E4E7224B00227F331B78002B0DD0214BE4
:107990000698079905F00AFF02000B0000201E4917
:1079A00006F080FDFAF7CEF8E6E71C4BF0E714ABE3
:1079B00012AAA068E168FAF769FF06980799FCF730
:1079C00093FE149A159B06F0FBFA07000E0008912F
:1079D00006980799FCF7CEFE129A139B06F0F0FA70
:1079E00000220690079100233800089906F0E8FA73
:1079F0000B0002000698079906F054FD80231B0631
:107A0000F618206061602F606E609FE7A808001084
:107A10000000F03F000069400000E03F0080664049
:107A2000F0B591B0FEF776FD684D2B002C00843345
:107A30001B78A8345BB20893012B42D12668676893
:107A4000A268E3683000390006920793FAF7D2FD86
:107A50000A900B9106980799FCF746FE02000B006E
:107A60000A980B9906F0ACFA0A900B913000390095
:107A7000FAF758FE06000F0006980799FCF77AFE01
:107A800002000B003000390006F09AFA00220600CE
:107A90000F000A980B99002306F092FA02000B00DF
:107AA0003000390005F066FB2B00B03320606160C8
:107AB0000A990B9A19605A60089BA4352B7011B073
:107AC000F0BD636826680693089B013344D1A26821
:107AD000E36808920993049205933200069B0CA870
:107AE00002920393089A099B009201933200069B2D
:107AF00004F0F2FD0C980D990022354B05F03AFB8D
:107B00000B000E99020000910F990CA80191FAF751
:107B1000FFFE0C980D993200069B05F02BFB089A8E
:107B2000099B06000F000E980F9905F023FB320009
:107B30003B00019100900CA8FCF78AF80C9A0D9B71
:107B4000226063600E990F9A2B00B03319605A605F
:107B50000122A4352A70B2E72F00FDF7B7FDB03738
:107B6000012823D02B007E331B78002B0ED0300051
:107B70000699FCF7B9FD20606160002300243B609A
:107B80007C602B000122A4331A7098E72B007F330E
:107B90001B780022002B07D00E4B3000069905F011
:107BA00005FEF9F7CFFFE6E70B4BF6E7E068A168C3
:107BB0003200069B019000910CA8FCF71DFE0C9A68
:107BC0000D9B226063600E9B0F9CD8E7A8080010F5
:107BD0000000F03F0000694000806640D0B5224CB4
:107BE0008CB023009C331B78DB0604D52F221F4B5F
:107BF000E2540CB0D0BDFEF78DFC2300A833196809
:107C00005A68069107929E68DF68069807990022D5
:107C1000002304F033FD00280BD0002200233000A5
:107C2000390004F02BFD002803D087340123237092
:107C3000DFE72300B8331868596804960597069E55
:107C4000079F029603979A68DB68009201930200EF
:107C50000B0008A804F0B4FF089809990A9A0B9B36
:107C6000FDF7A3FCA434E1E7A808001076070000A4
:107C700070B58AB0FEF74EFC154C2100B83188680B
:107C80000A684B680090C96801912100A8310D680D
:107C90004E68029503968868C9680490059106A805
:107CA000FCF7A2F80699079A2300F83319605A6086
:107CB0000899099A9960DA60089A099B06980799C9
:107CC000FDF773FC0123A43423700AB070BDC046D5
:107CD000A808001070B58AB0FEF71CFC134C1449BC
:107CE00025002600086C8A6BCB6B496CA835009088
:107CF00001912868696802900391F836A868E968DC
:107D00000490059106A8FCF76FF8069A079B08985F
:107D10000999326073602A606B600123A434B060FB
:107D2000F160A860E96023700AB070BDA808001077
:107D300000EE000030B587B0FEF7ECFB0C4D02A85A
:107D40002C00A834E368A4350193A368009322684B
:107D50006368FCF787FD029A039B22606360049AC4
:107D6000059BA260E36001232B7007B030BDC046C5
:107D7000A808001030B587B0FEF7CCFB0C4D02A868
:107D80002C00A834E368A4350193A368009322680B
:107D90006368FAF7BDFD029A039B22606360049A50
:107DA000059BA260E36001232B7007B030BDC04685
:107DB000A8080010842210B552000021014804F0E8
:107DC000E5F810BDB810001010B508210120FDF72E
:107DD00073FA02210020FDF76FFA00210220FDF75F
:107DE0006BFA06210220FDF767FA03210800FDF770
:107DF00063FA032100220800F8F75EFA0022062148
:107E00000220F8F759FA012206210220F8F754FA65
:107E1000FFF7D0FFFDF785FAA220FDF777FAA02043
:107E2000FDF774FAC020FDF771FAF820FDF76EFA3D
:107E30000020FDF76BFA0A20F8F706FA4020FDF75C
:107E400065FA2C20FDF762FA3220F8F7FDF92E20B2
:107E5000FDF75CFA3220F8F7F7F92F20FDF756FA14
:107E60000A20F8F7F1F92520FDF750FA0A20F8F773
:107E7000EBF98120FDF74AFA0020FDF747FAAF2021
:107E8000FDF744FAA420FDF741FA10BD70B50A20B1
:107E9000F8F7DAF9FDF75CFC0128F8D01D4D2C004D
:107EA00048342379002B19D0002323712372E37007
:107EB0006379002B07D1C122022152000E20F8F76E
:107EC00099FA012363710C22012148352B790800AE
:107ED0001A43AB795B001A43F8F78CFAAC20FDF734
:107EE00015FAAE20FDF712FAA520FDF70FFA0020D3
:107EF0000121F8F717FB0020F8F798FC002802D1C1
:107F00000121F8F70FFBFFF75FFFFFF753FFFDF7C6
:107F100008FA70BD18000010CC2270B5D200002104
:107F20000C4804F033F8EB230B4CDB00E51810335E
:107F3000E05806F06FFE094A094B05F037FCEC23C8
:107F4000DB00E4180022002328606960226063607F
:107F500070BDC046B0090010A80800100000C0FFA6
:107F6000FFFFDF411B4B1C491A002932FF3270B55D
:107F70000C6C4D6C886CC96C146055609060D1605D
:107F80001A003932FF32146055609060D1601A00D7
:107F90004932FF32146055609060D1601A00593246
:107FA000FF32146055609060D1601A0079336932F5
:107FB000FF33FF329860D960146055609060D160E3
:107FC0001C605D60FDF7BCFF40220021034803F008
:107FD000DDFF70BDA808001080ED00005009001002
:107FE00070B50F4C0F2223000E4E78331A703000FC
:107FF0000532002103F0CAFF230000259C330A4A02
:108000001D700A4B0C320A493000E55403F0B3FFEF
:1080100023008334A0331D602570FDF791FF70BDF0
:10802000A8080010300900100000001076070000BA
:10803000D8F60000F7B56F4C260083363378002B56
:1080400016D0230085331B78002B10D06A4D703575
:10805000280003F0D3FF012804D12800FDF7AEFD6E
:1080600001303070833421787620FCF7F3FFF7BDC0
:10807000230086331B78002B00D1A2E0FDF784FF9C
:1080800023007C331A885D4B9B185D78FDF71EFB3F
:1080900001280BD10C2D05D8594BEB409843C0B2A9
:1080A000002809D0022387342370E0E7022803D197
:1080B0002B00083B032BF5D92300A8331E685F680B
:1080C0002300681EB8331A685B68009201930B287E
:1080D00019D804F0B9FA061B262D343B4E5D6063B7
:1080E00066692100A83100228868C968002304F06D
:1080F000C5FA002812D0002200233000390004F015
:10810000BDFA00280AD0FCF781FF07E00022002317
:108110003000390004F0CCFA0028F4D0A434012354
:10812000C2E7002200233000390004F0ADFAF3E783
:10813000002200233000390004F0C4FAECE70022EA
:1081400000233000390004F0A9FAE5E721002300FC
:10815000A831B8339A68DB688868C96804F08EFA79
:108160000028D0D0009A019B3000390004F086FA34
:10817000D2E721002300A831B8339A68DB68886809
:10818000C96804F07BFA0028C8D0009A019BB4E7C4
:10819000009A019BBCE7009A019BC4E7009A019BEF
:1081A000C8E7009A019BCCE72100A831002288682B
:1081B000C968002304F062FA0028A4D0002200233A
:1081C000D2E7230085331B78002B00D14FE7FFF760
:1081D00007FF220020219C3211702200012309494F
:1081E000A03211607834084908483370237003F0D6
:1081F000C2FE3CE7A808001018000010D4000010D0
:10820000C210000035800000B0F6000030090010F8
:10821000F7B5384C23009C331D78002D56D03648D6
:10822000364D030070331B78002B0FD12300A03391
:108230001B68AB4202D0324A93421DD1314BE35C02
:10824000002B19D17030304903F095FE2300A03384
:108250001A68AA4222D12B4AA25C2B2A12D12B4A9D
:108260001A602300A0331B68873498472378002BBB
:1082700029D0FDF765FE04E0230083331B78002B33
:10828000E4D1F7BD2D2A01D1214AE9E72A2A01D1FB
:10829000204AE5E72F2AE4D11F4AE1E718498A423C
:1082A000DFD1184AA25C2B2A01D11C4AD8E72D2A1B
:1082B00001D11B4AD4E72A2A01D11A4AD0E72F2A32
:1082C000CFD1194ACCE7FFF78BFEDAE7FDF75CFE6A
:1082D0002300A8331E685F689A68DB6800920193E8
:1082E000009A019B30003900A434FDF785F9257010
:1082F000C7E7C046A808001018000010A1960000AB
:108300005197000076070000B6F60000A59800001F
:10831000F99800004D990000B1990000159A0000ED
:108320005D9A0000A59A0000F99A0000F0B56D4C26
:1083300091B023009C331B785B070BD56A4B7033DD
:108340001B7E002B02D14920FDF798FBFFF760FF51
:1083500011B0F0BDFDF718FEFDF7B8F9012835D1D1
:108360002500A835AA68EB6806920793230080339E
:108370001B78B03400260027002B22D02A686B68B7
:108380000892099308980999069A079BF9F764F9E6
:10839000089A099B0A900B9106980799FBF7A2FA95
:1083A0000A9A0B9B266067602A606B60FCF77CFD75
:1083B00032003B00FDF720F901224A4BA4331A702A
:1083C000C6E72660676006980799F1E7022802D1A0
:1083D00087342070BCE72200B83210685168956875
:1083E000D6682200230008900991069507968032EE
:1083F0001278A8331868596800260027002A4CD044
:1084000023007E331B78002B0FD17F34237800228A
:10841000002B40D0354B05F0C9F902000B0004F0E9
:10842000A9FE334A334B05F0CBFD2E4B324C1A00DC
:10843000B0331E605F600023A83210605160049367
:10844000059402000B000CA8029603970096019772
:1084500004F042F90E990C9A00910F990D9B01912D
:108460000CA8FCF7FFF90E9B0F9C0CA80493059435
:108470000C9B0D9C02930394069B079C0093019414
:10848000089A099B04F028F90C980D990E9A0F9BF5
:10849000FDF78BF890E7194BBDE70024164D0296C7
:1084A0000397049405950200DC689B680CA8009370
:1084B00001940B0004F010F9089A099B0C980D998F
:1084C00004F058FE069A079B04000D000E980F99C1
:1084D00004F050FE06000F002000290032003B008F
:1084E000D6E7C046A8080010180000100000794028
:1084F000182D4454FB2109400000F03F00807640D5
:108500001FB5124C23009C331B789B070AD51048DB
:108510007030037E002B02D10E4903F02CFDFFF7D3
:1085200077FE1FBDFDF7F6FF23008021A8339A6870
:1085300009060292DA68A434521803920299039A47
:108540009960DA6001232370EBE7C046A8080010A9
:1085500018000010BAF60000F0B5384B89B004934B
:108560000023374E0D00745C02A903900B739A42EE
:1085700004D01522334904A803F0FDFC2000FCF7C9
:10858000C3FC07002800FCF78DFD002F1ED000283B
:108590001ED12F007619767806AD0522002128001D
:1085A00003F0F4FCFE2E17D12749280003F0E3FC6A
:1085B000762C2DD13A00254BB6009E19B36C244978
:1085C000009304AB039803F0D6FC2CE000282CD0D9
:1085D0006F1EF45D765DDFE7FF2E01D11D49E4E7F4
:1085E0001D49FD2EE1D0632E0FD923004F3B012BF7
:1085F00004D92B2C02D0A31F012B06D8320011491D
:10860000233A280003F0B7FCD2E732001349F8E719
:10861000134BA400E358019500933A0004AB1149B1
:10862000039803F0A8FC09B0F0BD0D4BA400E3587B
:108630002A0000930C4904ABC4E7C0462020000088
:10864000D4000010A1F7000065F7000000EE000064
:10865000C7F60000BAF60000BEF60000C4F600003F
:1086600020F10000D0F60000DBF6000010B509286C
:108670000BD9094BFE2809D1E922D2009B181868B2
:10868000596806F057FA03F095FE10BD03228733B0
:108690001A700020F9E7C046A808001010B50300C2
:1086A0000E280CD90F20FE2B09D1E922044BD20051
:1086B0009B181868596806F03DFA03F07BFE10BD60
:1086C000A808001010B5682802D8FCF72DFD10BDD1
:1086D000094BFE280AD1E922D2009B181868596874
:1086E00006F028FA03F066FEC0B2EEE703228733F5
:1086F0001A700020EBE7C046A808001010B5030070
:1087000063280CD96420FE2B09D00130FD2B06D044
:10871000094CFF2B04D0032300208734237010BDA5
:10872000E923DB00E3181868596806F003FA03F040
:1087300041FE6328EFDCF2E7A8080010F0B50D0059
:1087400085B0040017000268436810001900009209
:108750000193FCF741FB534A28601300A5331B78B3
:108760000600012B30D1A6321378BB4200DB7B1E02
:108770000F2F00DD0F27BE4203DA5B429E4200DB73
:1087800082E03000FCF757FA02000B0000980199D4
:1087900005F00CF801262060616020686168FCF734
:1087A0001BFBB0424FDB3F4B2F68A5331B78032BDD
:1087B00000D06CE0032E00D069E000223A4B033772
:1087C000226063602F603EE0022BDAD0032B4DD194
:1087D000009801990022354B03F074FF002807D15F
:1087E000009801990022304B03F058FF00284BD02D
:1087F0003000FCF720FA02000B000098019904F009
:10880000D5FF20606160300003F0D4FD032103F048
:1088100017FF0E1E17D02B68009322686368029220
:108820000393009B002B10DD0800FCF704FA029A6A
:10883000039B05F0C5FB009B206061609F1B013618
:108840002F60002EA9D105B0F0BD03277F1A380094
:10885000FCF7F1F9029A039B05F0B2FB206061601E
:108860000420009B861BDF1B2F6096E7042BEAD1B8
:108870000E20801BFCF7DFF902000B000098019925
:1088800005F09EFB2060616000232B60DBE7701E1B
:10889000FCF7D1F904F03AFC04F056FC01372060F3
:1088A00061608FE7A80800100000F03F00408F4093
:1088B000F0B58BB0FDF72EFE3B4C08A82300260038
:1088C000A83319685A68089109929A68DB68069279
:1088D00007930223A53635780F2205A93370FFF7D9
:1088E0002DFF0F2206A804A9FFF728FFA634357034
:1088F0002078FCF7A0F904F009FC032D03D10A222B
:10890000002303F04BFC04F01FFC089A099B0400B1
:108910000D0005F055FBF8F731F822002B0004F0AC
:1089200045FF069A079B06000F002000290005F06E
:1089300047FBF8F723F822002B0004F037FF040070
:1089400005980D00FCF777F902000B0030003900A4
:1089500005F036FB029003910498FCF76CF9124E77
:1089600000900191002200232000290005F028FB3F
:10897000009A019B05F024FB029A039B370004F048
:10898000F9FB009A019BA837386079603700200016
:10899000290005F015FB0123B037A4363860796053
:1089A00033700BB0F0BDC046A8080010F0B597B00A
:1089B0000190190010000892099315001C00F8F7A7
:1089C00089FDC349049000280ED16300C14A5B08A9
:1089D000D3420ED4210000220023280003F068FEB9
:1089E000BD49002800D1BD49019803F0C4FA17B071
:1089F000F0BD002200232800210003F045FE0028DE
:108A00000FD0B74BA5331B780895043B1A00531EB3
:108A10009A4180231B06E4181C9B0492013B099495
:108A20001C931C9A0BA908A8FFF788FE089B099CB9
:108A3000180021000693079404F068FB03000C0063
:108A4000029003910E930F9404F07EFB0D0004003E
:108A5000FCF7C2F9220005902B00461C06980799E6
:108A600005F020FD029B039A0690079113430F2700
:108A7000002B00D11027BF1B3800FCF7DCF80200E8
:108A80000B0004000D000698079905F099FAF7F716
:108A900075FF04F03BFB0C900D9104F055FB220098
:108AA0002B0003F00FFE002820D00022002301201D
:108AB00000210C920D93029A039B12184B41100057
:108AC00019000B9C0E900F9104F03EFBFCF784F90B
:108AD000B0420BDB002C00D1B4E00598FCF7ABF8FA
:108AE00004F014FB0E900F9101340B940B9C002C9E
:108AF00007D0200006F054F8FCF76EF9E40F2418B4
:108B00000234774B1A00A533A63215781B782A0059
:108B1000032B02D1AA1BAE4200DC0F25002F00D18F
:108B200093E03B00974200DD13001C9A141BA11B2D
:108B30001A008B4200DD0A00D143C9170A40029295
:108B4000BA4200DB86E0BA1A39000CA8FCF7F0FC48
:108B500000281DD000220023012000210C920D933B
:108B60000E9A0F9B801859410E900F9104F0ECFA69
:108B7000FCF732F9B0420BDB0B9F002F68D0701E60
:108B8000FCF759F804F0C2FA0E900F9101370B97D9
:108B9000002C00DC0124A6425EDD341B22003100E3
:108BA0000EA8FCF7C5FC002809D00E980F990B23DE
:108BB00064220B93002303F0F1FA0E900F910B9BAC
:108BC0001C190B941422002111A803F0DFF9029A5A
:108BD000444911A803F0CFF9049B012B08D1019857
:108BE00003F00CFA019B2D2218183F4903F0C3F93A
:108BF000019803F003FA019B3C4918180E9A0F9B49
:108C000003F0B9F9029B002B4EDD019803F0F6F951
:108C1000019B11A918180C9A0D9B03F0ACF90B9B42
:108C2000002B00D1E3E62E4B0198A5331B78042BD3
:108C300047D103F0E3F92E22019B2B49181803F0CA
:108C40009AF9D4E6059E023650E701235B426CE7B1
:108C500001369DE702939BE7AE42B3DD771B3800F8
:108C6000FBF7E9FF3A0004000D000EA83100022EC8
:108C70000EDCFCF75DFC0E980F9904F065FA2200FB
:108C80002B0005F09DF904F041FA0E900F9199E741
:108C9000FCF74EFC0028EED0002301220E920F9329
:108CA0000B9B03330B938DE7029B002BB7D10198ED
:108CB00003F0A4F9019B2E2218180B4903F05BF96D
:108CC000ADE703F09BF9019B0B9A18180849B6E72A
:108CD000E3F6000000001080E8F60000E7F6000070
:108CE000A8080010ECF60000A1F70000F6F600005E
:108CF000FBF6000082B0F0B593B019931C9B18925C
:108D0000023BDA0FD3185B100390162200210CA847
:108D1000029303F03BF91622002106A803F036F96E
:108D20001A9C1B9D404E330080331B78002B5DD076
:108D30001898199922002B00F8F78EFC189A199BA5
:108D40000490059120002900FAF7CCFD33007E360F
:108D50007F331A78337804000D00134338D1002292
:108D6000324B05F02DF9324A324B04F01FFD1E261E
:108D700004000D00029B0CA80093049A059BFFF7CA
:108D800015FE0CA803F03AF9029B984206D20CA8F3
:108D900003F034F9029B5B001B1A0293029B06AF9F
:108DA000009322002B003800FFF700FE1E4B1A0034
:108DB000A5321278042A1FD133001F4900970CAA4C
:108DC000039803F0D8F813B0F0BC08BC02B0184701
:108DD0001E26002ACED00022184B05F0F1F8144AC6
:108DE000144B04F0E3FC04000D00C3E7189A199B30
:108DF000692604920593BDE780331B78002B04D0CD
:108E0000009733000CAA0E49DAE70022002329005C
:108E1000200003F04DFC00963B000CAA09490028F5
:108E2000CED10949CCE7C046A808001000807640A2
:108E3000182D4454FB21194000F700000000794030
:108E400007F7000010F700001AF7000070B5214C7A
:108E500023009C331B785B060AD51F487030037EC5
:108E6000002B02D11D4903F086F8FFF7D1F970BD40
:108E70002500A835FDF788F8AA68EB6828686968B6
:108E8000FCF7DAFBEB23DB00E618154A154B3068DC
:108E9000716805F095F804F01BF9ED23DB00E05054
:108EA000114803F08BFA05F07BFE0D4A0D4B04F0E0
:108EB0007DFCEC23DB00306071600022E6180023AB
:108EC00032607360AA60EB600123A434286069609B
:108ED0002370CCE7A808001018000010B6F60000B8
:108EE0000000C0FFFFFFDF411010001010B5284C3C
:108EF00028497034200003F093F8002802D1FDF7D0
:108F00001FF810BD200003F079F800280FD02000D2
:108F100003F074F80023201801380370200003F0D8
:108F20006DF80028EDD11C4BA4331870E9E71A4BFB
:108F30001A009C321278002A02D0FFF751F8E0E7BD
:108F40001A0085321278002A1AD07C331C88002C33
:108F5000D7D0124B185DFBF7D7FF002802D0A01C1A
:108F6000022107E02000FCF79DF801210300601CAE
:108F7000002BF5D14942FCF713F8FCF7BFF8C0E726
:108F8000200003F03BF80028BBD1FCF7E5FFB8E771
:108F900018000010BAF60000A8080010D400001055
:108FA00010B50F4CFE2070342378492B13D00D4997
:108FB000200003F035F80300FF20002B0BD00A49F6
:108FC000200003F02DF80300FD20002B03D02078B3
:108FD000402801D9233010BD2000FCF7EFFDFAE74F
:108FE00018000010BAF60000B6F6000070B5FCF7E5
:108FF000CBFF1E4C25009C352B78002B0AD08534E6
:10900000FFF7CEFF2378002B03D0C1B27320FCF70B
:1090100021F870BD230086331B78002B15D0230068
:109020007C331A88124B9B185878FFF71FFB2300DC
:1090300087331B78002BECD10E4B2418E4182378CF
:10904000002BE6D1FBF7E2FFE3E7FEF7C9FF0523BC
:109050002B702300084AA0331A6001237834074993
:109060000748237002F087FFD3E7C046A808001026
:10907000D40000106C070000ED8F000023F7000003
:109080003009001070B5FCF77FFF224C25009C359D
:109090002B78002B16D0FFF783FF230085331D7834
:1090A000C0B2002D04D001006F20FBF7D3FF70BDCC
:1090B000FFF7DCFA184B2018C01805700123A43400
:1090C0002370F4E7230086331B78002B11D0230094
:1090D0007C331A88114B9B185878FFF7C7FA230086
:1090E00087331B78002BE2D10B4A201880180370BD
:1090F000E4E7FEF775FF05232B702300084AA03331
:109100001A600123783407490748237002F033FFBF
:10911000CDE7C046A80800106C070000D40000107E
:10912000859000002FF700003009001070B5FCF7A3
:109130002BFF204C25009C352B78002B16D0FFF7F9
:109140002FFF230085331B78C0B2002B04D0010011
:109150006B20FBF77FFF70BDFFF788FA164B2018D6
:10916000C0180123A43403702370F4E7230086336E
:109170001B78002B0DD023007C331A880F4B9B18D3
:109180005878FFF773FA230087331B78002BE2D15E
:10919000E4E7FEF725FF05232B702300084AA033E0
:1091A0001A600123783407490748237002F0E3FE70
:1091B000D1E7C046A80800106C070000D4000010DA
:1091C0002D9100003BF7000030090010F8B5FCF7C6
:1091D000DBFE1D4C25009C352B78002B23D0FFF7A0
:1091E000DFFEC0B2FBF7A0FF184B984217DC02224B
:1091F000012103009446164F091AFA22CD18D20015
:10920000934206D0FA5C562A03D066460133B24335
:10921000F3D102214942491B4019FBF7C1FE00234B
:109220007C342380F8BDFEF7DBFE08232B7023007F
:10923000084AA0331A60022378340749074823708C
:1092400002F099FEEEE7C046A8080010CF07000024
:10925000D4000010CD91000045F700003009001047
:10926000F0B5334C89B025009C352B78002B0BD002
:109270008534FFF795FE2378002B03D0C1B24B2035
:10928000FBF7E8FE09B0F0BD230086331B78002B06
:109290003CD0FCF779FE23007C331A88254B9B18C1
:1092A0005878FFF72BFA05002D0165192F00224E83
:1092B00009373100FBF726FD3068716807AB009372
:1092C00005AA06ABFBF7E8FC059A079BFF379E183B
:1092D0000798BA68FB6805960292039305F060FC54
:1092E00002000B003868796803F044FF029A039B80
:1092F000F835AA61EB61069B286169619E4201DD38
:10930000FBF784FE0123A4342370BBE7FCF73CFE8B
:10931000FEF766FE07232B702300084AA0331A606D
:109320000223783406490748237002F024FEA9E797
:10933000A8080010D4000010A009001061920000DD
:1093400052F7000030090010F0B5334C89B0250009
:109350009C352B78002B0BD08534FFF721FE23782A
:10936000002B03D0C1B24720FBF774FE09B0F0BD5B
:10937000230086331B78002B3CD0FCF705FE23002E
:109380007C331A88254B9B185878FFF7B7F90500EE
:109390002D0165192F00224E09373100FBF7B2FC71
:1093A0003068716807AB009305AA06ABFBF774FC45
:1093B000059B079AFF379E1A0798BA68FB680596BF
:1093C0000292039305F0ECFB02000B003868796809
:1093D00005F068F8029A039BF835AA61EB61069BD9
:1093E000286169619E4201DCFBF710FE0123A43471
:1093F0002370BBE7FCF7C8FDFEF7F2FD07232B70D7
:109400002300084AA0331A6002237834064907482B
:10941000237002F0B0FDA9E7A8080010D4000010E6
:10942000A00900104993000056F700003009001011
:1094300070B52D4C25009C352B78002B19D0FFF7EB
:10944000AFFD230085331B78C0B2002B1ED0010076
:109450004320FBF7FFFD70BD2D0165190935FF3570
:10946000326873682A606B60B268F368AA60EB6068
:1094700023E0230086331B78002B22D0FCF784FDE9
:1094800023007C331A88194B9B185878FFF736F95C
:1094900026002100F836A8310A684B6805003260C2
:1094A00073608A68CB68B260F360FBF72BFC652DB4
:1094B000D2DD2300032287331A700123A4342370E2
:1094C000C9E7FCF761FDFEF78BFD07232B70230036
:1094D000074AA0331A6002237834064906482370ED
:1094E00002F049FDB7E7C046A8080010D4000010FC
:1094F000319400005AF700003009001070B51F4C7D
:1095000025009C352B78002B12D0FFF749FD230056
:1095100085331B78C0B2002B15D001004C20FBF71F
:1095200099FD70BD01221A700323A5342370F8E75A
:10953000230086331B78002B0DD023007C331A8840
:109540000F4B9B185878FFF7A9F82300A633002883
:10955000E8DD1870E8E7FCF717FDFEF741FD230092
:1095600002227833074908481A7002F004FD074BBD
:10957000A034236005232B70D3E7C046A808001051
:10958000D40000105FF7000030090010FD940000C7
:1095900070B51C4C25009C352B78002B0CD0FFF7A8
:1095A000FFFC230085331B78C0B2002B0FD00100D5
:1095B0004820FBF74FFD70BD230086331B78002B3E
:1095C0000ED023007C331A880F4B9B185878FFF776
:1095D00065F82300A63318700223A5342370EAE748
:1095E000FCF7D2FCFEF7FCFC23000222783307498B
:1095F00007481A7002F0BFFC064BA0342360052315
:109600002B70D8E7A8080010D400001063F7000002
:10961000300900109195000070B51C4C25009C3558
:109620002B78002B0CD0FFF7BBFC230085331B7875
:10963000C0B2002B0FD001004420FBF70BFD70BD22
:10964000230086331B78002B0ED023007C331A882E
:109650000F4B9B185878FFF721F82300A63318709A
:109660000123A5342370EAE7FCF78EFCFEF7B8FC73
:10967000230002227833074907481A7002F07BFC66
:10968000064BA034236005232B70D8E7A8080010F0
:10969000D400001067F70000300900101996000090
:1096A00070B5264C25009C352B78002B1BD0FFF77E
:1096B00077FC230085331B78C0B2002B20D001003B
:1096C0000D20FBF7C7FC70BD2300000120180930F6
:1096D000FF30A83319685A68016042609A68DB68F5
:1096E0008260C36014E0230086331B78002B13D004
:1096F000FCF74AFC23007C331A88114B9B185878DE
:10970000FEF7FCFF6528DFDD2300032287331A7094
:109710000123A4342370D6E7FCF736FCFEF760FC87
:1097200056232B702300074AA0331A600223783493
:1097300005490648237002F01EFCC4E7A808001083
:10974000D4000010A19600006BF700003009001053
:1097500030B5314C85B025009C352B78002B26D0B8
:10976000FFF71EFC230085331B78C5B2002B05D004
:1097700029001120FBF76EFC05B030BD274B196C9A
:109780005A6C009101929A6CDB6C009801990292DC
:109790000393029A039BFBF74FFF2800FEF7AEFFEF
:1097A0001F49FBF7AFFA0123A4342370E4E7230039
:1097B00086331B78002B1CD0FCF7E6FB23007C33A0
:1097C0001A88184B9B185878FEF798FF0500134B22
:1097D000196C5A6C009101929A6CDB6C009801999B
:1097E00002920393029A039BFBF726FF0C49280081
:1097F000D7E7FCF7C9FBFEF7F3FB56232B702300DA
:10980000094AA0331A6002237834084908482370B3
:1098100002F0B1FBB0E7C046A808001080ED0000E0
:1098200050090010D4000010519700006FF700009D
:109830003009001070B5174C01222300A4331A70B0
:10984000230086331B780500002B0ED07C34FCF7F8
:109850009BFB2288104B9B185878FEF74FFF0400A3
:109860000E492000FBF74EFA10E023009C331B78D2
:10987000002B0DD0FFF794FB85342378C0B2002B6A
:10988000EBD001002800FBF7E5FB054C200070BD84
:10989000034CE5E7A8080010D4000010A009001050
:1098A000FFFFFF7FF7B57920FFF7C4FF05006428AD
:1098B0001FDC104C2D0127002600A837F83632682F
:1098C00073683868796803F055FCBA68FB680090E3
:1098D0000191B068F16803F04DFC009A019B641996
:1098E000F83432607360B060F16022616361A0613E
:1098F000E161F7BDA8080010F7B57A20FFF79AFFDD
:10990000050064281FDC104C2D0126002700F836C6
:10991000A8373A687B683068716804F0C3FDBA689C
:10992000FB6800900191B068F16804F0BBFD009AFB
:10993000019B6419F83432607360B060F160226199
:109940006361A061E161F7BDA808001070B57B20DC
:109950008AB0FFF76FFF0500642824DC134C2D014B
:1099600023002600A8339968DA68049105921A68E2
:109970005B6802920393F836B268F3680092019331
:1099800064193268736806A8F83402F0A5FE0698D8
:109990000799089A099B30607160B260F36020619A
:1099A0006161A261E3610AB070BDC046A808001001
:1099B00070B57C208AB0FFF73DFF0500642824DCE9
:1099C000134C2D0123002600A8339968DA6804910E
:1099D00005921A685B6802920393F836B268F368DE
:1099E0000092019364193268736806A8F83403F092
:1099F000E7F806980799089A099B30607160B26091
:109A0000F36020616161A261E3610AB070BDC0468C
:109A1000A808001073B57D20FFF70CFF642819DC3F
:109A20000D4C25002600A835F836B268F368A86802
:109A3000E96803F09FFB3268736800900191286821
:109A4000696803F097FB009A019BB0342860696055
:109A50002260636073BDC046A808001073B57E2005
:109A6000FFF7E8FE642819DC0D4C25002600A83518
:109A7000F836B268F368A868E96804F013FD326844
:109A80007368009001912868696804F00BFD009AE2
:109A9000019BB034286069602260636073BDC0467A
:109AA000A808001030B57F208BB0FFF7C3FE6428F4
:109AB0001EDC104C06A823002500F8339968DA68EC
:109AC000049105921A685B6802920393A835AA680C
:109AD000EB68009201932A686B6802F0FDFD069A1C
:109AE000079BB0342A606B60089A099B2260636010
:109AF0000BB030BDA808001030B580208BB0FFF748
:109B000099FE64281EDC104C06A823002500F833BB
:109B10009968DA68049105921A685B680292039367
:109B2000A835AA68EB68009201932A686B6803F075
:109B300047F8069A079BB0342A606B60089A099B25
:109B4000226063600BB030BDA808001070B5114CE6
:109B5000114E2500A0352B68B3420DD1FFF720FA36
:109B6000C0B2FBF7F7FA002803D10423873423702F
:109B700001E07C34208070BDFEF732FA230002221F
:109B80007833064906481A709C3402F0F4F92E60C6
:109B90000923ECE7A80800104D9B000073F70000B4
:109BA0003009001070B5FCF7EFF9244C25009C3506
:109BB0002B78002B0AD085342378002B05D0FFF7B3
:109BC000EFF9C1B20720FBF745FA70BD23008633D9
:109BD0001B78002B19D0230001222500A4331A7012
:109BE0007C352A88164B9B185878FBF7B3FA002867
:109BF00007D12300042287331A700123A434237071
:109C0000E3E72880FBF77AFAF7E7230085331B7830
:109C1000002B0FD0FEF7E4F90C232B702300094A28
:109C2000A0331A600223783407490848237002F0F1
:109C3000A2F9CAE7FFF78AFFC7E7C046A8080010E5
:109C4000D4000010A59B00007EF700003009001032
:109C500070B5184C184E2500A0352B68B34213D1AF
:109C6000FFF79EF9061E00D10136FBF779F90500D2
:109C7000B04200DD35002800FBF714FA431E98417E
:109C80007C342D18258070BDFEF7AAF9FBF768F922
:109C900004F086FFFBF7A0F823000130783318703A
:109CA0000649074802F067F901239C342E602370AF
:109CB000E9E7C046A8080010519C000087F70000A3
:109CC00030090010F7B5304C220083321378002B96
:109CD00008D00C2B04D10B3B1370FBF77FFEF7BDB4
:109CE0000133F9E7294D70352B7E002B17D06E7E9E
:109CF000A97E744274410C40E97E701C2818AB198F
:109D0000AA7D0C4304D00100180002F062F9E4E7D8
:109D1000190002F05EF92D236C75AB55DDE72300C9
:109D20000122A4331A702300A8331A685E680192D6
:109D30009F68DD68002200230198310002F09EFC3C
:109D4000002802D180231B06F618002200233800C9
:109D5000290002F093FC002802D180231B06ED1895
:109D6000002200233800290004F02AF9019A330068
:109D700003F000FA064B3A00186059602B00B0342B
:109D800022606360A9E7C046A80800101800001010
:109D900050090010F0B5504D89B0280002F02EF99E
:109DA0004E4E009028220021300002F0EFF84C4F78
:109DB0004C4CE35D002B0FD0280002F01FF9201857
:109DC000873003782B2B39D1280002F017F9444B48
:109DD0002018E35C87300370230083331B78424FE5
:109DE000002B4AD0414A9B00D3189A6C390002A834
:109DF00002F0C1F823009C331B78DB0603D53C49F5
:109E0000300002F00FFB02A9300002F00BFB230030
:109E10009C331B78002B55D02200A032354B1268A2
:109E200000259A4208D0344F7037230078331B78CE
:109E3000BA7D9B1AAB423FDC09B0F0BD280002F0AE
:109E4000DDF82018873003782D2BBDD0280002F0D4
:109E5000D5F82018873003782A2BB5D0280002F0D7
:109E6000CDF82018873003782F2BADD0280002F0D2
:109E7000C5F820188830E35DADE71222009BD31AA5
:109E80001D4A019370320092937D019A93420CDD3A
:109E90001A4A1B490F32300002F06DF8009B9A7D80
:109EA000019BD21A009B9A18A0E72A0039003000C3
:109EB00002F061F8009A99E71249300002F0B2FA14
:109EC0000135B2E70C4B70339B7D0E2BB4D80D4996
:109ED000300002F0A7FAAFE730090010D0080010F8
:109EE00076070000A8080010D8F6000000EE000079
:109EF00045F8000035800000180000100000001038
:109F000093F7000097F70000F0B5CD4E89B02822F6
:109F10000021300002F03AF8CA4D28220021280022
:109F200002F034F8C84C14220021200002F02EF870
:109F300014220021C54802F029F8330085331B782C
:109F4000002B05D1330079331B78002B00D1E6E0DC
:109F500033007C331988002904D0013900223000F5
:109F6000FEF7FAFA37007C37012239882800FEF71D
:109F7000F3FA3888FBF7A8F80200692807DCB4492F
:109F8000632801DDB349233A200001F0F4FF9C3639
:109F90003378002B01D0FFF7FDFEA94C2300873357
:109FA0001B78002B44D0012B03D1AB49200001F0DA
:109FB000E2FF230087331B78022B03D1A74920003F
:109FC00001F0D9FF230087331B78042B03D1A44968
:109FD000200001F0D0FF230087331B78052B03D12D
:109FE000A049200001F0C7FF230087331B78032B13
:109FF00003D19D49200001F0BEFF230087331B7869
:10A00000062B03D19949200001F0B5FF23008733C7
:10A010001B78072B03D19649200001F0ACFF2300E9
:10A0200087331B78092B03D19249200001F0A3FF4D
:10A0300023007A331B78002B03D08F49200001F0D6
:10A040009AFF230086331B78002B14D12300A533FD
:10A050001B78042B0FD0230084331B7887495BB215
:10A06000012B00D1E7E0013300D0D7E01D22844965
:10A07000764801F080FF230085331B78724D002B5A
:10A0800028D12300A5331B78042B23D023007E3353
:10A090001B78002B03D07B49280002F0C3F9230072
:10A0A0007F331B78002B03D07749280002F0BAF9E0
:10A0B000EF23DB00E35C002B03D07449634802F01C
:10A0C000B1F9230080331B78002B03D0704928009E
:10A0D00002F0A8F9FDF76EFE20000021FBF720FE3C
:10A0E00008215848FBF71CFE002383211A00280092
:10A0F0008334FBF743FC2378002B00D1E0E00123FD
:10A10000082268216348FBF739FC01230822522109
:10A110006148FBF733FCFBF704F909B0F0BD3300ED
:10A1200086331B78002B0FD033007C331B885B4AAF
:10A13000D35C2A2B08D05A49300001F01CFF594942
:10A14000280001F018FF28E73300A53356481B7894
:10A150000C30042B50D101F051FF16245349241A1E
:10A16000300001F008FF374F5149380001F003FF7C
:10A17000300001F043FF3300B8331A6835180592F8
:10A180009E685A68DB68069207930022002330001D
:10A19000079902F073FA002832D10799059A069BB5
:10A1A0000294019100962800FEF7A4FD380001F00A
:10A1B00025FF234B3F18A8331A689D68DE68059277
:10A1C0005A682800069200230022310002F056FA55
:10A1D00000281CD1059A069B029401960095380030
:10A1E000FEF788FD334B70331B7E002B00D0D2E688
:10A1F000134B9C331B78CCE601F000FF1224ADE733
:10A200000094059A069B2800FEF7D0FBCEE7009449
:10A21000059A069B3800FEF7C9FBE3E7230082336B
:10A220001B782549002B06D1230081331B78002B96
:10A2300000D120E72149054802F0F4F81BE7C046A9
:10A24000A8080010D0080010F80800100C09001031
:10A25000A4F7000099F70000C3F70000CFF7000053
:10A26000DCF70000E5F70000F2F70000FDF7000062
:10A270000FF800001CF8000024F800002AF8000085
:10A280002CF8000032F8000036F8000039F8000021
:10A290003CF800003FF8000043F80000D400001034
:10A2A000AFF70000B7F7000000000010BDF7000096
:10A2B000C0F7000018000010B5F7000030F80000EB
:10A2C00008228321004824E70C090010F0B5434B15
:10A2D00083B005000191160098423DDC019B002BE4
:10A2E00059D0002840D07C21862301223C4CADB2BD
:10A2F0006552E2542800FAF7D5FE002840D1002E1E
:10A3000044D0384E384F0EE098478623E35C002B4C
:10A3100054D08723E35C002B0ED1FAF777FE002898
:10A320000AD17C23E55A735D9A00002B44D0802B20
:10A3300002D8D359002BE7D1012586230022E2540D
:10A34000FBF722FE8723E35C072B39D0019B002B10
:10A3500007D1F6F73BFA04E0872203210125204BC1
:10A360009954280003B0F0BD012386217C221C4CA7
:10A37000013528006354A352FAF794FE0028BED09A
:10A38000FAF744FE7C23E55A002EBAD1174B184A3F
:10A390005B69A350B5E7FBF7A7FA002D16D086221C
:10A3A00001217C230E4CA154E552124BE35C002B9F
:10A3B00009D07C23E55A9DE7FAF7A0FE0025BCE70B
:10A3C000FAF724FEC2E7FFF79FFDF2E7012386219B
:10A3D0007C22034C6354A352E7E7C046CF0700003A
:10A3E000A8080010D400001024F30000180000108A
:10A3F0007C07000077070000F8B5254C25009C3548
:10A400002B78002B26D0FEF7CBFDC5B22800FEF737
:10A4100059F9230085331F780600002F0AD0002841
:10A4200003D005238734237003E029002B20FAF79B
:10A4300011FEF8BD00280AD0FDF7D2FD0123A43497
:10A440003A00390030002370FFF740FFF1E787340E
:10A450000423E8E7230086331B78002BE9D1FBF7C0
:10A4600093FDFDF7BDFD08232B702300094AA0339F
:10A470001A602300022278331A7085342378064844
:10A480000649002B00D1064901F075FDD1E7C04611
:10A49000A8080010F9A300003009001047F80000D8
:10A4A00051F8000070B5194D2B009C331B781A072A
:10A4B00009D5174B70331B7E002B03D1FBF7DEFA57
:10A4C000FDF7A6FE70BD002BFCD12B0085331E7856
:10A4D0002330C4B2002E04D021000720FAF7BAFDC1
:10A4E000F0E7FBF751FD2B000122A43320001A7086
:10A4F000FEF7E8F8002804D032003100FFF7E6FE4E
:10A50000E0E7042287352A70DCE7C046A80800107F
:10A510001800001010B54520FFF7C4FF10BD10B59E
:10A520004420FFF7BFFF10BD10B54320FFF7BAFF6F
:10A5300010BD10B54220FFF7B5FF10BD10B541208A
:10A54000FFF7B0FF10BDF8B50B4C0600250010005A
:10A55000002300220F000949E8350E604F608A6031
:10A56000CB601031A942F8D10122A8341100FFF7C5
:10A57000ADFE20686168F8BDA80800105009001001
:10A58000C54BF0B51A0099B0A83211685268009115
:10A5900001921A00B8321668576800228733139068
:10A5A000009801991A70F8F721F802900391300091
:10A5B0003900F8F71BF8029A039B04000D0002F023
:10A5C00077F8002801D1029C039D0022B34B2000A4
:10A5D000290002F059F8002801D00024AF4D3200C4
:10A5E000009801993B0003F05DFFF7F7FFFF0022A1
:10A5F00004900591AA4B2000290003F0E1FC020021
:10A600000B000498059902F049F8002823D000981F
:10A6100001990022002302F055F8002400282AD1D5
:10A62000A04D0022029803999C4B02F041F80028AB
:10A6300003D10022994B02920393029A039B2000BC
:10A64000290003F0BDFC02000B003000390002F0CD
:10A6500091FD06000F0000980199139AFFF773FF10
:10A66000914B119010911C788B4D002C05D001243A
:10A67000200019B0F0BD8D4DD3E7109B8C4A5B00D4
:10A680005B08D34204D40924834B87331C70EFE763
:10A69000002200231198109901F0F0FF002806D045
:10A6A0000099019A2B00A83319605A601BE0139A95
:10A6B00030003900FFF747FF7B4B12900E911C785A
:10A6C000002CD4D14B007A4A5B08D342DBD5002260
:10A6D000002312980E9901F0D1FF002809D02B0019
:10A6E000A8331E605F6000220023B0352A606B60D3
:10A6F000BEE7002200231198109901F0C5FF002841
:10A7000008D00022002312980E9901F0D1FF0028F2
:10A7100000D0BBE1002200231198109901F0C8FF7E
:10A72000002808D00022002312980E9901F0ACFFF7
:10A73000002800D0AAE1009A019B3000390002F005
:10A7400019FD00225B4B03F03BFC009A019B149027
:10A7500015913000390003F0A5FEF7F747FF0022FE
:10A760004E4B04000D0001F08FFF002801D00024A3
:10A770004A4D129B08960A930E9B0B970793119BC9
:10A780000493109B0293009B0C93019B0D938023D9
:10A790009B001693002200230498029901F074FF95
:10A7A000002808D0002200230A98079901F080FFB2
:10A7B000002800D078E1002200230498029901F0DB
:10A7C00077FF002811D0002200230A98079901F092
:10A7D0005BFF002809D0002200230498029901F0B1
:10A7E00053FF002800D15FE17CE02B0014981599FD
:10A7F000220003F057FE0C900D91139A0C980D99BE
:10A80000FFF7A1FE284B049002911B781793002BB1
:10A8100000D02CE74B00264A5B08D3425AD50022D1
:10A8200000230498029901F029FF00280DD01A494D
:10A830000C9A0D9BA8310A604B6000240023164D32
:10A84000B0352B606C60002412E72B00149815992A
:10A85000220002F08FFC08900B91139A08980B9934
:10A86000FFF771FE104B0A9007911B781793002B8E
:10A8700000D0FCE64B000E4A5B08D3422AD50022EA
:10A8800000230A98079901F0F9FE002814D0024924
:10A89000089AA8310B9BCEE7A80800100000F03FF3
:10A8A0000000E03C000050BD2F0900100000503DAA
:10A8B000000010800000E03F2B0022002000290053
:10A8C00002F058FC169B0400013B0D001693002B70
:10A8D00000D05FE7002200230498029901F0D4FE23
:10A8E000002808D0002200230A98079901F0E0FE12
:10A8F000002800D0D8E0002200230498029901F03B
:10A90000D7FE002808D0002200230A98079901F0FA
:10A91000BBFE002800D0C7E0009A019B3000390040
:10A9200001F0B2FE00280DD0119A109B12991292DC
:10A9300011910E990E93009A019B009601971600B3
:10A940001F00109180239B000A9332000098019908
:10A950003B0002F00FFCD74B002203F031FB139AAF
:10A9600002900391FFF7EFFDD34D07902B00049168
:10A9700087331C78002C00D079E64B00CF4A5B0867
:10A98000D34200D47FE6002200230798049901F007
:10A9900075FE002804D02B000299039AA83383E6A1
:10A9A00000980199F7F722FE04000D0030003900ED
:10A9B000F7F71CFE22002B000890099101F078FEA9
:10A9C000002801D0089C099D0022BD4B20002900D1
:10A9D00001F05AFE002801D00024B94D009A019BD5
:10A9E0003000390003F05EFDF7F700FE002208900A
:10A9F0000991B44B2000290003F0E2FA02000B0099
:10AA00000898099901F04AFE002818D0079804997F
:10AA1000F7F7ECFDF52300229B0501F03FFE00282F
:10AA200000D130E602980399A34B1A00A8321060B7
:10AA3000516000210022B03319605A6003E7119879
:10AA40001099F7F7D3FD04000D0012980E99F7F74F
:10AA5000CDFD0B0002002900200001F01FFE079B26
:10AA600000280DD11193049B1093029B039C00932B
:10AA700001940A9B013B0A93002B00D065E702E694
:10AA80001293049B029E039F0E93F2E7129B08967B
:10AA90000A930E9B0B970793119B0493109B0293B1
:10AAA000009B0C93019B0D9380239B0010930C98AB
:10AAB0000D99F7F79BFD0090019108980B99F7F716
:10AAC00095FD009A019B04000D0001F0F1FD0028A6
:10AAD00001D000940195009801990022784B01F073
:10AAE000D3FD002803D00023754C009301940A9AEB
:10AAF000079B0498029901F0C1FD002800D082E074
:10AB00000A9A079B0C980D9903F05AFA049A0400CC
:10AB10000D00029B08980B9903F052FA02000B00FB
:10AB20002000290003F0BEFC049A04000D00029BE3
:10AB30000A98079903F0B6FC02000B0020002900D8
:10AB400002F034FE4B005D4A5B0807000E00D34262
:10AB500027D50D99089A0B9B0C9801F095FD0C9C3C
:10AB60000D99002801D1089C0B990B002200380098
:10AB7000310001F093FD002813D10D99089A0B9B29
:10AB80000C9801F095FD0C9C0D99002801D1089CB2
:10AB90000B990B0022003800310001F093FD0028D2
:10ABA0000BD0089A0B9B0C980D9902F0E3FA002247
:10ABB000404B03F005FA07000E00139A38003100ED
:10ABC000FFF7C1FC3C4B050087331B780C00002BC2
:10ABD00000D04CE54B00394A5B08D34200D452E523
:10ABE0000022002301F04AFD002817D0324933002B
:10ABF00008003A00A8300260436000240023B0310E
:10AC00000B604C601FE6089A0B9B0C980D9902F0A4
:10AC1000B1FA0022274B03F0D3F993E70C9A0D9B6E
:10AC200008980B9903F03EFCF7F7E0FC00220E9029
:10AC30000F9100980199234B03F0C2F902000B0019
:10AC40000E980F9901F02AFD0028CFD10022002391
:10AC50000498029901F018FD002807D00022002373
:10AC60002800210001F024FD00280FD1002200233C
:10AC70000498029901F01CFD002825D00022002331
:10AC80002800210001F000FD00281DD00498029941
:10AC90000022084B03F094F90A950490029107945E
:10ACA00008970B96109B013B1093002B00D0FEE6FB
:10ACB000E9E4C0460000E03FA80800100000108052
:10ACC0000000F03F0000D03C002200230A980799C2
:10ACD00001F0DAFC002807D0002200232800210020
:10ACE00001F0E6FC002811D1002200230A98079900
:10ACF00001F0DEFC002800D1C5E40022002328007A
:10AD0000210001F0C1FC002800D1BCE40A98079999
:10AD10000022054B03F054F904950A900791029420
:10AD20000C970D96BEE7C0460000E03FF0B53C4BE7
:10AD3000A5B01590A6331B78181C0F2B00D90F2037
:10AD4000C0B24042F9F777FF354C189019912300B3
:10AD5000A8331A685B680092019300980199230058
:10AD6000B8331E685F6832003B0001F0A1FC002888
:10AD70000CD000220023F83426606760A260E360F4
:10AD8000009A019B0096019716001F00009A019BF4
:10AD90003000390003F086FB32001A901B910098B6
:10ADA00001993B0002F0E6F91E4B002203F008F97E
:10ADB00000230024059314930023209021910293F3
:10ADC0000394059B0C2B2FD1029C039D144E1498C9
:10ADD000370003F0E5FEC8373300386079600022A1
:10ADE0000021D03319605A60029A039B2000290089
:10ADF00003F058FBF7F7FAFB3300B83318605960DB
:10AE0000330000210022C03319605A603300002053
:10AE1000A833B0361C605D603160726025B0F0BD53
:10AE2000A80800100000E03F059BC14C584203F009
:10AE3000B7FE0B0080210200C9050020F7F7B8FE1D
:10AE4000059B1C901D915A1E9341DAB201331E934B
:10AE5000DB009B181F9301235B421693179400237A
:10AE600000240A930B94069307940492049803F029
:10AE700097FE1C9A1D9B03F0A3F804000D00F7F742
:10AE800051FC0890099120002900F7F7B3FBA94A6B
:10AE90002290239108980999A74B03F091F8C023B9
:10AEA00000221B0603F08CF8F5F7F0FF00220023C8
:10AEB00004000D0001F0E2FB002800D0CEE00022EB
:10AEC0009E4B2000290002F055F9089009910200DC
:10AED0000B002000290002F069FC02000B00129018
:10AEE00013911A981B9903F06BF8009A019B0E902E
:10AEF0000F9102F03FF90E9A0F9B0C900D913000CC
:10AF0000390003F0CFFAF3230E900F9112981399A2
:10AF100000229B0501F0C2FB00281FD00C9A0D9B5C
:10AF20000098019901F0CEFB002807D00098019904
:10AF300032003B00F9F71AFE0C900D910E9A0F9B10
:10AF40003000390001F0AAFB002807D0009A019BCD
:10AF500030003900F9F70AFE0E900F911A981B99EC
:10AF6000744A774B03F02CF8229A239B03F028F8BD
:10AF700022002B0003F024F8089A099B04000D001E
:10AF80001000190003F01CF802000B00200029003B
:10AF900002F00CFC049B04000D00159A002B00D05D
:10AFA0008EE020982199FFF7CEFA664A4B005B08A5
:10AFB000D34207D502000B002000290003F000F85F
:10AFC00010901191149B013314935F4B87331B78BE
:10AFD000002B43D1109A119B0698079902F0CAF8EA
:10AFE0000690079110981199F7F700FB02000B00EB
:10AFF00004000D000A980B9902F0BCF81F9B049AFC
:10B000000A900B91934200DD7EE01698179922007A
:10B010002B0001F04DFB002800D178E0069807993D
:10B02000F7F7E4FA00220890099118981999474B0C
:10B0300002F0C6FF0A9A0B9B0C900D910898099993
:10B0400002F098F802000B000C980D9902F0B8FF7E
:10B0500022002B0001F02CFB002858D03A4B8733FC
:10B060001B78002B00D0AFE61C9A1D9B0698079911
:10B0700002F0A6FF059B04000D00002B1AD00298D9
:10B0800003990022324B02F09BFF02000B002000CC
:10B09000290002F06FF8029A039B04000D0003F0F0
:10B0A00001FAF7F7A3FA189A199B01F0EDFA0028B4
:10B0B00000D08BE6059B029403950133059380E64F
:10B0C0000C980D99FFF73FFA159A0C9008910E987D
:10B0D0000F99FFF738FA089B1A4A5B005B08D342C6
:10B0E000BCD54B005B08D342B8D502000B000C98CE
:10B0F000089902F03FF82B00220002F061FF149B38
:10B100001090119102335FE7049B002B07D0129837
:10B11000139900220F4B01F0C1FA00289ED11E9A0C
:10B12000049B944663440493169417959EE6C04688
:10B13000FFFFEF7F182D4454FB21F93F0000F03F43
:10B14000FB21094000001080A80800100000D03F3B
:10B150000000E03F0000A03CF7B5FAF715FF274CD0
:10B1600025009C352F78002F0AD085342378002BBA
:10B1700005D0FDF715FFC1B20620F9F76BFFF7BD4B
:10B18000260086363378002B1FD025007C352A8890
:10B190001B4B9B185878FDF795FA002803D1042320
:10B1A00087342370EBE72B883900019323000124B7
:10B1B000A43322001C70FFF789F8002801D03770F3
:10B1C000DDE7019B34702B80D9E7230085331B78A2
:10B1D000002B0FD0FCF704FF0C232B702300094A2F
:10B1E000A0331A600223783407490848237000F01E
:10B1F000C2FEC4E7FEF72CFDC1E7C046A808001058
:10B20000D400001059B100005AF8000030090010B5
:10B2100010B5FAF7B9FE084B1A00863211780029EA
:10B2200004D000231370F9F7F1FE10BD7C331888A9
:10B230000A00FFF74BF8F8E7A808001010B5064B16
:10B2400086331B78002B05D0FEF75EFEFA208000C7
:10B25000F4F7FAFF10BDC046A8080010F8B5FAF7D9
:10B2600093FE2D4C26009C363378002B2BD0FDF717
:10B2700097FEC5B22800FDF725FA230085331E7816
:10B280000700002E04D029004F20F9F7E3FEF8BD97
:10B29000FCF7A6FE002F11D02500012386352B7068
:10B2A000FEF732FEFAF720FB3800FFF73FFDF5F717
:10B2B0008DFA2E700123A4342370E8E723000422C2
:10B2C00087331A70F6E7250086352B78002B13D0CC
:10B2D00026007C363788114BDB195878FDF7F2F9D8
:10B2E000002806D0FFF722FD012337802B70A434FD
:10B2F000E2E787340423DFE7FCF772FE09233370AB
:10B300002300074AA0331A6002237834054906480F
:10B31000237000F030FEBAE7A8080010D400001037
:10B320005DB2000063F8000030090010F7B5FAF7CD
:10B330002BFE364C26009C363578002D2BD0FDF7A1
:10B340002FFEC5B22800FDF7BDF9230085331E7816
:10B350000700002E04D029005020F9F77BFEF7BD2E
:10B36000FCF73EFE002F11D02500012386352B70FF
:10B37000FEF7CAFDFAF7B8FA3800FFF701F9F5F75A
:10B3800025FA2E70A43401232370E8E72300042259
:10B3900087331A70F6E71E4B1B78002B25D026004A
:10B3A0007C3632881B4B27009B185878FDF78AF9AA
:10B3B0008737002816D033880193FFF7E1F8019B07
:10B3C000012233802300A4331A703B78092B04D167
:10B3D000F9F71CFE3D708634D5E7002BFBD00C4BF3
:10B3E0001D70BCE704233B70B9E7FCF7F9FD0923A6
:10B3F00033702300084AA0331A60022378340749C7
:10B400000748237000F0B7FDA9E7C046A808001060
:10B410002E090010D40000102DB3000072F80000B7
:10B42000300900104F4B10B51A694F4901321A61AB
:10B430004E4A1268D2B2302A66D01AD8182A0ED0D4
:10B4400005D8082A36D0102A44D008234EE0202AF6
:10B4500069D0282AF9D1D8689A69904248D2DA6826
:10B46000501CD86001339B18DB7F414ADBB213606C
:10B47000EBE7482A57D009D8382A4DD0402AE4D1E2
:10B48000DA690423012A4BD10B60DEE7502A53D03E
:10B49000582ADAD1364A12689868D2B2441C9C60A5
:10B4A0001C00383422540222FF325A608023F13AC1
:10B4B000DB0552E00022DA60D868421CDA605A1CD0
:10B4C0001218D27F2A48D2B2026028220A60273A94
:10B4D0005A6010BD00229A60DA68501CD8600133AF
:10B4E0009B18DB7F224ADBB2136028230B60F0E756
:10B4F0008022D869D205002801D02023B7E7022096
:10B50000FF3058601023B2E780221020D20510606F
:10B5100008220A60FA32DBE7822252005A6094E77E
:10B520008022D205A3E780221020D20510600822D5
:10B530000A600422FF32CBE70D4A12689868D2B243
:10B54000441C9C601C0038342254DA699868531EED
:10B550000422834203D98023DB051A6075E70A6061
:10B5600073E7C046180000101800004004000040B7
:10B5700008000040202130B5064A074C0378002B14
:10B5800001D1180030BD013015680D42FCD0236098
:10B59000F4E7C04614800040008000400E22174BA4
:10B5A00010B51B681340062B12D1154B90321B6847
:10B5B000134205D0134ADBB25360134B1B6810BD16
:10B5C000DB07FCD5104B1868C0B2F4F72DFEF6E788
:10B5D000042BF7D00C2B05D10A4AF43351680B43E6
:10B5E0005360ECE7022BEAD1054B1A68054B920633
:10B5F00002D500229A60E2E70122FBE708800040C2
:10B600001480004028100010008000400122034BED
:10B610001A60034AD3680133D36070470080014049
:10B62000980000100122034B1A60034A136901338A
:10B630001361704700400140980000100122034B45
:10B640001A60034A53690133536170470000014097
:10B65000980000100122034B1A60034A93690133DA
:10B660009361704700C0004098000010074A084BE3
:10B670005169013102D1D9690131D9615169013171
:10B6800051611A6A01321A627047C04618000010F0
:10B69000980000101B4B10B59A6D002A2AD0DA6D65
:10B6A0000132DA65184B9868FAF7F6FB8022174BDF
:10B6B0000121DA679218DA678022D200DA678022E5
:10B6C0005201DA6780221201DA6780229200DA677B
:10B6D00000230F4A494213600E4A11600E4A13605C
:10B6E0000E4A136001220E4B1A60F4F7E9FCC046C3
:10B6F000C04610BD08220B4B87331A70F5F766F869
:10B70000F7E7C046180000100000001004E100E058
:10B71000048204400882044004C000403CC0004051
:10B7200000C00040A8080010F7B5F4F7A3FDC04A18
:10B73000012413681B0B1B031360BE4A13681B0B09
:10B740001B031360BC4A13681B0B1B031360BB4A2B
:10B7500013681B0B1B0313600022B94B1A60B94B13
:10B760001C601A601C601A682242FCD02322B64B6F
:10B7700001201A60FAF790FBF4F77CFD40213F208E
:10B78000B24B1A688A431A60B14A1060B14A146019
:10B790001A688A431A60FCF717FBFCF70BFBFAF7F1
:10B7A00055FBF4F7EFFF0021AB48F4F771FD0021E2
:10B7B000AA48F4F76DFDF4F76BFEF4F739FEA84CD8
:10B7C000092248340021200000F0E0FB0020E07155
:10B7D000F5F72CF8A34D002822D0F4F7EDFD0C234B
:10B7E000184002D02378184320709D4C48342378A9
:10B7F0005B0711D5F4F7AAFDA378002B03D0237AB9
:10B80000012B02D80133237201E02B6A6B62002303
:10B81000934A2B624832D3700022914B48331A70FE
:10B820008F4B4833DB79002B01D1F4F78FFDFA23DE
:10B8300000269B002E626B62FAF78EFAF0228A4C89
:10B84000D2003100200000F0A1FB23000222A4332B
:10B85000FF321A802300FD3AA6331A7023000B3200
:10B8600078331A70814A82490C32824800F083FB97
:10B87000FAF766FBFAF7B2F8FEF746FBF9F768FF4E
:10B88000061E00D143E1EF22D200A35C002B04D0BE
:10B890000023A35422007C32138000222300AA61DB
:10B8A00087331F78974216D01A70FAF797F8AA696B
:10B8B000714B9A4203D9FCF7E9FA0023AB61FEF71A
:10B8C00023FBEF23DB00E35C002BD7D103210A200D
:10B8D000F4F728FED2E7A02E66DDA021300000F0AC
:10B8E000AFFE0D2927D1FCF77BFBFA27634800F058
:10B8F00037FB0126FF00624B6248995D013600F07C
:10B900002FFBBE42F7D1CC270026FF0033000933BE
:10B91000FF33E15C5B48013600F022FBBE42F5D10B
:10B92000594800F01DFB594E300000F019FB300063
:10B9300000F016FBB9E7112914D1FCF751FBFA22EC
:10B940003900D2004E4800F021FB2300EF227C3367
:10B950001F800123D2004E48AF62A35400F000FBC9
:10B960004A48E5E7072907D1230086331B78002BD7
:10B970009BD1FEF7EBF898E7062907D12300863321
:10B980001B78002B91D1FEF763F98EE732298CD119
:10B99000FA223900D2003A4800F0F8FA23007C334A
:10B9A0001F80FCF71DFB80E723009C331B78002BD6
:10B9B00074D033003D3B012B21D92821300000F009
:10B9C0003FFE12291BD004230A009A43012A16D0F5
:10B9D0003200153A132A03D82E4BD340DB070ED47E
:10B9E00033000422143B934304D1230083331B7898
:10B9F000002B04D133000422373B93430FD1F0B224
:10BA0000F9F772FA1648703000F0F8FA230078332C
:10BA10001B78984200D048E7FCF7FAFB45E7142969
:10BA2000F0D81D4BCB40DB07ECD52831C8B2E7E797
:10BA300000800050008001500080025000800350C0
:10BA40004080044044800440088004403882044020
:10BA500024800440D8800440984004409C40044026
:10BA60001800001098000010A80800100000001036
:10BA7000D8F60000300900105702000087F80000D7
:10BA8000D40000107DF8000010FA00008EF80000CD
:10BA900081F80000F3EE0F001091190023008533A8
:10BAA0001B78F6B23000002B29D0F9F72DFA0028C8
:10BAB00024D1202332009A43122A1FD033000222BD
:10BAC0009343012B1AD03300523B012B16D9612E20
:10BAD00014D02633DBB2102B03D84E4ADA40D307FA
:10BAE0000CD42821300000F053FBFB230539194208
:10BAF00004D033007F33DBB21E2B03D83000F9F7BC
:10BB0000F3F9D2E600213000F9F7A4FACDE6EF23ED
:10BB1000DB00E35C002B00D1C9E63F4A917B537BFD
:10BB2000994200D1AAE6937BD318DE7B937B013345
:10BB3000DBB293735BB2002B01DA002393730D2EFB
:10BB400003D00A2E01D0202E28D12F002C37380008
:10BB5000FAF734F80A2201900021380000F016FAB2
:10BB60002E4B5F612E4BE35C002B03D131002D483F
:10BB700000F0F6F9019BFF2B00D97FE622007C3212
:10BB8000138829498B4238D9AB6A28498B423BD864
:10BB9000274A0199D1540133AB626FE6082E01D0D8
:10BBA0007F2E18D11E4BE35C002B14D12B001B4FB2
:10BBB0002C337A699A420ED908211A4800F0D0F93C
:10BBC0002021184800F0CCF90821164800F0C8F9E7
:10BBD0007B69013B7B613300303B092B9DD8104BC7
:10BBE000E35C002B03D131000E4800F0B9F90B4A99
:10BBF0005369591C51611E708FE701339BB213804A
:10BC000001990C4AD15439E600231380EF22D20067
:10BC1000A35433E611310100281000100000001079
:10BC200077070000A1F70000CE0700005F060000C4
:10BC3000B0090010D400001070B500241E5D051975
:10BC4000002E08D1121B1300002B07DCD043C017B5
:10BC50001040001970BD06550134EFE72970013B13
:10BC60000135F1E7F8B505000C001E00571E092B41
:10BC700016D90A21180000F005FA210003003A0045
:10BC80002800FFF7EFFF04002D1830000A2100F014
:10BC90007FFA30312970601CF8BD2C70013F0135EE
:10BCA000002FFADC141E00DC0124013CEDE7F0B5A6
:10BCB00085B00B9E040003910A9F551E002E01D1F2
:10BCC000092F1DD90A2200233800310000F066FA3E
:10BCD0002A000090019120000399FFF7E8FF05007A
:10BCE0002418380031000A22002300F057FA681C9B
:10BCF0003032227005B0F0BD039B013D237001344A
:10BD0000002DF9DC151E00DC0125013DE9E7F7B542
:10BD10000F00D9171E005B184B4004000193551EFD
:10BD2000092B16D918000A2100F0ACF90300002EE7
:10BD300000DA43422A0020003900FFF7E8FF05003F
:10BD4000241801980A2100F023FA3031681C217070
:10BD5000FEBD002E00DA951E23006119CA1A002AC2
:10BD60000BDCE843C017054064196B1C002EE8DAB1
:10BD70002D221D0022700134E3E71F700133EDE72F
:10BD800073B5069E04001D0010003309013A002B14
:10BD900011D0009320002B00FFF7F2FF24180F238F
:10BDA0001E40F3B2092E0DD830330130237076BD1A
:10BDB0002170013A0134002AFADC002800DC01205D
:10BDC0000138ECE7002D01D03733EEE75733ECE7CD
:10BDD000F0B585B0040003911D00002801D00023B8
:10BDE0000370002630001378002B00D092E0039AF5
:10BDF000B24200D99AE00023013C2370013E96E054
:10BE00005178252902D1217002328CE0302924D0CA
:10BE1000531C029320239C46029B1B782D3B5A42C5
:10BE20005341029AD31800220293029B1B781F00F1
:10BE3000303F092F15D9039997198F4201D98A1BD1
:10BE4000D2B2692B46D015D8632B5ED0642B41D07B
:10BE5000582B4ED00126764269E0931C02938C4603
:10BE6000DAE70A214A439A18029B303A0133D2B2E8
:10BE70000293DAE7732B41D01FD86C2BEAD1029BD7
:10BE80005B786C2B14D1029B9B78752B10D1029B95
:10BE900007350233072102932B008B431D001868DE
:10BEA000596800900191614620000835FFF7FFFEB8
:10BEB000029A24180132361895E7752B12D0782B88
:10BEC000C8D12B682F1D0093002361462000FFF787
:10BED00057FF05E02B68614620002F1DFFF717FF75
:10BEE0003D00E5E72B68614620002F1DFFF7BAFEF5
:10BEF000F6E72B682F1D00930123E6E72B686146C8
:10BF000020002F1DFFF798FEEAE72B680120237021
:10BF10000435CDE70399B14200D86CE7252B00D159
:10BF20006EE701322370013601345CE72370300084
:10BF300005B0F0BD10B513000A006421FFF748FFFB
:10BF400010BD00B59BB00A00010001A8FFF7F2FF89
:10BF5000632800DDFEE701A8FFF70CFB1BB000BD66
:10BF60000FB407B504A901C90191FFF7EAFF03B0B7
:10BF700008BC04B018470EB403B503AA02CA019264
:10BF8000FFF7D8FF02B008BC03B01847F0B50500B2
:10BF9000830704D003009A189A4217D1F0BD03001A
:10BFA000032AF8D9131F0F049B080C063C439E007C
:10BFB00036180C430F0204363C4310C5B542FCD181
:10BFC000032401339B00C3182240E4E719700133B6
:10BFD000E2E710B5814208D20139431E002A00D1A0
:10BFE00010BD8C5C9C54013AF8E700238142F7D9DC
:10BFF0009A42F5D0CC5CC4540133F9E70200030047
:10C00000981A0133591E09780029F9D170470300A5
:10C010000A781A70002A00D1704701310133F7E71E
:10C02000002210B5835C8C5CA34201D0181B10BDAC
:10C030000132002BF6D11800F9E7FEE7FEE7000019
:10C04000002370B50A480B490B4C1A188A4207D3D3
:10C0500000210A4B0A4A934206D3FFF765FBFEE72D
:10C06000E55C01331570F0E719700133F3E7C04662
:10C070000000001018000010DCFA0000180000108A
:10C08000C0110010002243088B4274D303098B4275
:10C090005FD3030A8B4244D3030B8B4228D3030C98
:10C0A0008B420DD3FF22090212BA030C8B4202D33A
:10C0B0001212090265D0030B8B4219D300E0090A62
:10C0C000C30B8B4201D3CB03C01A5241830B8B426B
:10C0D00001D38B03C01A5241430B8B4201D34B0354
:10C0E000C01A5241030B8B4201D30B03C01A5241B9
:10C0F000C30A8B4201D3CB02C01A5241830A8B423E
:10C1000001D38B02C01A5241430A8B4201D34B0226
:10C11000C01A5241030A8B4201D30B02C01A52418A
:10C12000CDD2C3098B4201D3CB01C01A524183093E
:10C130008B4201D38B01C01A524143098B4201D378
:10C140004B01C01A524103098B4201D30B01C01AA3
:10C150005241C3088B4201D3CB00C01A524183081D
:10C160008B4201D38B00C01A524143088B4201D34A
:10C170004B00C01A5241411A00D2014652411046AA
:10C180007047FFE701B5002000F006F802BDC04689
:10C190000029F7D076E770477047C046002B11D1D1
:10C1A000002A0FD1002900D1002802D00021C94364
:10C1B000081C07B4024802A14018029003BDC04603
:10C1C000D9FFFFFF03B4684601B5029800F006F8F6
:10C1D000019B9E4602B00CBC7047C046F0B54F466E
:10C1E0004646D646C0B5040082B00D00914698463A
:10C1F0008B422FD82CD04146484600F0B1F8290098
:10C200000600200000F0ACF8331A9C46203B9A460A
:10C2100000D576E04B46524693401F004B4662469F
:10C2200093401E00AF4228D825D05346A41BBD41E1
:10C23000002B00DA7BE0002200230092019301230F
:10C24000524693400193012362469340009318E0C5
:10C250008242D0D900220023009201930A9B002B36
:10C2600001D01C605D600098019902B01CBC904632
:10C270009946A246F0BDA342D7D9002200230092DE
:10C2800001936346002BE9D0FB07984641467208AC
:10C290000A437B0866460EE0AB4201D1A2420CD8AD
:10C2A000A41A9D41012024196D410021013E24184A
:10C2B0004D41002E06D0AB42EED9013E24196D410E
:10C2C000002EF8D100980199534600196941002BBE
:10C2D00023DB2B005246D3402A006446E2401C0078
:10C2E00053461500002B2DDB26005746BE40330079
:10C2F00026006746BE403200801A994100900191A5
:10C30000ACE7624620239B1A4A46DA406146130096
:10C3100042468A4017001F4380E7624620239B1A4B
:10C320002A0066469A402300F3401343D4E762464E
:10C33000202300219B1A0022009101920122DA4061
:10C34000019280E72023624626009B1ADE402F00E0
:10C35000B0466646B74046463B003343C8E7C04652
:10C3600010B5002903D100F007F8203002E0081CC6
:10C3700000F002F810BDC0461C2101231B049842A6
:10C3800001D3000C10391B0A984201D3000A083966
:10C390001B09984201D30009043902A2105C40181D
:10C3A0007047C046040302020101010100000000C1
:10C3B00000000000C317C0185840704770B50568EA
:10C3C0000400002D22D01349280000F053F8C201C8
:10C3D000121A9200131ADA00D21A92001218D3001D
:10C3E000D2180D4BAA1A5A4303051B1A9B001B189F
:10C3F0009B001B181B011B1A9B00181A8000801839
:10C4000005D5064BC3185800400801E00448030056
:10C41000236070BD1DF30100A7410000FFFFFF7FF7
:10C4200067B7E12A70B50400830717D102680F4B84
:10C43000D31893430E4A150013420FD104300268FB
:10C440000A4BD31893432B4208D104300268074BA0
:10C45000D31893432B42F1D000E001300378002B36
:10C46000FBD1FFF7D4FD200070BDC046FFFEFEFEED
:10C470008080808003460B437FD4002243088B4298
:10C4800074D303098B425FD3030A8B4244D3030B5B
:10C490008B4228D3030C8B420DD3FF22090212BA20
:10C4A000030C8B4202D31212090265D0030B8B429C
:10C4B00019D300E0090AC30B8B4201D3CB03C01A86
:10C4C0005241830B8B4201D38B03C01A5241430B61
:10C4D0008B4201D34B03C01A5241030B8B4201D351
:10C4E0000B03C01A5241C30A8B4201D3CB02C01ABC
:10C4F0005241830A8B4201D38B02C01A5241430A34
:10C500008B4201D34B02C01A5241030A8B4201D322
:10C510000B02C01A5241CDD2C3098B4201D3CB01C9
:10C52000C01A524183098B4201D38B01C01A524178
:10C5300043098B4201D34B01C01A524103098B427C
:10C5400001D30B01C01A5241C3088B4201D3CB0067
:10C55000C01A524183088B4201D38B00C01A52414A
:10C5600043088B4201D34B00C01A5241411A00D2FA
:10C5700001465241104670475DE0CA0F00D0494263
:10C58000031000D34042534000229C4603098B42D3
:10C590002DD3030A8B4212D3FC22890112BA030A5B
:10C5A0008B420CD3890192118B4208D389019211DD
:10C5B0008B4204D389013AD0921100E08909C30962
:10C5C0008B4201D3CB01C01A524183098B4201D364
:10C5D0008B01C01A524143098B4201D34B01C01A4F
:10C5E000524103098B4201D30B01C01A5241C308C7
:10C5F0008B4201D3CB00C01A524183088B4201D336
:10C600008B00C01A5241D9D243088B4201D34B0050
:10C61000C01A5241411A00D20146634652415B1092
:10C62000104601D34042002B00D549427047634673
:10C630005B1000D3404201B50020FFF7ADFD02BD05
:10C640000029F8D016E7704702B47146490849003E
:10C65000095C49008E4402BC7047C0468446101CE9
:10C6600062468C46191C634600E0C0461FB501F0C7
:10C670003FFC002801D40021C8421FBD10B501F0C5
:10C6800097FB4042013010BD10B501F031FC00288D
:10C6900001DB002010BD012010BDC04610B501F027
:10C6A00027FC002801DD002010BD012010BDC04680
:10C6B00010B501F0B9FB002801DC002010BD0120FD
:10C6C00010BDC04610B501F0AFFB002801DA002014
:10C6D00010BD012010BDC046F0B5DE4657464E469F
:10C6E00045469446E0B595B09B461E9B65469946E7
:10C6F0001F9B04009846209B60460293219B029A50
:10C700009A46594653460A9501F05AFC239F229EA9
:10C710000490059132003B004846414603960B9732
:10C7200001F04EFC3D0006000F00039A2B000A9812
:10C7300059460C960D9701F043FC4A460690079126
:10C7400043460298514601F03BFC32003B00089002
:10C7500009910498059901F0A5FE089A099B060025
:10C760000F000698079900F005FD32000090019136
:10C770003B0030003900FFF781FF00280DD0009A00
:10C78000019B200026606760A260E36015B03CBC9E
:10C7900090469946A246AB46F0BD0098019902002A
:10C7A0000B00FFF76BFF0028E9D10A995B468C4626
:10C7B0000A0060465946654601F074FE4A461090EC
:10C7C000119143464846414601F06CFE0B000200C1
:10C7D000FFF754FF3822434258416B469B181870AC
:10C7E0004A46434641464846FFF748FF3822431E23
:10C7F00098416B469B181B782A0003400E93280033
:10C800005B465946FFF73AFF002800D123E1109814
:10C81000119902000B00FFF731FF002800D01AE148
:10C8200059460022D34B002900DAD34B9B460E9B7E
:10C830000A925A425341D14A5B421340CD4A944630
:10C840006344424600215B00D20FD2075B081343CA
:10C8500089469846029A534602985146FFF70EFFC2
:10C86000002800D168E10B99039D8C460B002A003B
:10C8700028006146FFF702FF002800D150E10123A4
:10C880000E93029A53460298514601F00BFE129005
:10C8900013910B99039D8C462A000B0028006146DA
:10C8A000654601F0FFFD0B000200FFF7E7FE4022A6
:10C8B000434258416B469B181870039A2B0029007D
:10C8C0000398FFF7DBFE4022431E98416B469B18FE
:10C8D0001B78029A03401093029853465146FFF783
:10C8E000CDFE002868D01298139902000B00FFF7C4
:10C8F000C5FE002860D1524600259E4B002A00DA72
:10C900009D4B9A46109B9D4A013B1340994A0295C4
:10C91000944663440B9A5B00D70F00220A9E5B0883
:10C92000FF073B4303920B9332005B4630005946AE
:10C93000FFF7A4FE002800D138E14A4643464846A6
:10C940004146FFF79BFE002800D125E1029A53469D
:10C950000A98594601F034FB0B9D06000F00039A1C
:10C960002B004846414601F02BFB02000B00300033
:10C97000390001F097FD0022814B01F021FB039A61
:10C980002B0006000F000A98594601F019FB029A85
:10C990000090019153464846414601F011FB0200C8
:10C9A0000B000098019900F0E5FB0022744B01F0A8
:10C9B00007FB00900191E2E6109B002B00D0A4E061
:10C9C0000E9B002BC2D10498059902000B0001F0C8
:10C9D00069FD0E900F910498059902000B00FFF776
:10C9E0004DFE002846D00E980F9902000B00FFF76D
:10C9F00045FE00283ED10A9E5B4632003000594673
:10CA0000FFF73CFE002800D1A0E04A4643464846D6
:10CA10004146FFF733FE002800D1B3E0029A5346A7
:10CA200002985146FFF72AFE002800D198E0039FA4
:10CA30000B9E3A00330038003100FFF71FFE00283C
:10CA400084D100220B991300914201DA80231B0646
:10CA500003920B937AE70E9B002B00D111E7002283
:10CA600059461300914201DA80231B069B460A9225
:10CA7000404BE6E60C980D9902000B0001F012FD08
:10CA8000049005910C980D9902000B00FFF7F6FD3C
:10CA9000002807D00498059902000B00FFF7EEFD6F
:10CAA0000028A8D00698079902000B0001F0FAFCB4
:10CAB000049005910698079902000B00FFF7DEFD30
:10CAC000002807D00498059902000B00FFF7D6FD57
:10CAD000002890D00898099902000B0001F0E2FCB0
:10CAE000049005910898099902000B00FFF7C6FD14
:10CAF000002800D143E60498059902000B00FFF7D7
:10CB0000BDFD002800D03AE675E7002552462B000F
:10CB1000AA4201DA80231B069A460295154BF9E6D4
:10CB200000220B991300914201DA80231B060B931C
:10CB3000012303920E93A4E652464D464B464A45C6
:10CB400001DA80231B0602959A468CE600265A4697
:10CB50003300B24201DA80231B060A969B4654E753
:10CB6000002552462B00AA4201DA80231B060295BB
:10CB70009A465CE70000F03F0000F0BF000010C0E4
:10CB80000000F07F002241461300914201DA802329
:10CB90001B069146984641E7002241461300914208
:10CBA00001DA80231B0691469846CFE600265A46B6
:10CBB0003300B24201DA80231B060A969B46BCE68C
:10CBC000F0B557464E464546DE46E0B58BB0169961
:10CBD000824689461799189888461999149E8B465B
:10CBE00041464C005946159F4900019203930500A8
:10CBF000059002004B084846610802960497FFF72B
:10CC000043FD00284BD02A005B4648464146059527
:10CC100000F0CCFD04000D0002000B004846414628
:10CC200001F0CEF9059A5B4600F0A4FA22000690C6
:10CC300007912B000198039901F0C2F932003B00E3
:10CC40000296049700F096FA069A079B00F0AEFD54
:10CC500022002B0006000F000298049901F0B0F9A1
:10CC6000019A039B01F01EFC069A079B00F09EFDB3
:10CC7000320004000D003B0030003900FFF7FEFCDD
:10CC800000283ED0534650461E605F609C60DD60C9
:10CC90000BB03CBC90469946A246AB46F0BD059E03
:10CCA0004A4643463000594600F080FD04000D001E
:10CCB00002000B003000594601F082F94A46434613
:10CCC00000F058FA06000F00029A049B2000290089
:10CCD00001F076F9019A039B00F04CFA32003B0018
:10CCE0000696079700F062FD019A039B06000F006D
:10CCF0002000290001F064F902000B000298049959
:10CD0000B0E722002B0020002900FFF7B7FC002825
:10CD1000B8D10022002348464146FFF7AFFC002867
:10CD200028D00022002305985946FFF7A7FC0028C9
:10CD300020D00399019A0B000198FFF79FFC00286F
:10CD400000D176E143460024DE4D002B01DA0024B9
:10CD5000DD4D019A039B2000290001F031F9029A70
:10CD600006000F0020002900049B01F029F90400AF
:10CD70000D0087E7019803990690079102000B00C8
:10CD80000698079901F08EFB089009910399019A82
:10CD90000B000198FFF772FC00287ED008980999D3
:10CDA00002000B00FFF76AFC002876D14A46434692
:10CDB0004846414601F076FB02000B00FFF75EFC9F
:10CDC000002800D146E105995B460A000800594653
:10CDD00001F068FB02000B00FFF750FC002800D1B7
:10CDE00095E0BA4B039A029FD20F049ED2071343D9
:10CDF00001933A0033003800310001F053FB3A0050
:10CE000004000D00330038003100FFF737FC002824
:10CE100000D153E122002B0020002900FFF72EFC57
:10CE2000002800D04AE1A94C049B0022DB0FDB075D
:10CE30001C434846019B414601F0C2F8230006000E
:10CE40000F0000220598594601F0BAF802000B00C5
:10CE50003000390000F08EF900229A4B01F0B0F852
:10CE60002300002206000F004846414601F0A8F8C2
:10CE7000002204000D00019B0598594601F0A0F81E
:10CE800002000B002000290001F00CFB00228D4B5A
:10CE900001F096F804000D00F4E60298049906905B
:10CEA000079102000B000698079901F0FBFA069023
:10CEB00007910499029A0B000298FFF7DFFB002804
:10CEC00000D1C7E00698079902000B00FFF7D6FBD8
:10CED000002800D0BEE04A4643464846414601F09D
:10CEE000E1FA02000B00FFF7C9FB002800D1B1E016
:10CEF00005995B460A000800594601F0D3FA0B0079
:10CF00000200FFF7BBFB0023984200D06AE70599B7
:10CF10005B4689460A000800594601F0C3FA4A46B2
:10CF2000069007915B4648465946FFF7A7FB002845
:10CF300000D1A7E60698079902000B00FFF79EFBB9
:10CF4000002800D09EE60898099902000B00FFF720
:10CF500095FB002800D195E6029989460A000499BC
:10CF600048460B0001F09EFA0B000200FFF786FB1B
:10CF70000023984200D185E64246D70F059EFF0761
:10CF80003B433200994630005B46594601F08AFA2D
:10CF9000320004000D005B4630005946FFF76EFB7F
:10CFA000002800D18CE022002B0020002900FFF790
:10CFB00065FB002800D083E0444E5B46DB0FDB07B7
:10CFC0001E4300224B460198039900F0F9FFB0463A
:10CFD0003300049E04000D0000223100029800F08E
:10CFE000EFFF02000B002000290000F0C3F8002230
:10CFF000002300F0E5FFB34600224B4606000F0079
:10D000000298594600F0DCFF002204000D00434660
:10D010000198039900F0D4FF02000B0020002900C2
:10D0200001F040FA0022002300F0CAFF04000D00C6
:10D0300028E60499029A0B000298FFF71FFB0028CC
:10D0400000D07FE60399019A0B00019801F02AFABB
:10D05000089009914A4643464846414601F022FA63
:10D060004A4606900791434648464146FFF706FB6D
:10D07000002800D14BE70698079902000B00FFF744
:10D08000FDFA002800D042E70898099902000B0039
:10D09000FFF7F4FA002800D1F4E5029989460A0066
:10D0A000049948460B0001F0FDF902000B00FFF760
:10D0B000E5FA002800D1E5E5044B5DE70024B3E67E
:10D0C00000267AE70000F07F0000F0FF0000F03F4C
:10D0D00070B500220C4B04000D00FFF7F3FA002896
:10D0E00004D12000290001F025FD70BD064B00226F
:10D0F0002000290001F0D6F901F01CFD80231B0659
:10D100009C466044F1E7C0460000E04170B5002253
:10D110000B4B0D00040000F053FFFFF7D9FF060092
:10D1200001F078FD0022074B00F04AFF02000B00DF
:10D130002000290001F0B6F9FFF7CAFF310070BDE9
:10D140000000F03D0000F04170B50600080001F05D
:10D1500061FD0022064B00F033FF0D00040030009B
:10D1600001F058FD2B00220000F004F870BDC0460D
:10D170000000F041F0B54F464646D6460C00090384
:10D18000C0B5490A470F5E0039431F03DB0F9C46B9
:10D1900065007B0A570F1F436D0DE40F760DA14606
:10D1A000C000B846D200AB1B64457BD0002B5FDDCE
:10D1B000002E00D0A4E03E00164300D112E15E1E16
:10D1C000002E00D09EE1871A4346B84280410125D7
:10D1D000C91A4042091A0B0200D431E149024E0A31
:10D1E000002E00D16EE13000FFF7C6F80300083BC7
:10D1F0001F2B00DD61E120223900D21A9E40D14070
:10D200009F400E439D4200DD51E15D1B6B1C1F2BB7
:10D2100000DD7CE12021C91A3D0030008F408840AC
:10D22000DD40791E8F41310007222843D940002577
:10D2300007433A40002A09D00F233B40042B05D076
:10D240003B1DBB42BF417F42C9191F000B0200D4E6
:10D2500026E26A1CC64B55056D0D9A4200D106E1C7
:10D26000C44AFF080A40530752023B43120B8EE0A8
:10D27000002B00D0B8E06B1C5B055B0D012B00DCC4
:10D2800030E1871A4346B842B641CB1A76429E1B1C
:10D29000330200D54CE13B003343A1D100220024EE
:10D2A000002570E0002B00DCE5E0002E00D183E0DB
:10D2B000AF4EB54260D0802636043743B846382B8F
:10D2C00000DC3EE1434613431F007A1E97413F189E
:10D2D00087428041404209180B0200D4B0E0A44BC1
:10D2E00001359D4200D1C3E0A24A7B080A400121DA
:10D2F0000F401F435108D30707221F433A4099E7C5
:10D300009B4EB54238D0802636043743B846382B7A
:10D3100000DDDCE01F2B00DC30E11E004746203E34
:10D32000F740BC46202B04D04026F31A46469E40C8
:10D330003243170063467A1E97411F43CCE0002B0F
:10D3400000D104E24346134300D159E14B07C00822
:10D3500018438023C9081B03194208D04546ED082D
:10D360001D4204D14346D008590708432900420F03
:10D37000C9007F4D1143C0004B07CA087C49C00853
:10D3800003438D4268D012036D05120B6D0D002111
:10D3900012031800130B0A0D12051A43764B2D05C4
:10D3A00013402B435B00E4075B08234319001CBCBC
:10D3B00090469946A246F0BD3E00164312D05E1E2E
:10D3C000002E00D000E1871887428041414440424E
:10D3D000091801250B0233D5022585E76446330081
:10D3E000414610001D00C7E7002D00D0DAE00C0018
:10D3F0000443F3D05C1C00D19FE15D4CA64200D1F8
:10D400002FE1DB43382B00DD66E11F2B00DD83E1DC
:10D4100020240500E41A0F00DD40D940A040434617
:10D42000A7405B1A441EA04198462F433843171A61
:10D43000BA42924143465242991A64463500CAE6BE
:10D4400007223A40002A00D0F6E64B07CA084849AE
:10D45000FF083B438D4296D11900114300D19EE154
:10D46000802109030A431203120B414D8FE7150077
:10D47000002200238BE7002B00D0C7E06B1C5F0568
:10D480007F0D012F00DCF1E0394DAB4200D1B9E056
:10D4900085180A00854289414244494251180722B1
:10D4A000CF076D082F4349083A401D00C2E6072206
:10D4B0003049ED1A31403A40BCE63E0028388640FB
:10D4C00000279FE63800FEF757FF20308EE64346E0
:10D4D00013431F007A1E9741C71BB8428041404248
:10D4E000091A78E60E003B0006431343002D61D174
:10D4F000002E00D0F4E0002B00D11BE1644639007F
:10D50000100039E71A4FBB427AD03300FFE63000F3
:10D510001F3DE840202B03D04021CB1A9E403743CB
:10D520007B1E9F41072207433A400021002589E7DF
:10D53000171A4346BA42B641591A76428E1B6446C0
:10D540004EE61F2B00DDADE020264746F61AB74019
:10D55000B9461700B246DF404E463E4337005646B6
:10D56000B240561EB24117434246DA408918AEE631
:10D57000FF070000FFFF7FFFFFFF0F8020264746C9
:10D58000F61AB740B9461700B246DF404E463E4352
:10D5900037005646B240561EB24117434246DA4063
:10D5A000891A99E77F4CA6425BD0802424045B4211
:10D5B000214327E7002E0CD1002B00D1CBE064469D
:10D5C00039001000774DD7E6764FBB4218D03300B4
:10D5D00075E6002B14D04B07C00818438023C908F8
:10D5E0001B03194207D0FC081C4204D17907D0085C
:10D5F0000843E14621004C46420FC9001143C000D8
:10D60000684DB9E61D0000220023C0E6002D5BD165
:10D610000D00054300D1E2E65D1C00D1B0E0614D94
:10D62000AE421FD0DB43382B71DC1F2B00DD96E0B0
:10D6300020250F00ED1AAF40B9460700AA46DF408B
:10D640004D463D432F005546A840D940451EA841B0
:10D6500088440743BF1897429241514241443500E4
:10D660003AE6644635004146100085E60B00034368
:10D67000002D00D063E6002BF5D04346134300D1C4
:10D680007AE68718874280410722414440420918C0
:10D690003A400B0200D4D5E6434B01351940C9E5A9
:10D6A000380069E61E004746203EF740BC46202B66
:10D6B00004D04026F31A46469E4032431700634684
:10D6C0007A1E97411F4302E6364DAE42CAD08025EE
:10D6D0002D045B422943A6E70843411E8841A6E684
:10D6E000002B00D148E6871A4346B842B641CB1A10
:10D6F00076429E1B33024BD5171A4346BA429241DB
:10D70000591A5242891A072264463A4092E5014367
:10D710000F00791E8F419DE71C000F00203CE74061
:10D72000202B03D04024E31A99400843411E88412E
:10D7300038437CE60022002425E6171A4346BA4205
:10D740009241591A5242891A6446350043E54146CE
:10D750001000144D10E680220024120380E61D0004
:10D760000F00203DEF40BC46202B03D04025EB1A94
:10D770009940084307006346781E87411F4369E7C5
:10D78000871897429B4141445B42C9183500A3E585
:10D790003B003343CED0072231003A4052E600230B
:10D7A0001A00F4E5FF070000FFFF7FFFF0B55746C2
:10D7B000DE464E464546E0B5834607000E03480068
:10D7C00085B092461C00360B400DCD0F002800D1CD
:10D7D0009DE0954B984239D08023F6001B041E43F0
:10D7E000924A7B0F33439946944603006344009367
:10D7F00000230026FF00029323031B0B98466300BF
:10D80000E40F52465B0D019400D1B3E086498B4290
:10D8100000D19EE04246D100802212040A435146C4
:10D82000490F11438B46814952468C460099634407
:10D83000CB1A0021D20000932B0063409A460F2E92
:10D8400000D905E17A4BB6009B599F465B463343AE
:10D85000994600D0B8E002230826002700900293E2
:10D86000CAE7CB463A0002990195019B9A460229E4
:10D8700027D0032900D180E2012944D06D49009BC3
:10D880008C4663441C00002C38DD530700D013E2A3
:10D89000D2085B46DB0109D55946674B19408B46D8
:10D8A0008021C9008C46009B63441C00634B9C4252
:10D8B00007DC5B4664055F075B0217431B0B620DC9
:10D8C00002E000230027584A00211B031C0B0B0D0C
:10D8D0001B05234314055A4A380013401C43534682
:10D8E0006400DB0764081C43210005B03CBC904683
:10D8F0009946A246AB46F0BD0122524201231B1BB2
:10D90000382B00DCADE1002200230027DCE75B467A
:10D91000334399465ED0002E00D18AE13000FEF7F5
:10D920002BFD03000B3B1C2B00DD7BE11D22D31ADA
:10D930005A460100DA4008398E4013005F463343EF
:10D9400099468F403F4B00261B1A009300230293F9
:10D9500052E7414653460B433B499B468C46009B4E
:10D96000634400935B46002B3BD1022300221E43FD
:10D97000022161E7434613439B4637D04346002BC1
:10D9800000D162E14046FEF7F7FC03000B3B1C2B85
:10D9900000DD53E102004146083A914088461D21CE
:10D9A000CB1A5146D9400B0041460B439B46534688
:10D9B00093401A00009B25499C46604403008C4616
:10D9C00063440093002137E70323B14600900C26FF
:10D9D000029311E7002300930133042600270293EA
:10D9E0000AE70323C3461E43032125E701331E43F1
:10D9F0000022012120E700239A46802300271B03F1
:10DA0000094A61E7802349461B03194200D1E2E03D
:10DA10005946194200D0DEE00B431B0317001B0BD5
:10DA2000A246014A50E7C046FF07000001FCFFFF85
:10DA300054FA0000FF030000FFFFFFFEFE07000096
:10DA4000FFFF0F800DFCFFFF01F8FFFFF303000055
:10DA5000D94500D9CBE000D1C6E03C0048460027BC
:10DA6000009B013B00935B46160E1B021E431302F4
:10DA7000984633041B0C9946310C0191FEF788FB44
:10DA80004A4642430B04210C050019438A4207D938
:10DA90008919013D8E4203D88A4201D9851E891910
:10DAA000881A0199FEF774FB09048C464A46210442
:10DAB00064464243090C030021438A4204D9891970
:10DAC000013B8E4200D8F1E02D041D43AB46434696
:10DAD000891A4246280C12041D0C5B46140C2200C5
:10DAE0001B041B0C5A4303946B4344430295684345
:10DAF0001B19150CEB189C4203D980246402A44620
:10DB000060441C0C15041B042D0C20185D19814267
:10DB100077D373D00C1AA24A7D1BAF42BF41944603
:10DB2000009B7F426344E01B1C00864200D1DBE087
:10DB30000199FEF72DFB4A4642430B04290C0700CE
:10DB400019438A4207D98919013F8E4203D88A4274
:10DB500001D9871E8919881A0199FEF719FB090452
:10DB60004A46894629044D464243090C030029438D
:10DB70008A4207D98919013B8E4203D88A4201D9CA
:10DB8000831E89193F04891A3A00039F1A433800FB
:10DB900013041B0C584381460298150C6F434343F2
:10DBA00045434846000C8446DB1963449F4203D931
:10DBB000802040028446654448461F0C00041B0434
:10DBC000000C7D191818A94200D284E000D17FE032
:10DBD00001231A4357E680234A461B0313431B03C2
:10DBE0001B0BAA466F4A6FE6BA4200D935E74B468F
:10DBF000DC0758087B081C43FF0734E70024AF42CA
:10DC000089D247444745A4415B466442A41964183D
:10DC1000013BA6421ED2A0426DD800D1B6E0241A24
:10DC20009B4678E703005A46283B9A4000279146D6
:10DC300088E65846FEF7A0FB203072E60300524605
:10DC4000283B9A4093460022B4E65046FEF794FBE8
:10DC500020309AE6A642E2D1B845DCD9341A9B4678
:10DC600059E71F2B65DC504C0099A4465C46614483
:10DC700008008C4011008240D940501E82410C4364
:10DC800014435A46DA401300620709D00F2222409B
:10DC9000042A05D02200141D9442894149425B1890
:10DCA0001A0262D50122002300270DE68A4200D81D
:10DCB0000AE7831E891907E70F231340042B00D1BD
:10DCC000E6E5171D9742924153429B44FA08E0E56E
:10DCD000002800D1D7E57118531EB14227D3A942BD
:10DCE00015D358D01A0073E7002B00DC04E601239B
:10DCF00000229B44CDE502234744474589415B42CE
:10DD00009C46494289190C19E344241A03E7434607
:10DD10005F0047459B41B8465B429E19023A89190C
:10DD2000A94200D054E7404500D051E7ABE51A00C6
:10DD3000F6E71F215F4649420C1BE740202B07D026
:10DD40001A49009B8C46634418005B4683401A4383
:10DD5000501E82413A4307270023174009D00F2164
:10DD6000002311401400042995D122005F075B02B3
:10DD70001B0BD20817430022A6E5802359461B033C
:10DD80000B431B0317001B0B064A9DE5BD42B2D88F
:10DD90009B460024BFE68045B9D31A00C3E7C046BE
:10DDA000FF030000FF0700001E0400003E04000007
:10DDB000F0B54F464646D6468446C0B58046194E15
:10DDC00018030F034D00000B5C0082463F0B6D0DE6
:10DDD000C90F9146640DDB0F0120B5420AD0B44251
:10DDE00003D0A54201D157450CD01CBC90469946A2
:10DDF000A246F0BD66463E43F7D1AC42F5D154464B
:10DE00001443F2D10120C845EFD1994207D0002D2B
:10DE1000EBD163461F433800471EB841E5E70020B9
:10DE2000E3E7C046FF070000F0B54F464646D6463A
:10DE30004D00C0B50E03C90F8A462C491F035C0074
:10DE40008046360B6D0D91463F0B640DDB0F8D4206
:10DE50001ED08C4216D0002D1ED130438446002C9B
:10DE600001D13A4323D06246002A1AD09A4529D0DC
:10DE7000514602200139084001381CBC90469946A1
:10DE8000A246F0BD39001143E5D002204042F4E73C
:10DE90003043FAD1AC420FD0002C0FD13A43E7D037
:10DEA0000CE00122013B934318000130E5E7634693
:10DEB0000020002BE1D0DBE73A43E6D19A45D7D1E9
:10DEC000A542D5DCA54205DBBE42D1D808D0002052
:10DED000BE42D2D250460123013898430130CCE7EC
:10DEE000C845C5D80020C845F4D3C6E7FF070000E1
:10DEF000F0B54F464646D6464D00C0B50E03C90F95
:10DF00008A462E491F035C008046360B6D0D9146F4
:10DF10003F0B640DDB0F8D4218D08C4211D0002DC9
:10DF200018D130438446002C1ED13A431CD163469D
:10DF30000020002B30D05146022001390840013822
:10DF40002AE039001143EAD0022025E03043FBD11A
:10DF5000AC4226D0002C26D13A4324D1514602208F
:10DF600001390840013817E06246002A0FD09A456F
:10DF7000E1D1A54205DBBE42DDD819D00020BE426A
:10DF80000AD25046012301389843013004E00122AF
:10DF9000013B9343180001301CBC90469946A246B1
:10DFA000F0BD3A43D0D19A45C5D1A542C3DCE0E7E4
:10DFB000C845C0D80020C845E3D3EDE7FF070000FF
:10DFC000F0B55746DE464E464546E0B58346060068
:10DFD0000F03480087B092461D003F0B400DCC0F49
:10DFE000002800D16FE0DE4B984238D08023FF003C
:10DFF0001B041F43730F3B430193DA4B00279946E1
:10E0000000239B46F60081442B0369001B0B5246FC
:10E010009846490DED0F002900D185E0D04B99427B
:10E0200000D173E04346DA0080231B0413435246B9
:10E03000CC48520F84461343524600206144D2001C
:10E0400089442100694000918C46012149448A4657
:10E050000F2F00D990E0C449BF00CF59BF465B469F
:10E060003B43019300D06AE1022308270026814642
:10E070009B46C9E732005846019B61460091022841
:10E0800000D175E0032800D1FEE1012800D02CE189
:10E0900000230027002600253F032A0D3F0BB3482D
:10E0A00012053A4302401B051343009A5B00D10757
:10E0B0005B080B433000190007B03CBC9046994602
:10E0C000A246AB46F0BD5B463B43019300D12FE136
:10E0D000002F00D1A5E13800FEF74EF903000B3BFD
:10E0E0001C2B00DD96E11D22D31A5A460100DA40AE
:10E0F0005E4608398F4013008E403B4301939C4B92
:10E1000000271B1A994600239B467DE7414653464C
:10E110000B4393498C46E144002B00D01AE10222C4
:10E120000220174300228CE7134300D10DE1434640
:10E13000002B00D181E14046FEF71EF902000B3AA8
:10E140001C2A00DD72E10100434608398B409846E5
:10E150001D239A1A5346D3401A004346134352468E
:10E160008A404946081A824989468144002068E766
:10E170007B4B002700268EE7140C1204120C1100B2
:10E18000370C3604350C794328008C462E0060434A
:10E190006044834656432100300C804658467943FC
:10E1A00040440291844506D98846802149028C4624
:10E1B000E044414602913604010C360C00048B46C3
:10E1C00081191E0C1B041B0C0391190079438C460A
:10E1D000280075436544A8465843050C45447743D9
:10E1E000A94203D9802149028C466744290C8C46F8
:10E1F00039000004000C2D042D186144AB44059136
:10E200005946049101990F043F0C080C3900514301
:10E210004243904602008C46090C8B4662437C4385
:10E2200044445C44A04503D98021490288464244C5
:10E23000210C884661460904090C8C463900594373
:10E24000434370437E430F0CF6182404BE19644404
:10E2500042448C46B34203D980235B029846404433
:10E26000029B61469846049B370443449B46AB455A
:10E27000AD416B420D0405992D0C8C467F19674406
:10E28000FD18A8465D462D19A542A4419346644257
:10E29000A446C344DC448F42BF4198459B4193450B
:10E2A0009241A445A4415B427F421F43360C524237
:10E2B0006442BF192243BF18624638184302D20D88
:10E2C000039913436A020A43501E82416146ED0DD1
:10E2D0002A434E023243D90100D4B3E0012650084C
:10E2E00032400243DE0732435B08224C5444002C88
:10E2F00062DD510709D00F201040042805D0101D01
:10E300009042924152429B180200D90104D58024C8
:10E310001948E400034054441848844200DD27E7CC
:10E320005E075B02D2081F0B630516435B0DB2E666
:10E33000002399460133042700269B4664E6032305
:10E34000019781460C279B465EE601220120174378
:10E35000002276E6032303201F43434671E6C046AE
:10E36000FF07000001FCFFFF94FA0000FFFF0F8091
:10E370000DFCFFFFFF030000FFFFFFFEFE07000094
:10E380000023802700933F030026434B83E6019B35
:10E390003200A446584670E6AC466EE680270199E6
:10E3A0003F0339422DD03B422BD11F433F033F0B4C
:10E3B00000951600384B6EE601252D1B382D00DD2B
:10E3C00066E61F2D40DC35481C0050441600824094
:10E3D0008440EE40501E824134431443EB406207B8
:10E3E00009D00F222240042A05D02200141D944295
:10E3F000804140421B181A023ED501230027002607
:10E4000049E68027019B3F031F433F033F0B0094D6
:10E41000214B40E603005A46283B9A4000260192D1
:10E420006DE65846FDF7A8FF203057E60300524638
:10E43000283B9A401300002293E65046FDF79CFFCC
:10E4400020307BE6CA4650E71F201E004042041BD6
:10E45000E640202D03D0124C5444A3401A43501ED2
:10E460008241324307260027164009D00F2000239F
:10E47000104014000428B9D122005E075B021F0B74
:10E48000D2081643002306E680273F031F433F03BD
:10E490003F0B1600004BFEE5FF0700001E040000C6
:10E4A0003E040000F8B557464E464546DE460C0091
:10E4B0000903E0B5490A460F5F0031431E03DB0F35
:10E4C000760A9B46530F3343C84E6500C000E40FE5
:10E4D000D2006D0DA24681467F0D9C469046B74204
:10E4E00000D1B9E05B46012673409B46EE1BA34575
:10E4F00000D183E0002E63DD002F00D0B1E0634641
:10E50000134300D123E1731E002B00D0BAE1861A19
:10E510006346B04280410125C91A4042091A0B02E4
:10E5200000D447E149024B0A98464346002B00D1EC
:10E5300089E14046FDF720FF0300083B1F2B00DD6B
:10E540007CE120223000D21A4146D040994002009E
:10E550009E400A439D4200DD6AE15D1B6B1C1F2B40
:10E5600000DD94E1202110003500C91A8E40DA4008
:10E570008840DD40711E8E4111000722284300258E
:10E5800006433240002A09D00F233340042B05D024
:10E59000331DB342B641764289191E000B0200D4E6
:10E5A0003DE26A1C914B55056D0D9A4200D119E16F
:10E5B0008F4AF6080A40570752023743120B9BE076
:10E5C000002E00D0C5E06E1C7605760D012E00DC15
:10E5D00048E16746861ACB1BB042BF417F42B8462E
:10E5E0001F004346FF1A3B00B8461B0200D55FE1FF
:10E5F00037439AD100220024002579E0002E00DC68
:10E60000FAE0002F00D18DE0784B9D4267D0802347
:10E6100067461B041F43BC46382E00DC52E16346AC
:10E6200013435A1E93411E188642804140420918E6
:10E630000B0200D4BEE06D4B01359D4200D1D2E00B
:10E640006B4A73080A4001210E401E435108D3074C
:10E6500007221E43324095E71E00164300D045E7CF
:10E6600040E7624B9D423AD0802367461B041F431C
:10E67000BC46382E00DDEBE01F2E00DC3AE1330013
:10E680006746203BDF403B00202E05D04027BF1BC4
:10E690006646BE40324390464646721E964133431C
:10E6A000DAE0002B00D114E26346134300D168E1A5
:10E6B00080234E07C008C9081B030643194208D02F
:10E6C0006046C008184204D163460100D2085E07C4
:10E6D0001643F3009946C900720F444D11434B464F
:10E6E000DE08424B4F073743CA089D4200D16EE017
:10E6F00012036D05120B6D0D00211203130B0A0D91
:10E7000012051A433B4B2D0513402B435B00E407D6
:10E710005B082343380019003CBC90469946A2464A
:10E72000AB46F8BD6346134311D0731E002B00D0D7
:10E7300007E186188642804161444042091801255C
:10E740000B0237D502257BE73E0061469146350036
:10E75000C5E75C46002D00D0E1E00B000343F3D099
:10E76000731C00D1ACE1214B9F4200D13AE1F3434D
:10E77000382B00DD6FE11F2B00DD8CE120250E0022
:10E78000ED1AAE40B0460600AA46DE404546354387
:10E790002E005546D940A8406346451EA8415B1A45
:10E7A0009C463043161AB242924163465242991A2D
:10E7B0003D00B4E607223240002A00D0E4E60B4BCD
:10E7C000F6084F073743CA089D4200D090E73B0048
:10E7D000134300D1A6E180231B031A431203120B3B
:10E7E000024D89E715000022002785E7FF0700009A
:10E7F000FFFF7FFFFFFF0F80002E00D0C7E06B1CE4
:10E800005E05760D012E00DCF0E0C84DAB4200D174
:10E81000B9E085180A00854289416244494251188D
:10E820000722CE076D082E43490832401D00A9E695
:10E83000BF49ED1A114007223240A3E632002838C2
:10E840008240002686E63000FDF796FD203073E614
:10E85000634613435A1E9341C61AB0428041404258
:10E86000091A5CE60E00674606431743002D5ED189
:10E87000002E00D0F3E0002F00D11EE15C4661467F
:10E8800091462CE7A94FBE427BD01E00F1E6100056
:10E890001F3DE840202B03D04021CB1A9A4016435D
:10E8A000731E9E410722064332400021002583E764
:10E8B000161A6346B2428041591A40420B1A9846D2
:10E8C0005C4632E61F2E00DDABE02027BB1B9A46DC
:10E8D00063465746BB40994613004F46F3401F43DB
:10E8E0003B005746BA40571EBA4113436246F240B6
:10E8F000891898E62027BB1B9A4663465746BB40BB
:10E90000994613004F46F3401F433B005746BA4019
:10E91000571EBA4113436246F240891A9CE7834B63
:10E920009F425FD080252D047342294320E7002EAB
:10E930000CD1002F00D1D0E05C46614691467B4D62
:10E94000CDE67A4FBE421CD01E0065E6002F18D0DF
:10E95000C0084E0706438020C9080003014208D0C2
:10E960006346DC08044204D12100DA46D2085E077F
:10E970001643F300994601245346C900720F114310
:10E980001C406A4DABE61D0000220027B4E6002DB6
:10E9900059D10B00034300D1D6E6731C00D1B2E07D
:10E9A000624B9F421ED0F343382B6FDC1F2B00DDE0
:10E9B00097E020250E00ED1AAE40B0460600AA46AC
:10E9C000DE40454635432E005546A840D940451EF9
:10E9D000A8418C440643B618964292415142614484
:10E9E0003D0025E63D006146914678E60B00034375
:10E9F000002D00D055E6002BF5D06346134300D11F
:10EA00006DE6861886428041614440420918002222
:10EA10000B0200D4D0E6464B01351940B2E5B146B1
:10EA20005DE633006746203BDF403B00202E05D0EB
:10EA30004027BF1B6646BE40324390464646721E84
:10EA400096413343EFE5394B9F42CBD080252D04CF
:10EA500073422943A8E70843411E8841A2E6002FDC
:10EA600000D13CE66346861ACF1AB0429B415B4216
:10EA7000FB1A98461B024ED5161A6346B2429241C3
:10EA8000591A5242891A5C4600227BE501430E0066
:10EA9000711E8E419FE71D000E00203DEE40B046E6
:10EAA000202B04D04025EB1A994008438146484664
:10EAB0004346411E8841184374E60022002417E6AD
:10EAC000161A6346B2429241591A5242891A3D00BF
:10EAD00025E561469146154D01E68022002412038A
:10EAE00079E61D000E00203DEE40B046202B04D0FC
:10EAF0004025EB1A9940084381464E464346711E15
:10EB00008E411E4367E7861896429B4161445B42F3
:10EB1000C9183D008CE547463743CED00722414611
:10EB2000324049E600273A00E6E5C046FF0700000C
:10EB3000FFFF7FFF30B5144D0A034B00120B5B0D36
:10EB4000C90F0024AB4211DD104CA34210DC80241D
:10EB5000640322430E4CE41A1F2C0CDD0D48C31A2B
:10EB6000DA4013005C42002900D11C00200030BDB7
:10EB7000094BCC18FAE7094DE040AC4663449A4093
:10EB800013000343EEE7C046FE0300001D0400002F
:10EB90003304000013040000FFFFFF7FEDFBFFFFC5
:10EBA00070B500282DD0C317C5185D40C40F2800CC
:10EBB000FDF7E2FB154B1B1A5B055B0D0A2815DD03
:10EBC0000B38854000222D032D0B002110002D0352
:10EBD0000A0D2D0B12052A430D4D1B052A40134328
:10EBE0005B00E4075B082343190070BD02002900A5
:10EBF000153291400A000B21081AC5402D032D0B38
:10EC0000E3E70024002300250022DEE71E040000C5
:10EC1000FFFF0F8010B5041E25D0FDF7ADFB144B90
:10EC20001B1A5B055B0D0A2812DD0B38844000229D
:10EC30002403240B0021100024030A0D240B1205C9
:10EC400022430C4C1B05224013435B00590810BDA6
:10EC500002002100153291400A000B21081AC4401D
:10EC60002403240BE6E7002300240022E2E7C04649
:10EC70001E040000FFFF0F80A30000000000000042
:10EC8000FC3F0150FC3F0250FC3F0350008001500C
:10EC900000800250008003502024282C383C40443F
:10ECA000484C0207020802010003010903040204A0
:10ECB00002050305000600070008000A0100000025
:10ECC0000000E0FE422EE63F0000E0FE422EE6BFDE
:10ECD000763C7935EF39EA3D763C7935EF39EABD56
:10ECE000000000000000E03F000000000000E0BF66
:10ECF0000000000000000000000000000000008094
:10ED000000000040FB21F93F000000002D44743E4C
:10ED1000000000809846F83C0000006051CC783B31
:10ED200000000080831BF0390000004020257A3865
:10ED3000000000802282E336000000001DF36935E8
:10ED4000000000000000F03F000000000000F83F5D
:10ED5000000000000000000006D0CF43EBFD4C3E59
:10ED600000000000000000000000004003B8E23F87
:10ED70004FBB610567ACDD3F182D4454FB21E93FD3
:10ED80009BF681D20B73EF3F182D4454FB21F93FC2
:10ED9000E2652F227F2B7A3C075C143326A6813C48
:10EDA000BDCBF07A8807703C075C143326A6913CF3
:10EDB000000000000000F87F000000000000F07F6D
:10EDC0000000000000000000000000000000000043
:10EDD000010000000000F03F8A1EBD726654B6407C
:10EDE0004E543EF2A6EFCCC078844D13BFE9CB4021
:10EDF0004FFA050429CCB8C06C5C8AE26E56944088
:10EE0000CC5CF6234F0B5BC0563BD76877D80440E9
:10EE1000AC5913DC0D687EBFA38C9F98E6E76C3E6F
:10EE20005610B1E5EB4731BE182D4454FB21094083
:10EE3000000000000000000000000000000024406E
:10EE40000000000000000000000000000CFA0000BC
:10EE500012FA000018FA00001EFA000024FA00005E
:10EE60002AFA000030FA000036FA00003CFA0000EE
:10EE700042FA000048FA00004EFA00000606103878
:10EE80007C101010050554341C1615060611514A45
:10EE90002A2410060610242A4A5111080804423E6A
:10EEA00002023E42200505007F3E1C080303403E4F
:10EEB00001070760584641465860040463554941BC
:10EEC000020225520505080C7E0C08050510307E4F
:10EED000301006061010107C381004040404000ED4
:10EEE0000505605068444005056000600060000250
:10EEF00001015F03030600060505147F147F140556
:10EF000005042A7F2A1005052313086462050536C7
:10EF10004951225001010602023E410202413E05D2
:10EF2000054428102844050510107C1010020240EA
:10EF30003005051010101010020260600303601805
:10EF40000605053E5149453E050500427F40000546
:10EF500005625149494605052241494936050518CA
:10EF600014127F100505274545453905053C4A49DA
:10EF7000493005050171090503050536494949363A
:10EF80000505064949291E020242000202402205E7
:10EF9000050814142222050514141414140505225E
:10EFA000221414080505020151090608083C02391B
:10EFB00045453D417E05057E0909097E05057F49D8
:10EFC00049493605053E4141412205057F4141221F
:10EFD0001C05057F4949494105057F0909090105C6
:10EFE000053E4141513205057F0808087F03034172
:10EFF0007F410505304040403F05057F0814224110
:10F0000005057F4040404005057F020C027F050555
:10F010007F0408107F05053E4141413E05057F09FB
:10F0200009090605053E4151215E05057F0919299B
:10F030004605052649494932050501017F010105BB
:10F04000053F4040403F0505071860180705057F4C
:10F050002018207F05056314081463050503047850
:10F0600004030505615149454302027F410303063C
:10F0700018600202417F05050804020408050540E6
:10F080004040404002020204040420545478040426
:10F090007F44443804043844444404043844447FDE
:10F0A0000404385454580303087C0A040418A4A424
:10F0B0007C04047F0404780303447D400202847DC1
:10F0C00004047C10284401017F05057C0438047C7D
:10F0D00004047C0404780404384444380404FC44E4
:10F0E00044380404384444FC04047C080404050542
:10F0F00008545454200303047E4404043C40407CE0
:10F1000005050C3040300C05053C403C403C0505F5
:10F110004464384C4404041CA0A07C030364544C95
:10F1200091F800000000000097F8000000000000C7
:10F130009BF8000000000000A0F80000A4F8000008
:10F14000A8F8000000000000ACF80000AFF80000D4
:10F15000B3F800006BF70000B8F80000BEF800003C
:10F16000C2F800006FF7000000000000C6F80000C1
:10F17000CAF80000CEF80000CEF80000D4F8000075
:10F18000D8F8000010FA0000DCF80000DEF80000FB
:10F19000E0F80000BBF7000072F90000E2F80000A0
:10F1A000E4F80000E6F80000E9F80000EBF80000E1
:10F1B000EDF80000E7F80000CBF9000005FA0000C8
:10F1C0000AFA000000000000EFF80000F3F8000069
:10F1D000F7F8000000000000F9F8000001F9000055
:10F1E000A2F80000000000000000000005F9000087
:10F1F0000CF9000009F900000EF9000018F90000F0
:10F2000059F900000000000022F900002AF900006E
:10F2100058F70000BEF60000BEF6000033F900000B
:10F220003AF9000041F9000044F900002FF900000C
:10F2300067F7000047F900004BF9000056F700009F
:10F2400063F7000051F9000056F9000052F7000082
:10F250005FF700005BF9000060F9000068F900004A
:10F260006AF900000000000000000000000000003B
:10F2700070F900000000000074F9000078F9000047
:10F280007EF900000000000081F9000084F9000010
:10F290008AF900008EF90000B6F6000092F900002D
:10F2A000A4F900000000000098F900009DF900009A
:10F2B000A3F90000A6F90000A6F90000ADF90000CE
:10F2C000AFF90000B3F90000B8F90000BBF9000085
:10F2D000CEF90000BEF90000C4F90000C7F9000033
:10F2E00057F90000CAF90000CDF90000D2F900007A
:10F2F000D5F90000DAF90000DFF900000000000095
:10F3000000000000E4F90000E9F90000EEF9000057
:10F31000F3F90000F8F90000FDF9000002FA00001E
:10F3200007FA0000000000008D7E000011B200000E
:10F33000E1540000757D0000C554000059B1000083
:10F34000A59B0000357D0000A95400000564000065
:10F35000217A0000D57C0000A1960000B163000076
:10F36000F9770000717C000051970000ED8E0000DD
:10F37000F57200006164000011820000118200003B
:10F38000FD5A0000C59C0000B35B0000A95B0000B3
:10F390008B5B00006D5B0000355B00009F5B000035
:10F3A000815B0000635B000029710000955B000039
:10F3B000775B0000595B0000C970000029720000F3
:10F3C00089720000DD7B00008D7E00003DB20000F0
:10F3D000F9A300003DA5000000000000657F0000CB
:10F3E0008D54000033A5000000000000CD91000006
:10F3F0006D54000029A50000BD6E0000197F0000BB
:10F40000018500001FA500005D540000615600004A
:10F410002D83000015A500004D8E00004D8E0000CC
:10F420007D5400007D530000156E00005F54000005
:10F430003194000019960000716C0000B16F00005B
:10F44000499300009195000031620000356F000083
:10F4500061920000FD940000156C000071630000D3
:10F460005DB200002DB300008D7E000095680000A5
:10F47000E9530000C56B000000000000915300003C
:10F48000D1530000856B000000000000C96100003E
:10F49000B9690000FD6A0000E9660000B18800005B
:10F4A0001D690000A96A00007F530000595F000039
:10F4B000BD680000496A0000916100009161000090
:10F4C000F5610000156A0000016100008153000031
:10F4D0002D9100004D540000CD5F000099670000A1
:10F4E000859000003D540000E96500004167000080
:10F4F000ED8F00002D5400003965000035800000BC
:10F50000AD53000009540000A5980000F9980000D0
:10F510004D990000B1990000159A00005D9A000015
:10F52000A59A0000F99A0000FB21F93FFB21094050
:10F530007CD91240FB2119407A6A1F407CD92240B5
:10F54000BBFD2540FB2129403A462C407A6A2F40DA
:10F550005C4731407CD932409C6B3440BBFD354028
:10F56000DB8F3740FB2139401BB43A403A463C40E0
:10F570005AD83D407A6A3F404C7E40405C4741400B
:10F580006C1042407CD942408CA243409C6B44406A
:10F59000AC344540BBFD4540CBC64640DB8F4740C1
:10F5A000EB584840FB21494083F9A200444E6E00CD
:10F5B000FC291500D1572700DD34F50062DBC000BF
:10F5C0003C999500419043006351FE00BBDEAB00C7
:10F5D000B761C5003A6E2400D24D42004906E000F2
:10F5E00009EA2E001C92D100EB1DFE0029B11C007F
:10F5F000E83EA700F535820044BB2E009CE984005C
:10F60000B4267000417E5F00D691390053833900E3
:10F610009CF439008B5F840028F9BD00F81F3B0083
:10F62000DEFF97000F980500112FEF000A5A8B009C
:10F630006D1F6D00CF7E360009CB2700464FB70007
:10F640009E663F002DEA5F00BA277500E5EBC70014
:10F650003D7BF100F739070092528A00FB6BEA000C
:10F660001FB15F00085D8D00300356007BFC460033
:10F67000F0AB6B0020BCCF0036F49A00E3A91D006C
:10F680005E619100081BE60085996500A0145F008B
:10F690008D40680080D8FF0027734D0006063100BA
:10F6A000CA561500C9A873007BE260006B8CC000CD
:10F6B000544553543A00524E44002869290052419F
:10F6C0004E202300257500256425732025733F00F7
:10F6D0002564257320257320257300256425732058
:10F6E0002573004E414E002D494E46002E252530F3
:10F6F00025646C6C7500256C6C75002045256400D4
:10F700002573256325730025732020256325730049
:10F710002573202B25732025630025732025732056
:10F72000256300436865636B20466C61673A00435C
:10F730006C65617220466C61673A005365742046BF
:10F740006C61673A0044656C657465205072676D42
:10F750003A004953470044534500582019200045BA
:10F760004E4700534349004649580053544F0052F6
:10F77000434C00476F20546F204C424C3A00475492
:10F780004F204C424C3A00476F20546F204C696E1A
:10F79000653A00257320005F0050726F6772616DDB
:10F7A0002025630050726F6772616D2025640052DE
:10F7B000756E6E696E67002E202E202E00593A005D
:10F7C000583A0044697669646520627920300049BE
:10F7D0006E76616C69642074797065004E6F206C80
:10F7E0006162656C004C6162656C20657869737458
:10F7F00073004F7574206F66204D656D004D617804
:10F8000020497465727320526561636865640055B0
:10F810007365722061626F72746564004E6F20724E
:10F820006F6F740041626F72740068006825630036
:10F830006600726164006772002010002050002092
:10F840001C2000201020005069636B204C424C3A71
:10F850000052756E204C424C3A00475342204C42B5
:10F860004C3A00494E54454752415445204C424C75
:10F870003A00534F4C5645204C424C3A00256420E8
:10F88000005061737465204D656D6F72793A0D0A91
:10F8900000456D70747900522F530053515254003B
:10F8A0004753420047544F00655E5800521B0053B7
:10F8B000494E0031305E5800582019205900434FFE
:10F8C0005300595E580054414E00312F5800454EA8
:10F8D0005445520045455800434853003100340018
:10F8E000370035003800182B00330036003900503F
:10F8F0005345004C424C004100434C4541522018B6
:10F90000004859500044494D004652414300434C81
:10F910004541522052454700436F6D7020636F6E22
:10F920006A0072756E54696D650059202B20695804
:10F93000201900524553554C54004D4154524958DA
:10F94000007821001C5200792C72001C482E4D5367
:10F95000004C2E522E001C5241440050792C78004D
:10F960005265201920496D001600534F4C56450032
:10F97000585E320052544E00485950201D004C4EE3
:10F9800000521A0053494E201D004C4F4700494E6B
:10F990005400434F53201D00434C20580054414E07
:10F9A000201D001725004C415354205800140041DD
:10F9B0004253004D45414E001C50005346005354E5
:10F9C000444556001C4800434600182D001C444581
:10F9D0004700463F00475241440043792C78005489
:10F9E0004553540053544F2B0053544F2D00535440
:10F9F0004F2A0053544F2F0052434C2B0052434C7C
:10FA00002D0052434C2A0052434C2F005820112005
:10FA1000300058203E20300058203C203000582034
:10FA20001220300058201320300058203D2059006B
:10FA300058201120590058203E20590058203C20C1
:10FA400059005820122059005820132059005820DE
:10FA50003D20300050DA0000C2D8000006D9000076
:10FA60006AD8000006D90000F6D9000006D90000C7
:10FA70006AD80000C2D80000C2D80000F6D9000041
:10FA80006AD8000062D8000062D8000062D8000086
:10FA900004DA000078E100007AE000007AE000007B
:10FAA00098E3000074E0000074E0000080E30000D0
:10FAB00098E3000074E0000080E3000074E00000C0
:10FAC00098E300008EE300008EE300008EE3000068
:04FAD0009CE30000B3
:08FAD40008C7FF7F01000000DC
:10FADC000508107A7CEE00004D000000583A001F1B
:08FAEC002C000000C400001012
:040000030000C041F8
:00000001FF
